:1000000000400020056000004560000047600000DF
:1000100000000000000000000000000000000000E0
:100020000000000000000000000000004960000027
:1000300000000000000000004B6000004D60000068
:100040004F6000005D470000816400004F600000C9
:100050004F600000000000004F6000004F60000093
:100060004F600000516700004F6000004F600000CB
:100070004F6000004F6000004F6000004F600000C4
:100080004F600000E96800004F6000004F60000012
:100090004F6000004F6000004F6000004F600000A4
:1000A0004F6000004F6000000000000000000000F2
:1000B0000000000000000000000000000000000040
:1000C00010B5064C2378002B07D1054B002B02D02E
:1000D000044800E000BF0123237010BD4C02002043
:1000E00000000000B0D00000044B10B5002B03D07E
:1000F0000349044800E000BF10BDC04600000000F6
:1001000050020020B0D00000164B002B00D1144B41
:100110009D46402292029A1A924600218B460F4633
:100120001348144A121A0AF087F90F4B002B00D01B
:1001300098470E4B002B00D0984700200021040068
:100140000D000D48002802D00C4800E000BF0AF066
:1001500033F92000290006F0B1F90AF007F9C0468A
:100160000000080000400020000000000000000027
:100170004C020020A02F0020000000000000000022
:100180000123034010D104280CD90268120909D0B8
:10019000531E9B001A1DC1180979002902D0013392
:1001A0009342F8D1180070470023FBE70378002B37
:1001B00003D05AB2002A01DB013070473F2293433B
:1001C000C03B59424B41C01803789343802BF4D174
:1001D0000130F9E710B500240378002B01D120008D
:1001E00010BDFFF7E3FF0134F6E770B5002204000D
:1001F0000D00411C092002F00DFF002806D001234C
:100200006200134343600023A34200DB70BD9A00E9
:10021000A958821891600133F6E770B5012803DC14
:100220001C2000F093FE70BD01230D6811201D42BB
:10023000F7D04868184206D1042804D90F23026871
:100240001340042B01D00E20EBE702F04DFD6D10A2
:100250000400002D03DDFFF7BDFFA84206DA1220DF
:10026000DFE72000FFF7A2FF0400013D012DF8D1D8
:1002700020787F2809DDDF280BDCF8233F22DB0014
:10028000800118406378134018430123400018434D
:10029000C9E7EF280BDCFC22637812019B011340B5
:1002A0003F220007000C0343A0781040ECE7F7283A
:1002B00012DCFC22637892021B031340E0228004CC
:1002C000520310403F221843E3781340FC220343BB
:1002D000A07812018001E8E701204042D5E7F0B59F
:1002E000070085B00D001C20012F06DD4C6801239E
:1002F00022001A40019203D10D2000F027FE54E0A5
:10030000022F02D08A681A42F6D001232E681E42BC
:1003100000D07EE0042E00D87BE01C41002C00DCE5
:100320001C000F2332681340092B29D173685B101E
:100330000193022F05D0AB68019A5B109A4200DD51
:100340000193019B01221F1B0137FB43DB171F4059
:10035000791C092002F05EFE061E09D001237F00F1
:100360001F4303002A68083347600199A14202DA5B
:10037000300005B0F0BD0134A100515802C3F4E7CC
:10038000042B46D1300002F0AFFCFFF723FF0290B0
:10039000022F04D0AB685B10984200DD0293029BF1
:1003A0009C4204DD002002F0A1FE0600E0E73000E0
:1003B00002F09AFC0700019B9C4222DC300001976E
:1003C00002F092FC03903800FFF7F0FE029B01342C
:1003D0000700A342F7DA019BC71A380002F086FE35
:1003E000061EC5D002F080FC0400286802F07CFCE8
:1003F000039A019B991A41183A0020000AF000F86C
:10040000B6E73800FFF7D2FE019B070001330193E6
:10041000D1E7212071E7F8B54D680F00EB0706D44E
:10042000042D04D90F232E683340092B03D00B2051
:1004300000F08CFDF8BD6B6836095C10731EA3429A
:100440000FD80321200007F0B3FE6421642803DCE9
:100450000100032800DA03212800891902F00AFEAE
:1004600005002B6800201B09013B9C42E2D23A6840
:10047000A31C9B005A510123013464001C436C608F
:10048000D8E7F0B585B0012803DC1C2000F05EFD44
:1004900029E001254F682A00022806D08B682B42EC
:1004A00003D05D10002D00DC15000124274200D090
:1004B00074E0042F00D871E00F223B680E681340EF
:1004C000042B25D1264205D1042E03D933681340CD
:1004D000042B01D00E20D9E73800FFF751FEA842C7
:1004E00003DA0120404205B0F0BD380002F0FCFB09
:1004F0000700300002F0F8FB013D010078190AF016
:100500003AFB0028EDD0C01B013040002043EAE751
:10051000092B43D17B685B1000939D42E1DC3000E6
:1005200020402ED1042E2BD90F22336820001340F7
:10053000042B26D1300002F0D7FB0F2325000290B8
:100540000393631C01939B00F858864202D1640018
:100550002800DBE728420ED104280CD90368039A4F
:100560001340042B07D102F0BFFB010002980AF0F0
:10057000D5FA0028EBD0019C009B9C42E1DDB0E75E
:100580002000431C9A00BA58B24202D14000012414
:10059000BCE71800009B9842F3DDA2E7212075E735
:1005A00010B502F085FB43000120184310BD000088
:1005B00010B57F2902DC0170013010BD1A4B994241
:1005C0000CDC40238A115B42134303703F230B4032
:1005D00080214942194341700230EEE7134B9942A2
:1005E00010DC20230A135B4213433F248022037054
:1005F0008B1152422340214013430A4343708270BF
:100600000330DAE70A4B9942D7DCF0230370603BF2
:100610004370113B8A11FF3B1A4382703F22114005
:100620001943C1700430C8E7FF070000FFFF000056
:10063000FF0F0100F0B50D0085B0002803DC1C2081
:1006400000F084FC0DE009680122080010400AD087
:1006500002AC11412000FFF7ABFF011B200002F0AC
:1006600051FD04001AE004293FD90F230C682340F0
:10067000092B3AD14B685B10019303239C46019BE5
:100680009A420EDD02F032FD041E07D02E680125CD
:1006900002F02AFB2F00019B9D421DDD200005B0CA
:1006A000F0BD01329300CC580123234001D10D202D
:1006B000C6E764107F2C0DDD0D4E0223B44209DD28
:1006C0000C4E6346B44205DD00270B4EE30FA642F5
:1006D0007B419B00C018D2E70135AB00F15839428D
:1006E000E5D04910FFF764FFD5E72120A8E7C04611
:1006F000FF070000FFFF0000FF0F010010B504001E
:100700000120084010D104290DD90F230A68134095
:10071000042B08D1080002F0E7FA010020000AF0DB
:10072000FDF94342584110BD0020FCE7F7B50F002A
:10073000012803DC1C2000F009FCFEBD01264D68E9
:100740002E4006D1042D04D90F222B681A40092A05
:1007500001D00B20EFE76A681B095410A34200D8B0
:100760005C1E39681E48FFF7C9FF0123019000286D
:1007700013D139681B48FFF7C1FF002811D0002CA6
:100780000DD00123621C013C9C4092005351234335
:100790006B6004E00136B200AB50B442FADA0020DC
:1007A000CBE73B680D20DA07C5D55B10002B11DDC8
:1007B0009C420FDB9B00A200291DEB188918043313
:1007C000994209D10123013C9C40AA181C43536063
:1007D0006C60E4E71220AEE758681860EFE7C046A7
:1007E00093BA000097BA0000002310B50C000B70FC
:1007F000C30705D50D49421020000AF061F908E051
:100800000B49002802D0042804D10A4920000AF02C
:1008100077F910BD0428FCD90F2302681340042B7C
:10082000F7D102F061FA04490200E5E7ECC20000EA
:100830009CBA0000A2BA0000A7BA0000F0B593B0BD
:100840000390030002911C20012B1DDD029B01255A
:100850001B681C002C4000D0A8E0042B00D8A5E0A9
:100860001A680F231A40092A48D10194019A029963
:1008700092008A5816002E4005D1042A03D9106828
:100880001840092804D0222000F060FB07002CE06B
:1008900052685210A418019A013201920199039AE8
:1008A0008A42E3D1611C012202F0B4FB071E01D190
:1008B00000271AE064002543456005000835029AC8
:1008C000B300D1584B680A685B1012099A4200D8ED
:1008D000531E002293420BDCDA43D21713409B00D5
:1008E000ED18019B01369E42E9DB380013B0F0BDE4
:1008F00090000C18A46801322C50EBE7042A55D163
:100900002F0026001D00029AB300D058384237D17C
:10091000042835D903682B40042BB4D1FFF730FCF1
:10092000039B01362418B342EDD1200002F0DEFB18
:10093000071EBDD0039B029D9B00EB18041D029374
:1009400001232E681E4222D1042E20D90F223368A3
:100950001340042B0DD13000FFF712FC0190300042
:1009600002F0C2F9019A0100200009F049FD019B43
:10097000E418029B0435AB42E2D100232370B4E7B4
:1009800005A9FFF731FF05A80AF0DAF8C8E705A9BD
:100990003000FFF729FF05A80AF0D2F80600020090
:1009A00005A9200009F02CFDA419E2E7212000F0A0
:1009B000CDFA7DE7F0B50D0095B0002806DC1C20CF
:1009C00000F0C4FA0400200015B0F0BD0C6801214D
:1009D00023000B40009306D1042C04D922680F3366
:1009E0001A40092A01D00B20EAE7626852100392EC
:1009F000002A03DC009802F079FBE3E73F4A01920A
:100A000001280BD06868084208D1042806D902687A
:100A10001340042B02D102F067F9019001980AF00B
:100A20008FF806000F27039B0834013B04935E43B5
:100A3000039B02909B001B19059301232068184219
:100A400051D104284FD903683B40042B52D1FFF702
:100A500097FB059B04343618A342EED1300002F018
:100A600045FB041EAFD02B680593029B002B03D0DF
:100A7000686802F039F90190200002F035F90500AC
:100A8000009B059A9B00D3189F68380002F02CF950
:100A9000012306001F4201D1042F04D807A9380002
:100AA000FFF7A2FE07AE30000AF04AF80700020086
:100AB0003100280009F0A4FC029BED19002B0AD09C
:100AC000049B009A934206DD2800029A019909F0DE
:100AD00097FC029BED18009B01330093009A039B47
:100AE0009342CDD16FE707A9FFF77EFE07A80AF072
:100AF00027F8AEE702F0F8F8F9E7C046F6BD0000C7
:100B000010B50024A04207DD0B6801341C4003D05F
:100B10005C10E343DB171C40611C0122092002F03A
:100B200079FA002803D0012364001C43446010BDFF
:100B30000B6870B518000125284032D1042B30D93C
:100B40000F241A6849681440092C16D15C681209F0
:100B50002C41A24200D8541E844205DC02200132FE
:100B6000904206DB00200FE085005D19A96001308E
:100B7000F2E7840019510130F2E7032C11D1294228
:100B800003D1132000F0E2F970BD4910FF29F8D815
:100B90001209043392009A189A42E3D9197001336A
:100BA000FAE70B2000F0D2F9DCE700000123F7B5EB
:100BB00000264D680F002B400093B3420DD11E005C
:100BC000042D0AD90F222B681A40092A0FD16A680E
:100BD0001B095610B34200D85E1E3968CB0713D5E7
:100BE0004C10002C01DDA64219DA12202EE0042A56
:100BF00004D12800FFF7C4FA0600EEE7009E032A9E
:100C0000EBD11E09B600E8E72E48FFF777FD002874
:100C100014D009F0F1FE310007F0B0FB4C1C009B32
:100C2000002B4CD1042D4AD92A680F331340092BCD
:100C300010D10134A40064592000FEBD3968224857
:100C4000FFF75CFD34000028E9D1113000F07EF997
:100C50000400F1E7042B2AD1280002F045F8060031
:100C6000FFF7B8FAA042C0DB012C1ADC280002F022
:100C70003BF800903000FFF799FA851B280002F03E
:100C800035FA041ED8D002F02FF80190786802F0EF
:100C90002BF8009B2A00F11A4118019809F0B0FBCB
:100CA000CAE73000FFF782FA013C0600DCE7032BBD
:100CB00005D12C19E478023B64001C43BCE70B20EF
:100CC000C4E7C0468CBA000097BA0000F7B54C687C
:100CD0000F000120210001402AD1042C28D90F2225
:100CE0002368BE681A40092A13D162681B0955108F
:100CF0000191AB4200D85D1E39682848FFF7FEFC21
:100D0000002829D00F2322681340092B19D1012371
:100D100013E0032A0CD1064203D1132000F016F988
:100D2000FEBD72100192FF2AF7D81D09AD00E3E75E
:100D30000B20F3E701339A00A6509D42FADA002017
:100D4000EEE7032BFBD1230001331A1BAA42F6DC8A
:100D50006A461279DA70F7E73968CB0706D5491089
:100D6000002901DD8D4209DA1220D7E70C48FFF790
:100D7000C5FC2900002801D11130CFE70F232268DC
:100D80001340092B03D1013189000E51D7E7032B02
:100D9000D5D16B461B796418E370D0E793BA000095
:100DA00097BA000010B501240868204216D1042823
:100DB00014D90F2203681A40092A01D1406810BDD6
:100DC000032A03D11809C0002043F8E7042A05D1FB
:100DD00001F08AFFFFF7FEF94000F5E70B2000F075
:100DE000B5F8ECE710B5034A0A21034803F0C0FD4B
:100DF00010BDC0463CBA000034BA00000200012019
:100E0000104001D0501070470D22014B1A70FAE7C4
:100E10008C020020F0B585B00393019002912C4E16
:100E20002C4B002A02D002223270013A00251A60AF
:100E30001B68F554019B9D4201DB05B0F0BD029A91
:100E4000AB00D058234B1C68C8239B0037191C1BD0
:100E50000123184206D0204A43102100380009F02F
:100E6000FDFD09E01D4A002802D004281BD11C4AC0
:100E70002100380009F0F2FD300009F061FE154A4A
:100E8000039B1060002B0CD0019B013BAB4208DDA3
:100E9000144B984205D8431C136020223254002280
:100EA000F2540135C6E704280FD90F230268134016
:100EB000042B04D101F018FF0B4A0300CDE7092BE6
:100EC00004D14368094A5B10C7E70123084AC4E715
:100ED0008D020020B0050020ECC200009CBA00008A
:100EE000A2BA00001F030000E3C800000CBD000010
:100EF0001BBD00000123020010B51A4015D10428C3
:100F000001D9026812090B4011D1042901D90B68DB
:100F10001B090024934206D104309B000431C318FE
:100F2000984206D30124200010BD0022EBE70023E5
:100F3000EFE704780A78002C01D1002AF2D00130C2
:100F400001319442ECD00024EDE70000014B187011
:100F5000002070478C02002070B501F0D5FC094CD0
:100F60000100251D1F22280009F0F1FD280009F0CD
:100F7000E7FD0423043080080001184320602000AE
:100F800070BDC04668020020C368F0B59D0083684C
:100F900089B05D190300183306930369069A9F0010
:100FA000069B0290DF19436901939B00D3180393BA
:100FB000CD4B1B78002B26D17F222B68CB491C12EE
:100FC00013409B005B58043501929F46029B587862
:100FD00004F0AAF80023029A137027E0C24B1B7892
:100FE000002B10D12B68019A1C121340BF4A9B00A2
:100FF0009B580435E9E7069B3A1DD11ABA4BD8290C
:1010000028DD1A221A70029BB74C9B682178019345
:10101000EA1A029B92109B7812021A43029B58789C
:1010200004F08AF80023029A23701370029B069A38
:101030009B680193ED1A029BAD10DD60069BFE1AC2
:10104000029BB6101E61039B9B1A029A9B10536170
:1010500009B0F0BD1B783C60002B01D01700D2E72F
:101060002B6801991C120B40A0499B005B5817008C
:101070000435AAE7069B3A1DD11A9B4BD82902DDFD
:101080001A221A70BFE728681B78291D3860002BC8
:1010900002D017000D00B6E76B6801991C120B40D7
:1010A00092499B005B58170008358EE7069B3A1D56
:1010B000D11A8D4BD82902DD1A221A70A3E7A40099
:1010C0001B782C193C60002B01D017009BE72B6884
:1010D00001991C120B4085499B005B581700043591
:1010E00073E7069B3A1DD11A7F4BD82902DD1A22DD
:1010F0001A7088E77E49A40061581B783960002B7C
:1011000001D017007FE72B6801991C120B4077492B
:101110009B005B581700043557E7043F744B3A684F
:10112000A400E250704B1B78002B00D06BE72B68BB
:10113000019A1C1213406D4A9B009B58043544E7EA
:101140006B4BA400E058FFF759FE043F06003868D7
:10115000FFF754FE36180120654B76000643E65033
:10116000614B1B78002B00D04DE72B68019A1C12B5
:1011700013405E4A9B009B58043526E7069B3A1DA8
:10118000D11A594BD82902DD1A221A703BE706986A
:10119000039C0121A04202D221000C3909681B786E
:1011A0003960002B01D017002DE72B6801991C1224
:1011B0000B404E499B005B581700043505E7069B22
:1011C0003A1DD11A484BD82902DD1A221A701AE7A3
:1011D0000699039881420FD203000C3B1B684549D6
:1011E0005B106418E41AA40023583B603E4B1B7844
:1011F000002B05D0170006E7182119700023F4E72B
:101200002B6801991C120B4038499B005B58170052
:101210000435DAE6069B039A934219D213000C3B7D
:101220001B68344A043FA4185B10E31A039A396818
:101230009B0099502C4B1B78002B00D0E3E62B68C9
:10124000019A1C121340294A9B009B580435BCE6A6
:101250001822254B1A70EDE7069B039A93422DD274
:10126000244B3E1FE31814000C3C04932368049A9B
:101270005B10D31A039A9B009858FFF7BFFD0790A5
:101280003068FFF7BBFD2468049B64101C1B079BA0
:10129000A4001F1801207F00039B0743E75037007D
:1012A000114B1B78002B00D0ADE62B68019A1C1265
:1012B00013400E4A9B009B58043586E618220A4BC1
:1012C0001A70EDE7069B3A1DD11A074BD82902DDAB
:1012D0001A221A7097E60399A40061581B783960A6
:1012E000002B09D017008EE68C0200200CBB0000FA
:1012F000482D0020FDFFFF3F2B6801991C120B4079
:10130000D7499B005B58170004355EE6043F039BFA
:101310003A68A400E250D34B1B78002B00D072E651
:101320002B68019A1C121340CD4A9B009B58043530
:101330004BE6039BA4001C192368043F38685E1029
:10134000FFF75CFD36180120C64B76001B7806437C
:101350002660002B00D056E62B68019A1C12134021
:10136000BF4A9B009B5804352FE6069BA4003F1BF9
:10137000BC4CBB420CD82378002B00D043E62B6832
:10138000019A1C121340B64A9B009B5804351CE678
:10139000B54801F099FC2378002B00D033E62B6888
:1013A000019A1C121340AE4A9B009B5804350CE670
:1013B000A300ED18002C00DA38E6AA4B1B78002BAE
:1013C00000D020E62B68019A1C121340A44A9B000F
:1013D0009B580435F9E5043F3B68042B04D1A30076
:1013E000ED18002C00DA21E69E4B1B78002B00D074
:1013F00009E62B68019A1C121340994A9B009B58DE
:101400000435E2E5043F3B68042B06D0A200AD188A
:10141000002C02DA002B00D108E6924B1B78002B3F
:1014200000D0F0E52B68019A1C1213408C4A9B00F7
:101430009B580435C9E53A1F13685B10013B002B2C
:1014400006DD01215B00A4000B432D191360EDE5BF
:10145000844B17001B78002B00D0D4E52B68019A31
:101460001C1213407E4A9B009B580435ADE53A00A0
:10147000069B0C32D31AD82B03DD1A22794B1A7033
:10148000C1E5FF2361005B001940FE3BFF3B1943B0
:101490003960029906988968241204916D1A02999C
:1014A000AD1089782D020D4303999D40091A8910CA
:1014B00099401D430B43BB60029B7D609C70E4B26E
:1014C0006A4BE4000392E358029A9360654A1278EB
:1014D000002A03D008331D00039F94E51D00019AE4
:1014E0009B680C351C1213405D4A9B009B58039F60
:1014F0006BE53B1F1C68039A069B93422DD10A2083
:10150000E3070CD4042C13D90F2322681340042BB7
:1015100011D1200001F0E8FB09F012FB0630643025
:1015200003F0B6FA00280FD1043D069B03937DE536
:101530000720042CF3D02000431E9841FA23404298
:10154000FF3318400730EAE7029B2100587803F088
:1015500005FE0023029A1370E7E7039B039A0C3BF6
:101560001B6802995B109B00D31A0C3B1C601F1D6B
:101570001300083B1B685A108A70D2B23B49D20054
:101580005B0055589B0A029A9B009560ED18039BDF
:10159000069A043B1B685B109B00D3180393314BE6
:1015A0001B78002B00D02EE52B68019A1C121340EB
:1015B0002B4A9B009B58043507E53B1F1868FFF733
:1015C0001DFCA40006003F1B1E2827DC00280DDCA4
:1015D000244B1B78002B00D015E52B68019A1C12B8
:1015E00013401F4A9B009B580435EEE401F07AF942
:1015F000033E361801F076F91D4B801B9842F9D84E
:10160000184B1B78002B00D0FDE42B68019A1C12AC
:101610001340134A9B009B580435D6E40123029AD9
:10162000137001F05FF9029B0A3886195E60FDE4D1
:101630003B1F1868FFF7E2FBA40006003F1B0028D1
:1016400018DC084B1B78002B00D0DCE42B68019AD7
:101650001C121340024A9B009B580435B5E4C04657
:101660000CBB00008C0200202DBD00005025002086
:101670003F420F00CA4B984203DD1D22C94B1A702E
:10168000C1E40123029A137001F02CF9FA239B00A4
:101690005E43029B0A3E30185860C7E4A300FF1A5D
:1016A000002320001A003900FFF7B4FBBE4EBF4CE8
:1016B0003168200001F026FDBD4B31681860200024
:1016C00003F000FC3168200003F04FFD316820007A
:1016D00001F0B4FDB34B1B78002B00D093E42B68D2
:1016E000019A1C121340B34A9B009B5804356CE4CA
:1016F000AC4BA4001B783F1B002B00D083E42B686D
:10170000019A1C121340AB4A9B009B5804355CE4C1
:10171000029803F021FAA34B1B78002B00D072E44F
:101720002B68019A1C121340A24A9B009B58043557
:101730004BE43B1F1B68002B3ED13B000C3B1B685E
:10174000DA072CD5390001225B1058000839024312
:101750000A60002B44DD012259001143381F01604B
:101760003900083909681141CB1A39000C39096868
:10177000114224D09B189340A4001343039AA35012
:10178000884B1B78002B00D03DE42B68019A1C127B
:101790001340884A9B009B580435FFF716FC042B26
:1017A00006D90F2219680A40092A01D15B68C9E7E6
:1017B00019227C4B1A7026E45B10013BC9E704290F
:1017C00009D90F2208680240092A04D102339B007C
:1017D0005B58A400D2E71922724B1A70FFF713FC72
:1017E0000435CDE7A300069AFB189B1AD82B13DC0F
:1017F0000122631E002C14DC6A4B1B78002B01D0E5
:10180000FFF701FC2B68019A1C121340694A9B00E8
:101810009B580435FFF7D9FB1A22624B1A70FFF769
:10182000F2FB3A601C000437E3E7069A3B1D9B1A63
:101830005C4ED82B03DD1A233370FFF7E4FB069BC5
:10184000039AA40093422AD23B1F1868FFF7D6FAE6
:10185000011E21DD039B0C3B1A68521082421BDBE8
:101860009007801A544B4018C018039B8000C25840
:101870003B1B1A604B4B3F1B1B780437002B01D0DE
:10188000FFF7C1FB2B68019A1C121340494A9B00C9
:101890009B580435FFF799FB20233370EAE71823A0
:1018A000FBE7434BA4001A683B1B1F001A603D4B2B
:1018B00004371B78002B01D0FFF7A5FB2B68019A9A
:1018C0001C1213403B4A9B009B580435FFF77DFBDD
:1018D000A3009C46FE1A002C17DC1C22314B1A7008
:1018E000002333606346FF1A2E4B04371B78002B0E
:1018F00001D0FFF788FB2B68019A1C1213402D4A78
:101900009B009B580435FFF760FB002033685A109A
:101910008300F15801230B4003D10D21214A11709E
:10192000DFE749108A4200DD0A0001308442EFDC23
:10193000012352001343D4E7A3009C46FE1A002C57
:1019400017DC1C22174B1A70002333606346FF1A02
:10195000144B04371B78002B01D0FFF754FB2B6886
:10196000019A1C121340134A9B009B580435FFF741
:101970002CFB002033685A108300F15801230B40E0
:1019800003D10D21074A1170DFE749108A4200DABE
:101990000A0001308442EFDC012352001343D4E7F4
:1019A00080EE36008C020020B00500208D02002061
:1019B000080000200CBB0000FCFFFF3F3B00083B81
:1019C0001868FFF71BFA3B1F06001868FFF716FAA6
:1019D0000023864200DA0433A4003A1B1700136088
:1019E000E34B04371B78002B01D0FFF70CFB2B686F
:1019F000019A1C121340DF4A9B009B580435FFF7E5
:101A0000E4FA3B00083B1868FFF7F8F93B1F0600B3
:101A10001868FFF7F3F9F30FC217B0425341A4005F
:101A20003A1B17009B001360D14B04371B78002B27
:101A300001D0FFF7E8FA2B68019A1C121340CD4A37
:101A40009B009B580435FFF7C0FA3B00083B186821
:101A50003B1F1968A600BE1B0423814202D0042844
:101A600002D80023336016E001231842F9D10F2376
:101A700002681A40042AF4D1033A1142F1D1042930
:101A8000EFD90A681340042BEBD1FFF733FA431E5A
:101A9000984180003060B64BA4001B783F1B043790
:101AA000002B01D0FFF7AFFA2B68019A1C121340EC
:101AB000B04A9B009B580435FFF787FA3B00083B70
:101AC00018683B1F1968A600BE1B0023814202D084
:101AD000042802D80423336016E001231842F9D108
:101AE0000F2302681A40042AF4D1033A1142F1D1BB
:101AF0000429EFD90A681340042BEBD1FFF7FAF958
:101B00004342584180003060994BA4001B783F1B32
:101B10000437002B01D0FFF776FA2B68019A1C12CC
:101B20001340944A9B009B580435FFF74EFA3B0044
:101B3000083B1868FFF762F93B1F06001868FFF7BB
:101B40005DF9F317C20F86425341A4003A1B1700F8
:101B50009B001360864B04371B78002B01D0FFF7E6
:101B600052FA2B68019A1C121340824A9B009B5820
:101B70000435FFF72AFA3B00083B1868FFF73EF9E7
:101B80003B1F06001868FFF739F90023864200DD85
:101B90000433A4003A1B17001360754B04371B78FD
:101BA000002B01D0FFF72FFA2B68019A1C1213406B
:101BB000704A9B009B580435FFF707FA3B1F1B68D0
:101BC000A400043B5A1E93413A1B17009B0013606C
:101BD000674B04371B78002B01D0FFF714FA2B68F2
:101BE000019A1C121340634A9B009B580435FFF76F
:101BF000ECF93B00083B1868FFF700F93B1F0600B3
:101C00001868FFF7FBF832180120A4003B1B1F00E7
:101C1000520002431A60564B04371B78002B01D048
:101C2000FFF7F1F92B68019A1C121340514A9B00EF
:101C30009B580435FFF7C9F93B00083B1868FFF7CC
:101C4000DDF83B1F06001868FFF7D8F8321A0120AC
:101C5000A4003B1B1F00520002431A60444B043790
:101C60001B78002B01D0FFF7CEF92B68019A1C12CC
:101C70001340404A9B009B580435FFF7A6F93B00F0
:101C8000083B1868FFF7BAF83B1F06001868FFF713
:101C9000B5F802000120A4003B1B1F007243520054
:101CA00002431A60324B04371B78002B01D0FFF738
:101CB000AAF92B68019A1C1213402E4A9B009B58CC
:101CC0000435FFF782F93B1F1868FFF797F8061EE7
:101CD00017D11F22264B1A70A4003B1B1F001E6049
:101CE000234B04371B78002B01D0FFF78CF92B68AE
:101CF000019A1C1213401F4A9B009B580435FFF7A2
:101D000064F93B00083B1868FFF778F8310006F0EB
:101D10004FFA012640000643DEE73B1F1868FFF735
:101D20006DF8061E17D11F22114B1A70A4003B1B21
:101D30001F001E600E4B04371B78002B01D0FFF7ED
:101D400062F92B68019A1C1213400A4A9B009B58A7
:101D50000435FFF73AF93B00083B1868FFF74EF8E7
:101D6000310006F00BFB012649000E43DEE7C046BA
:101D70008C0200200CBB00003B1F1868FFF73EF8E8
:101D8000C217801850400122A4003B1B1F004000D6
:101D900010431860F64B04371B78002B01D0FFF777
:101DA00032F92B68019A1C121340F24A9B009B588F
:101DB0000435FFF70AF9A300FE1A3068012C24D17C
:101DC000FFF71CF80494079008F016FE0799002905
:101DD00000DC012106F0D2FA049BA400C9180123FB
:101DE00049001943E24B3F1B1B7831600437002B3D
:101DF00001D0FFF708F92B68019A1C121340DD4A45
:101E00009B009B580435FFF7E0F8FEF7F7FF0490BE
:101E10007068FEF7F3FF049B0130C31A0793D3E702
:101E2000A300FE1A31002000049301F0A7F9049BDF
:101E30003060FF1ACE4B04371B78002B01D0FFF720
:101E4000E2F82B68019A1C121340CA4A9B009B5867
:101E50000435FFF7BAF83B00083B1868FEF7CEFFE1
:101E60003B1F06001868FEF7C9FF02000120A4000E
:101E70003B1B1F003240520002431A60BC4B043728
:101E80001B78002B01D0FFF7BEF82B68019A1C12BB
:101E90001340B84A9B009B580435FFF796F83B0067
:101EA000083B1868FEF7AAFF06003B1F1868FEF7FC
:101EB000A5FF320002430120A4003B1B1F0052007B
:101EC00002431A60AA4B04371B78002B01D0FFF79E
:101ED0009AF82B68019A1C121340A64A9B009B5843
:101EE0000435FFF772F83B00083B1868FEF786FFE1
:101EF00006003B1F1868FEF781FF320042400120B8
:101F0000A4003B1B1F00520002431A60984B043789
:101F10001B78002B01D0FFF776F82B68019A1C1272
:101F20001340944A9B009B580435FFF74EF83B1F23
:101F30001868FEF763FFC0430122A4003B1B1F008B
:101F40004000104318608A4B04371B78002B01D0E7
:101F5000FFF759F82B68019A1C121340854A9B0021
:101F60009B580435FFF731F83B00083B1868FEF733
:101F700045FF06003B1F1868FEF740FF3200824015
:101F800051000122A4003B1B1F000A431A60784B3A
:101F900004371B78002B01D0FFF735F82B68019A26
:101FA0001C121340734A9B009B580435FFF70DF831
:101FB0003B00083B1868FEF721FF06003B1F18682E
:101FC000FEF71CFF3200024151000122A4003B1B1E
:101FD0001F000A431A60664B04371B78002B01D0A0
:101FE000FFF711F82B68019A1C121340614A9B00FD
:101FF0009B580435FEF7E9FF3B000C3B1868FEF7E1
:10200000FDFE3B00083B06001868FEF7F7FEF117DF
:102010000200C317300006F003FA3B1F049005913D
:102020001868FEF7EBFE02000498059906F0ACF97B
:1020300043000120A4003E1B370018434C4B306086
:102040001B780437002B01D0FEF7DDFF2B68019AC7
:102050001C121340474A9B009B580435FEF7B5FFFE
:10206000A300FE1A310020000493FEF749FD049BF3
:102070003060FF1A3E4B04371B78002B01D0FEF76F
:10208000C2FF2B68019A1C1213403A4A9B009B58CE
:102090000435FEF79AFFA300FF1A39002000FEF76F
:1020A00047FD334B1B78002B01D0FEF7ACFF2B68AC
:1020B000019A1C1213402F4A9B009B580435FEF7CF
:1020C00084FFA300FE1A310020000493FEF76EFD8A
:1020D000049B3060FF1A264B04371B78002B01D07D
:1020E000FEF791FF2B68019A1C121340214A9B00B6
:1020F0009B580435FEF769FFA300FF1A3900200042
:10210000FEF7E4FD1A4B1B78002B01D0FEF77BFF96
:102110002B68019A1C121340164A9B009B580435E9
:10212000FEF753FFA300FE1A310020000493FEF7D0
:1021300039FE049B3060FF1A0D4B04371B78002BCF
:1021400001D0FEF760FF2B68019A1C121340094A68
:102150009B009B580435FEF738FF069B3E1DF31A83
:10216000034CD82B08DD1A232370FEF74CFFC04622
:102170008C0200200CBB000000F0BEFB43000120DD
:10218000184323783860002B02D03700FEF73BFF5E
:102190002B68019A1C121340F44A9B009B5837008D
:1021A0000435FEF712FF069B3E1DF31AF04CD82BA8
:1021B00003DD1A232370FEF726FF00F093FBED4B9F
:1021C000400018400123184323783860002B02D0C8
:1021D0003700FEF718FF2B68019A1C121340E34AE0
:1021E0009B009B5837000435FEF7EFFE0123A60045
:1021F000BE1B20001A003100FEF70CFEDE4C2068EA
:10220000643002F045FC002802D1043DFEF70EFFC9
:10221000029B21685A78D94802F0B5FF0123029A3F
:102220003700137000F05EFBD54B22681B68063246
:1022300053431818029B5860FEF7F8FEA600BE1B19
:102240002000012300223100FEF7E4FDCA4C206883
:10225000643002F01DFC0028D7D0C84802F08AFD87
:10226000DCE7A4003E1BFEF777FE3700C04B306072
:102270001B780437002B01D0FEF7C5FE2B68019AAE
:102280001C121340B94A9B009B580435FEF79DFE73
:10229000A4003E1B300000F05EFB3700B44B306002
:1022A0001B780437002B01D0FEF7ADFE2B68019A96
:1022B0001C121340AD4A9B009B580435FEF785FE67
:1022C000A4003E1B300000F048FB3700A84B3060F4
:1022D0001B780437002B01D0FEF795FE2B68019A7E
:1022E0001C121340A14A9B009B580435FEF76DFE5B
:1022F000A300FE1A31002000049300F031FB049B80
:102300003060FF1A9A4B04371B78002B01D0FEF780
:102310007AFE2B68019A1C121340944A9B009B582A
:102320000435FEF752FEA4003F1B380000F04AFBC4
:102330008F4B1B78002B01D0FEF765FE2B68019AAE
:102340001C121340894A9B009B580435FEF73DFE42
:10235000A300FE1A31002000049300F05BFB049BF5
:102360003060FF1A824B04371B78002B01D0FEF738
:102370004AFE2B68019A1C1213407C4A9B009B5812
:102380000435FEF722FEA4003F1B380000F084FB5A
:10239000774B1B78002B01D0FEF735FE2B68019A96
:1023A0001C121340714A9B009B580435FEF70DFE2A
:1023B0000121200000F058FB6D4B1B78002B01D051
:1023C000FEF721FE2B68019A1C121340674A9B00FE
:1023D0009B580435FEF7F9FD0021200000F044FB76
:1023E000634B1B78002B01D0FEF70DFE2B68019A82
:1023F0001C1213405D4A9B009B580435FEF7E5FD17
:10240000A4003E1B300000F069FB3700584B3060E1
:102410001B780437002B01D0FEF7F5FD2B68019ADD
:102420001C121340514A9B009B580435FEF7CDFD0A
:10243000A4003E1B300000F065FB37004C4B3060C1
:102440001B780437002B01D0FEF7DDFD2B68019AC5
:102450001C121340454A9B009B580435FEF7B5FDFE
:10246000A4003F1B380000F027FB414B1B78002BDA
:1024700001D0FEF7C8FD2B68019A1C1213403B4A9D
:102480009B009B580435FEF7A0FDA4003F1B3800BD
:1024900003F05AF9364B1B78002B01D0FEF7B3FD41
:1024A0002B68019A1C121340304A9B009B5804353C
:1024B000FEF78BFDA4003E1B300003F0EDF9370062
:1024C0002B4B30601B780437002B01D0FEF79BFDAF
:1024D0002B68019A1C121340244A9B009B58043518
:1024E000FEF773FDA4003F1B380003F0FDF8204BFE
:1024F0001B78002B01D0FEF786FD2B68019A1C1279
:1025000013401A4A9B009B580435FEF75EFDA40059
:102510003E1B300003F0FEF83700154B30601B788F
:102520000437002B01D0FEF76EFD2B68019A1C12B8
:1025300013400E4A9B009B580435FEF746FDA3004E
:10254000FF1A3900200001F01BF9094B1B78002B02
:1025500001D0FEF758FD2B68019A1C121340034A64
:102560009B009B580435FEF730FDC0460CBB0000B5
:102570008C020020FEFFFF7FB00500208D020020AE
:1025800004000020A300FF1A3900200000F080FFA3
:102590009F4B1B78002B01D0FEF735FD2B68019A6D
:1025A0001C1213409B4A9B009B580435FEF70DFDFF
:1025B000A300FF1A3900200000F07AFF944B1B782B
:1025C000002B01D0FEF71FFD2B68019A1C1213404F
:1025D000904A9B009B580435FEF7F7FCA300FF1AB6
:1025E0003900200000F08CFF894B1B78002B01D0B4
:1025F000FEF709FD2B68019A1C121340854A9B00C7
:102600009B580435FEF7E1FCA300FE1A31002000C0
:10261000049303F0BCF9049B3060FF1A7C4B043731
:102620001B78002B01D0FEF7EEFC2B68019A1C12E0
:102630001340784A9B009B580435FEF7C6FCA30064
:10264000FE1A31002000049303F0A9F9049B3060C6
:10265000FF1A6F4B04371B78002B01D0FEF7D3FC19
:102660002B68019A1C1213406A4A9B009B58043540
:10267000FEF7ABFCA300FE1A31002000049303F028
:1026800096F9049B3060FF1A614B04371B78002BCE
:1026900001D0FEF7B8FC2B68019A1C1213405D4A6A
:1026A0009B009B580435FEF790FCA300FE1A3100F6
:1026B0002000049303F083F9049B3060FF1A544B0D
:1026C00004371B78002B01D0FEF79DFC2B68019A84
:1026D0001C1213404F4A9B009B580435FEF775FCB3
:1026E000A300FF1A3900200000F0D2FF484B1B78EE
:1026F000002B01D0FEF787FC2B68019A1C121340B7
:10270000444A9B009B580435FEF75FFCA300FF1A68
:102710003900200000F01CFF3D4B1B78002B01D03E
:10272000FEF771FC2B68019A1C121340394A9B007A
:102730009B580435FEF749FCA300FE1A3100200027
:10274000049300F073FE049B3060FF1A304B043793
:102750001B78002B01D0FEF756FC2B68019A1C1247
:1027600013402C4A9B009B580435FEF72EFCA30017
:10277000FF1A3900200000F0E9FF254B1B78002BE1
:1027800001D0FEF740FC2B68019A1C121340214A2D
:102790009B009B580435FEF718FC069B029AFB1A17
:1027A0009B101361A300FF1A3900200002F0F4F817
:1027B000174B1B78002B01D0FEF725FC2B68019AE4
:1027C0001C121340134A9B009B580435FEF7FDFB77
:1027D000069B029AFB1A9B101361A300FE1A31009C
:1027E0002000049302F0D8F8049B3060FF1A084BD5
:1027F00004371B78002B01D0FEF705FC2B68019AEB
:102800001C121340034A9B009B580435FEF7DDFB66
:102810008C0200200CBB00000023F7B55A1E019269
:10282000002B07DA00F0C2FF02F0AAFB02F00AFD5B
:102830001923019300263000194B1968B14212DDAB
:10284000184B1A6801328A420FDAF0241A601D68A8
:10285000154F6C43E35D002B1FD0E419022B06D10A
:102860002000FEF791FB019BD8E70022EDE7012B4A
:102870000DD1002801D100F035F8F0226A43BB18D1
:102880005B680A49C31A8B4201D80223BB54F02368
:102890005D43054BEB5C022BE2D00136CCE7C04632
:1028A000B405002000000020F01B00203F420F0074
:1028B00000207047002070470020704700207047BC
:1028C00001220020054B06491A615850043103309B
:1028D00058500831801858501A60704700800040E6
:1028E000040500000122034B1A64A822D200985864
:1028F0007047C0460080004010B5FFF7F3FFFA2193
:10290000890005F0CBFB10BD0048704780BD00007A
:102910001A20704770B5054E0400335C0D008B42E1
:1029200002D003F061FF355570BDC046B8050020E8
:1029300070B50024064D635D012B05D100212000F8
:1029400003F052FF0023635501341A2CF2D170BDFD
:10295000B805002070470D207047352070470000F3
:10296000F8B501240B6806000D00234204D10D20A8
:10297000FEF7ECFA2000F8BD5B102000052BFAD81A
:102980000E4A9B009C580E4F3B5D002B05D000214A
:10299000200003F029FF00233B55012E06DD6B6864
:1029A000042B03D10221200003F01EFF200003F0BE
:1029B000C9FD012440002043DDE7C04668BD00009A
:1029C000B8050020F8B501260568354202D04468F4
:1029D000344203D10D20FEF7B9FAF8BD6D10192D60
:1029E000FBD80A4F7B5D012B04D03100280003F097
:1029F000FBFE7E55064964108C4202DCE143C91798
:102A00002140280003F024FEE7E7C046B805002077
:102A1000FF03000070B501240D68254204D10D208C
:102A2000FEF794FA200070BD6D10192D17D8002400
:102A3000012804DD4C68043C63425C416400094E9B
:102A4000735DA34204D02100280003F0CDFE74552D
:102A5000280003F0FDFE03000420012BE3D000203A
:102A6000E1E7C046B805002070B504000D00192844
:102A70000ED8084E335C012B04D0012103F0B4FEC4
:102A800001233355290020004D1EA94103F0CAFE41
:102A900070BDC046B8050020036810B5DA0703D43E
:102AA0000D20FEF753FA10BD4168581004394A4210
:102AB0005141FFF7D9FFF6E737B569460A00064BE3
:102AC00030CB30C203680220042B02D100F0F0FCAE
:102AD00037BD00F015FDFBE740BD000010B5084C08
:102AE000237D002B05D00021142003F07DFE002360
:102AF0002375142003F0ACFE43425841800010BD02
:102B0000B805002010B5084CA37D002B05D000218E
:102B1000162003F069FE0023A375162003F098FE2B
:102B200043425841800010BDB805002070477047EF
:102B300010B5034A0421034801F01AFF10BDC04636
:102B400048BD00001CC40000E12170B549021448D2
:102B500003F0F0FAFFF7B4FE0A2003F0EDFC0023C7
:102B6000FF21104A995401331A2BFBD10122002076
:102B70000D4B01001A6004230C4A0D4D1468002C03
:102B8000FCD02C680002013B20431160002BF5D1E2
:102B90000122084B1A6003F089FC00F053FF70BD5E
:102BA000781B0020B805002000D0004000D1004074
:102BB00008D5004004D00040F8B50B4E07003000A7
:102BC0000D0003F0FFFA0400A84200DD2C003D00D8
:102BD000EB1B9C4205DD300003F0FEFA2870013546
:102BE000F6E72000F8BDC046781B002010B50100B4
:102BF000014803F0A7FA10BD781B002010B5054C62
:102C0000200003F0ADFAE1212000490203F092FA1E
:102C100010BDC046781B0020C3070CD4064B1B68B0
:102C2000834208D8054B1B68984204D8031F1B68D1
:102C3000002B00D018007047DC050020D8050020CC
:102C40000023012210B50A48990001334250642B39
:102C5000FAD1084C084B00211A602000074A07F0FF
:102C6000EBFB074B074A6360074B1A6010BDC04679
:102C7000482D0020E005002008000020D4090000B5
:102C800030270000E4050020D405002010B5044BD7
:102C9000044A1A60044B054A1A60FFF7D1FF10BDC1
:102CA000DC050020E0050020D8050020B40F00203E
:102CB000044B1B68186800090238C343DB1718402F
:102CC0007047C046D405002000B59BB002000549FE
:102CD00001A807F0F5FE01A802F068F802F0B2FAC8
:102CE000FCE7C046E6BD00000A4BC20704D4042836
:102CF00004D8094B00D0094B180070470F22036815
:102D00001A40031D042AF7D0054B092AF4D0054BBD
:102D1000F2E7C046CCBD0000A2BA00009CBA000099
:102D2000DFBD0000D6BD00000020064A0649131F83
:102D3000186013681B0902339B00D2188A42F6D32D
:102D40007047C046E4050020B40F0020F7B50F24FB
:102D50000126304B304A1968304B314D18681368E2
:102D60001F002740072F25D813681B0902339B003B
:102D7000D218AA42F3D300242A4EA500AD19286820
:102D8000FFF74AFF01342860642CF6D1264C2068F6
:102D9000FFF742FF2060254C2068002802D0FFF793
:102DA0003BFF20600025224B1B680093009B9D4247
:102DB00013DBF7BD1B099B00D3189A42D4D01F68C0
:102DC000374208D1B94206D2B84204D3043F3F6823
:102DD000002F00D01F60043BEFE7F0236B43154A40
:102DE0009B181A78002A01D10135DFE71F693C23BF
:102DF00000266B43DB199B0001930136BB1BF3D408
:102E0000019BB4001C1B0B4B1C19A069FFF704FFAE
:102E1000A061F2E7DC050020E4050020D8050020D1
:102E2000B40F0020482D002008000020B40F00201F
:102E3000B4050020F01B0020F7B50124204244D146
:102E4000224B1B689C4698423FD3214B1B68019341
:102E500098423AD8031F1B68002B36D10200036842
:102E600000941B09002B0FD10099131F1960904289
:102E70002BD015682B1F1B68990069180C68013B43
:102E800014600A602A00EDE79D0055192968009C2E
:102E9000214218D18C4516D8019C8C4213D30E1FA9
:102EA0003468002C0FD10F680F343C40072C07D931
:102EB0002F60151F2B600B680A601B090A00D1E701
:102EC00000993160CEE7013BCCE7F7BDDC0500207F
:102ED000D80500200D49F0B50B000F260C4D1868E1
:102EE0001C1F276802090232002F0BD000208B42E2
:102EF00000D0080020609000091892009B18AB4297
:102F0000EDD3F0BDB0431860F7E7C046E4050020FC
:102F1000B40F0020F8B5114C26000F2233681F09AA
:102F200013420DD07D1CAD00A64204D02A00310012
:102F3000200007F06EFA00226319043564191A6044
:102F40000237BF00064BF6199E42E6D31B1B9B10AF
:102F5000013B1B012360034B1C60F8BDE40500200E
:102F6000B40F0020D4050020F0B59BB0FFF7BAFCE9
:102F700000240700204AA300D0580134FFF75CFF6B
:102F8000642CF7D11D4B1868FFF756FF1C4B1868CF
:102F9000002801D0FFF750FF00261A4B1B689E4205
:102FA00016DBFFF797FFFFF7D1FEFFF7B3FFFFF741
:102FB00099FC154BC21B1B6814491B6801A81B090F
:102FC000023B07F07DFD01A801F0F0FE1BB0F0BD53
:102FD000F02575430E4BED182B78002B01D10136EF
:102FE000DBE72B695C1E002CF9DBA300EB1898696A
:102FF000FFF722FF013CF6E7482D002008000020E3
:10300000B40F0020B4050020D4050020ACBD0000A2
:10301000F01B0020F7B5164D4F1C2B6806001B68EF
:103020000C0001921B099F420ADBFFF79DFF2B68F2
:103030001B681B099F4203DB0A20FDF787FFFEBDCB
:103040002868A71CBA00DB1B81181B010B602960D4
:103050000021031F19600F231E4003002401264393
:1030600040C3083A9A189A42E9D9019902C3FAE78B
:10307000D4050020F7B503000122134004000D0021
:103080000193002B2AD1164B1B68834226D8154B7F
:103090001B68834222D90F23134F38600068184001
:1030A000FFF7B8FF019B3C68061E3B6016D0236803
:1030B00004301B099D4200DD1D00AA00211D251FB3
:1030C00007F09EF9FFF730FE2E60FFF73FFE00236A
:1030D0002B6022680F339A43226034002000FEBD2B
:1030E000DC050020D8050020B40F002003230430A5
:1030F00010B5C11719400918891000220420FFF7E4
:1031000089FF10BD70B5050008000C00FFF7EEFF49
:103110000023002804D170BDE95CC218117101338D
:10312000A342F9DBE343DB171C400023041923719E
:10313000F1E7000010B501240B681C4016D05C10AC
:10314000200005F0C9FA0B4905F094F907F07AF868
:1031500003F0C2FC0022084B06F02EFA03F064FCD8
:1031600007F000F843000120184310BD0D20FDF7C3
:10317000EDFEE5E7D30237390000D040086870B5AE
:1031800001240500254006D1042804D90F23026834
:103190001340042B03D00E20FDF7D8FE70BDFFF7BF
:1031A000A3FD03782900233B5A4253411022C01843
:1031B00007F07CFD80239B05C218044B9A4201D97D
:1031C0001420E9E740002043E8E7C046FFFFFF3F47
:1031D00010B5034A0221034801F0CAFB10BDC046E6
:1031E000FCBD0000F7BD00000020704710B51E2098
:1031F000FDF7ACFE10BD10B51E20FDF7A7FE10BDFB
:1032000010B51E20FDF7A2FE10BD10B51E20FDF763
:103210009DFE10BD10B51E20FDF798FE10BD10B527
:103220001E20FDF793FE10BD10B51E20FDF78EFE8B
:1032300010BD10B51E20FDF789FE10BD70470000BF
:1032400010B5034A0921034801F092FB10BDC046A6
:103250001CBE000064BE00000120034B1860034B3D
:103260001B68834018437047D80F0020B80F002018
:10327000F0B5EFF310810123194083F31088134C4C
:10328000134AA4461268134E013A9340124F134A50
:10329000002B17D0146803420FD03D682C60C04645
:1032A000C046C046C046C046C046C046C0460C4C9C
:1032B0001568246825605B08EAE765462C60146899
:1032C0003460F8E781F31088F0BDC046080500506F
:1032D0000C0000200C050050C40F0020CC0F002073
:1032E000C00F002030B585B001AD0C220649280082
:1032F00007F086F80024285D01210134FFF70AFB5E
:103300000C2CF8D105B030BDF0BE0000F7B56A4610
:10331000394B01AD13800F239370384B2B800A2358
:10332000AB70FFF7DFFA364B364CC0182368984273
:1033300001D2002323602668002E3DD16B469F5D9D
:1033400001213800FFF7E6FA01360021380003F0CA
:1033500069FA032EF2D10026AF5D01213800FFF794
:10336000D9FA01360121380003F05CFA032EF3D1BB
:10337000C8200138C046C046C046C046C046C04608
:10338000C046C046C046C046C046C046F1D1002136
:103390002878FFF7BFFA68780021FFF7BBFAA87812
:1033A0000021FFF7B7FAFFF79DFAFA2300251B016A
:1033B000C01820602800FEBDFFF794FA236800259E
:1033C0009842F7D3032003F0BDF80600042003F071
:1033D000B9F836180A2003F0B5F80B4B9B1B181AE6
:1033E0000A4BA84206DB18600023094A23601360D9
:1033F0000125DFE71D60F7E70D0E00000304000064
:1034000010270000D00F0020E3030000B80F0020B9
:10341000D80F002010B50124044002D04410200031
:1034200010BD0D20FDF792FDF9E700000868F8B522
:10343000C3071AD5FFF7EEFF0300203B5E2B23D80E
:103440000520012258430023104E451DA84217D0E5
:1034500005211024375C3C4200D09B1801395200F2
:1034600064100029F7D10130F0E704280CD90F22AD
:1034700003681A40042A07D11B0905D00079DBE74D
:1034800001205B001843F8BD0120FCE7FCBE0000F2
:103490000022054B10B51A60044B1B68934201D003
:1034A00002F0F8FA002010BDD40F00209C1A002072
:1034B00070B508680D00FFF7ADFF04006868FFF7FE
:1034C000A9FF621E0100042A14D8451E042D11D83C
:1034D00005236B439B18012215009D402B000648D5
:1034E00005682B430360054B1B68002B02D02000AE
:1034F00002F0D1FA002070BDD40F00209C1A0020E9
:1035000070B508680D00FFF785FF04006868FFF7D5
:1035100081FF621E0100042A13D8451E042D10D815
:1035200005236B439B1801229A4007480368934385
:103530000360064B1B68002B03D00022200002F022
:10354000AAFA002070BDC046D40F00209C1A0020AB
:10355000F0B5050089B008680C00FFF75BFF069026
:10356000022D36DD6068FFF755FF0190A068FFF778
:1035700051FF04000127231D661E0793731C02934D
:10358000079B9E4235D0052373430593019B019D04
:1035900005330493049BAB421ED0042E16D86B1E39
:1035A000042B13D80122059B2349013B5B199A4048
:1035B0009446224A0B681068069A3A4003920DD04E
:1035C00062461A430A60012200280DD17F000135AE
:1035D000E0E701240194CDE7029ECFE762469343E2
:1035E0000B600028F2D0039A0299280002F053FAE7
:1035F000ECE7019B1E1D042E1AD8012C18D10025C2
:1036000005273B0021006B439B1999400B000A4A98
:10361000013511689943094B11601B68002B05D0D7
:10362000019B0022581D290002F035FA052DE8D132
:10363000002009B0F0BDC046D40F00209C1A002025
:1036400010B5041E10DA1A240A4BA400E258012314
:103650009340094A09491360094A1160094A0A4915
:1036600011600A4A136010BDFFF752F9A042EADD6B
:10367000EAE7C04670CB0000CC0F002008050050E0
:10368000C40F0020C00F00200C050050180500508A
:103690002B4BF7B51B680C00002B03D101204042D7
:1036A000FFF7CEFF24680126250035401AD0FF22FF
:1036B0006310120260121040DAB21043FF221B02A4
:1036C0001204134018431F4B1B68202B06D1B44033
:1036D0001D4BA40EA400E35800021843FFF7C8FDD9
:1036E0000020FEBD042CFBD90F2322681340092BB8
:1036F000F6D1FF2763683F025B100193019B9D4257
:10370000EEDAAB00E3189B68334216D05A10581219
:10371000D1B238400843FF21120209040A40104385
:10372000084A1268202A06D15B009B0E06499B00BE
:10373000020258581043FFF79BFD0135DEE7C046F3
:10374000CC0F00200C000020D8C000000200086848
:1037500010B5C3070FD540101823012A03DD4A68AE
:10376000042A00D10833054A1360FFF7F3F8FFF786
:1037700067FF002010BD01204042EDE70C00002053
:10378000086810B5C30703D5FFF744FE054B186062
:10379000054B1B68002B03D0024B186802F07CF924
:1037A000002010BDD40F00209C1A00207FB5A04C33
:1037B0002368002B0AD19F4A1268002A06D19E4B2B
:1037C0001B68002B01D0FFF7A1FD7FBD9B4D2A6830
:1037D000002A26D1984A1268002A1BD0FFF796FDCE
:1037E0000028F2D0FFF77EFD924B24681A681C6017
:1037F000002A16D0002C14D101AD0C2290492800CB
:1038000006F0FEFD285D00210134FFF783F80C2C43
:10381000F8D1DAE7874A1268002AE5D1002BE3D015
:10382000E0E700210D2002F0FDFF00210E2002F054
:10383000F9FF00210F2002F0F5FF2E68012E5DD068
:10384000022E00D1A2E0002E51D101363100794C78
:1038500004202368994302F0E5FF04212368052032
:1038600019404B42594102F0DDFF10212368062028
:1038700019404B42594102F0D5FF802123680901CC
:1038800019404B4259410C2002F0CCFF80212368A3
:10389000090219404B4259410B2002F0C3FF80211D
:1038A0002368490219404B4259410A2002F0BAFFED
:1038B00080212368890219404B425941092002F0B6
:1038C000B1FF80212368C90219404B4259410820A9
:1038D00002F0A8FF802321681B0319404B42594185
:1038E000072002F09FFF31000D2002F09BFF2B68A4
:1038F0000321581C04F042FD296066E702214D4C6B
:103900000720236819404B42594102F08BFF0820E1
:10391000216801404B42594102F084FF8021236815
:10392000C90019404B425941052002F07BFF80211C
:103930002368490119404B425941062002F072FFA9
:1039400080212368C90119404B425941042002F0EB
:1039500069FF80212368890319404B4259410A209D
:1039600002F060FF802321681B0419404B4259413B
:10397000092002F057FF31000C2002F053FF310004
:103980000B2002F04FFF31000E20AEE72021294C22
:103990000720236819404B42594102F043FF402160
:1039A0002368082019404B42594102F03BFF802117
:1039B0002368092019404B42594102F033FF80210E
:1039C0002368490019404B4259410A2002F02AFF5E
:1039D00080212368890019404B4259410B2002F095
:1039E00021FF80212368890119404B4259410C2055
:1039F00002F018FF80212368490319404B425941C6
:103A0000062002F00FFF80212368C90319404B42B2
:103A10005941042002F006FF802321685B0419400D
:103A20004B425941052002F0FDFE01210F205CE7C9
:103A3000D40F0020C80F0020D80F0020BC0F00209A
:103A4000F0BE0000012010B54042FFF7F9FD002054
:103A5000FFF70EFC10BD000010B5034A0921034812
:103A600000F086FF10BDC046D8C1000020C2000093
:103A700030B502248025094B094AED009C505C5961
:103A8000002CFCD0A124E400884202D300219950EC
:103A900030BD8025ED0018514019F5E700E00140E8
:103AA0000405000010B5002806D1C020B021400256
:103AB0008902FFF7DDFF10BDB02080218002C9021E
:103AC000F7E7000043425841064B40421840B023FC
:103AD0009B02C018036800201A0E532A01D11B0252
:103AE000180A704700C0FEFF30B501248025054B41
:103AF000054AED009C505C59002CFCD0016000216F
:103B0000995030BD00E00140040500004342584197
:103B1000074B40421840B0239B02C018A62310B5A3
:103B20000902DB05090A1943FFF7DEFF10BDC04695
:103B300000C0FEFF70B5012480250D4B0D4EED0039
:103B40009C515C59002CFCD0002902DC00229A51C7
:103B500070BD557814782D022543947801392404DA
:103B60002543D478043224062C4310C0ECE7C04629
:103B700000E001400405000070B505004B680A0034
:103B80009C1C2100A400FFF7D5FF281970BD000080
:103B9000134B1B68002B0CD08022B023D2029B0257
:103BA00000280BD11A1D5B681B0E522B00D1100090
:103BB0007047B022C02392025B02F1E782420DD926
:103BC00003681B0E522B09D1436802339B00C018B7
:103BD000824203D903681B0E522BE9D00020E7E78D
:103BE000DC10002070B50020FFF7D2FFFF26050093
:103BF000002801D1280070BD03681C143440FFF771
:103C0000C7FFDA2CF4D10500F2E700008022F0B5FE
:103C10005200A1B00021674806F00EFC802200216E
:103C20005200654806F008FC644BFF271B681A0029
:103C3000049353425A4110000592FFF733FF049C4E
:103C40000020631E9C415E4B64421C405D4BE418A7
:103C5000FFF7C8FF0600002E2DD10498FFF732FFB2
:103C6000411C0598FFF752FF059A574D534B2C60A6
:103C70001A60FEF7C3FF514B64201B68A0215A4213
:103C800053414F4A5B421340B0222C6892029B186A
:103C9000E41A6043490204F08BFAA02252020300A6
:103CA00000924A49220007A806F00AFF07A801F07F
:103CB0007DF821B0F0BD3268131412123A403B4037
:103CC00003921A000A3A092A49D83A4B039A995C96
:103CD000002931D110223E4806F0AEFB35002B689A
:103CE00003991A123A40914209D11A143A400B2A08
:103CF00027D0132A2DD00A2A01D1354B1D60280068
:103D0000FFF746FF051EEAD1314B196800290FD095
:103D10002000FFF731FF04002D4B5B195968002983
:103D200003D02000FFF728FF040004350C2DF3D149
:103D3000204B0121039A99543000FFF729FF060018
:103D400089E73B40022BDADC214A9B00D3185D60F7
:103D5000D5E7102200211E4806F06EFBCFE71A00BF
:103D6000153A082AE8D8144A0399525C002AE3D18C
:103D70003500152B00D01500300003681A143A40A6
:103D8000152A0FD01D2A00D10025FFF701FF0028BA
:103D9000F3D1002D04D020002900FFF7EDFE040030
:103DA000054BC6E7039A1B123B409A42EDD1050032
:103DB000EBE7C046DC0F0020E4100020DC10002000
:103DC00000C0FEFF04C00200E0100020B9C20000E5
:103DD000D82E0020F0B50020B7B00024FFF7D8FEA1
:103DE000270005002600002D2ED1284D2868FFF75A
:103DF00069FE32003B0001900094254904A806F0BA
:103E00005FFE04A800F0D2FF224B64201C682B68E0
:103E1000A0215A425341204A5B421340B0229202F1
:103E20009B18E41A6043490204F0C2F9A02252022E
:103E3000030000921949220004A806F041FE04A8DC
:103E400000F0B4FF37B0F0BDFF226B6829689C46D4
:103E50000233FF180B12013613409C4200DA1C009B
:103E6000FF200A1402400392624601400192009131
:103E7000039A0B4904A806F023FE04A800F096FF5D
:103E80002800FFF785FE0500ADE7C046DC100020E6
:103E90002AC30000E010002000C0FEFFD4C20000D2
:103EA00016C3000070B50020FFF70CFE04000120CF
:103EB000FFF708FE844200DA04000A4B1D686A42DC
:103EC000554128001D60FFF7EDFDA0226B42520214
:103ED0001340054A28009B18044A611C1360FFF731
:103EE00015FE70BDDC10002004800100E0100020F1
:103EF000F8B50020FFF7E6FD07000120FFF7E2FD1F
:103F00003E00204D0643204C0DD18021C020C90227
:103F10004002FFF7ADFD01213000FFF7F7FD1B4B1D
:103F20002E6023601DE0874209DD0023B0212B6055
:103F3000164B8902236023680020012517E0012326
:103F400080212B60124BC9022360F4E7120E522A23
:103F500008D0002800D023600E4800F027FFFFF7AC
:103F6000A1FFF8BD28005A68023292009B188B42CC
:103F700005D21A68561CE9D10028F2D0D1E7216099
:103F8000EFE7C046DC100020E010002004800100B4
:103F900004C00200EFC20000F0B585B00392032216
:103FA0000333DC17294D1440E4182B68284F5A427C
:103FB000534180225B42D202A4103B409B18A21CBA
:103FC0000291244E910000910190316800980A18E6
:103FD000934215D2FFF71AFE2B685A4253418022B2
:103FE0005B421F40D202BF183368009A9B189F4261
:103FF00006D2194800F0DAFE0025280005B0F0BD11
:10400000029B356819066B461A7BA423DB05134314
:10401000FF222F00090C1943019B12041B041340BB
:1040200019432800FFF760FD0837281D210037607D
:10403000FFF75AFD002C04D00A9A21003800FFF740
:1040400079FD009B083BFF183760D6E7DC100020A5
:1040500000C0FEFFE010002093C2000010B5FFF783
:10406000D5FD10BD70B59AB0FFF742FFFF221E4C80
:10407000D2000021200006F0DFF9FF25FFF7B2FD96
:104080000026002814D10200C300E3580130591E55
:104090008B41D218FF28F7D1144901A806F010FD72
:1040A00001A800F083FE124800F080FE1AB070BD37
:1040B00003681A142A400A2A0AD11A122A40FF2A2F
:1040C00003D0D200A1180B71A050FFF761FDD8E713
:1040D000132AFAD11B122B40FF2BF6D0DB00E2187B
:1040E0001671E650F1E7C046502500205FC300007E
:1040F00073C300000021094B094A59600131516026
:1041000059680029FCD00021196101239360022223
:10411000044B8131FF315A501A607047FC10004047
:104120000010004000E100E00222064B0121DA67A6
:104130000022054B5A61054A11615A69002AFCD0D8
:104140007047C04604E100E0FC1000400010004051
:1041500010B5044C2378002B01D0FFF7E5FF0020B9
:10416000207010BDE51100200120024B1B685B0090
:10417000184370476812002003480368002B02D1DF
:104180001422037102607047002F00200120024BAF
:104190001B685B00184370471000002070B50400D6
:1041A0000D001600FEF7A8FB8023012200215B050D
:1041B0005B6E6270E270020AA271020CE2711A0A6E
:1041C00060716372000EA2721A0C1B0E26702571AC
:1041D000A1702072E272237370BD0000124B10B503
:1041E0001B68124C5A1C0FD0114C002B0CD0114CD8
:1041F000012B09D0104C022B06D00D4C042B03D000
:104200000E4C052B00D10B4C21000D4806F090FC04
:10421000200006F095FC0300042204339B080948A3
:104220001B011343036010BD14000020FBC30000FA
:10423000F4C3000006C400000BC4000000C400006A
:10424000EC2E0020E82E002070B5214C2278002AA8
:104250003DD1204B01215A608022D20511605A685D
:10426000002AFCD0002207201B4B1C4901255A5074
:104270000439585008315A5019481A4958501A49A7
:104280001A485A501A495A50A622D2009D50082264
:1042900018495A50043158500220174958501749AC
:1042A0001748585017480439585018201649585084
:1042B000C12189005A500539FF39585892180243D4
:1042C0005A501249124A9950FFF714FF257070BDD9
:1042D000E5110020FC000040001000400C0500002B
:1042E000746962751C0500002405000020000402AA
:1042F0002C05000014050000340500003C050000FA
:10430000FFFF00002110010054050000E61100200D
:104310000405000070B50E4B06001B78002B01D180
:10432000FFF792FF00200B4D2C7884420ED00A4BF1
:10433000202219780323091B1940084B4901C91889
:10434000300006F05DF80120013C2C7070BDC046C5
:10435000E51100206C120020E4110020E61100207D
:10436000002370B588B0984227DD0D6801262C0027
:1043700034409C4221D12300042D1ED90F222B68EA
:104380001A402300092A18D16A681F2A15D96846DD
:10439000FFF7C0FF230000280FD06B4619783300C9
:1043A000A14203DB6B461B5D5B003343A200AA18EE
:1043B00001349360202CF2D10423180008B070BDA2
:1043C00070B5414B8AB01B78002B01D1FFF73CFF41
:1043D00002AD2800FFF79EFF002802D100200AB09E
:1043E00070BD2B780B2BF9D96B78012BF6D1EB78BC
:1043F000012BF3D10023354E354C336023712B79DB
:10440000344A1360002B0ED1152169444A780B7889
:1044100012021A438B781B041A43CB781B061343F2
:104420003360002318E0012B20D1152169444A781C
:104430000B7812021A438B781B041A43CB781A218B
:104440001B06134333600E236A7C6944934200DDEC
:10445000130000229A4232D104200021E2180433D2
:104460009B101B01034311712360B8E7022B03D19A
:104470006A7B10331621E8E7042B0DD115210822A1
:104480006944684605F0BCFF0098019902F03CFAC7
:1044900005F068FE3060C4E7052BC2D11521082263
:1044A0006944684605F0ACFF0098019902F02CFAC7
:1044B00005F058FE30606A7D0A231E21C5E78D5C39
:1044C000A01805710132C5E7E5110020681200202F
:1044D000002F00201400002010B5134B04001B789F
:1044E000002B01D1FFF7B0FEFFF71EFE00200F4AA0
:1044F0000F49104B54505860013010605868002824
:10450000FCD0002018610130906018690028FCD0B0
:10451000094B0A481B785B011B185350FFF704FE38
:10452000FFF7E8FD10BDC046E51100200010004077
:1045300004050000FC100040E4110020E6110020FA
:1045400010B588B000281DDD0A68012113000B405A
:1045500018D1042A16D90F2014682040092811D137
:1045600050681F280ED9980010188068002408424F
:1045700001D04010C4B26846C4540133202BF2D19C
:10458000FFF7AAFF002008B010BD000010B50028FA
:1045900013DD0C68E30710D56410532C0DD8084BBD
:1045A0001B78002B01D1FFF74FFEFFF7BDFDA123C4
:1045B000044ADB00D450FFF79DFD002010BDC0462B
:1045C000E51100200010004010B500280EDD0C6839
:1045D000E3070BD56410FF2C08D8054B1B78002B84
:1045E00001D1FFF731FE034A034BD450002010BD28
:1045F000E5110020001000402405000013B500283C
:1046000014DD0C68E30711D5094B64100093094BC6
:104610000193072C0AD8084B1B78002B01D1FFF718
:1046200013FE6B46054A1957054BD150002016BDA5
:10463000E2ECF0F4F8FC0004E5110020001000406A
:104640000C05000070B588B0002820DD0124086842
:1046500004401CD104281AD90F2302681340042BEC
:1046600015D1FEF741FB060006F06AFA0500122894
:1046700000D912252A0002210D326846FFF78EFD6F
:104680006B465D73A54205DC6846FFF725FF0020F9
:1046900008B070BD2300325D6B449A730134F1E7BA
:1046A000F0B50D008BB0012832DD0868012204004E
:1046B00014402DD104282BD90F2301680B40042B63
:1046C00026D16B68134223D0FEF70EFB6E680700FD
:1046D0007310019306F034FA05000E2800D90E2558
:1046E0002A000121113202A8FFF758FD6A4612790B
:1046F00002AB5A7302AA73129373019B76141B0EBA
:10470000D67313745574A54205DC02A8FFF7E4FEC6
:1047100000200BB0F0BD3A5D02A963189A74013411
:10472000F1E730B589B0002814DD0C68E30711D536
:10473000102268460021FFF731FD6B466A4665107E
:104740005D73684663122D0E64149373D4731574ED
:10475000FFF7C2FE002009B030BD0000174B184A19
:104760005968002903D0002159600131916019690D
:1047700000291FD0002018618023DB00D358114985
:10478000012B18D1A923DB00D3585B420B600E49E3
:104790000B78032B01D801330B7003200B490B78E6
:1047A000013303400B700A495B015B180949535000
:1047B0000123936070470860FAE7C046FC10004090
:1047C00000100040100000206C120020E4110020B6
:1047D000E61100200405000010B5034A0E2103482D
:1047E00000F0C6F810BDC04684C300007BC30000C3
:1047F000044A05491368C85401339B059B0D136097
:104800007047C046881600208812002070B5114CF1
:10481000114A2368834202DC0023236016E0155C02
:10482000411C2E00FA3E012E05D899420FDA555C44
:10483000013D1F2D01D90800ECE70100151A565C57
:104840006E5401318B42FADC181A206070BD15706D
:10485000FAE7C046941A00209416002010B5FEF71F
:1048600041F8064B1A68824201D900221A601B687F
:10487000C31A034898428041404210BD8412002070
:10488000204E000010B5094C094A23681268934273
:1048900000D110BD074AD05CFEF7A8F90028F8D077
:1048A000236801339B059B0D2360ECE78C160020E9
:1048B000881600208812002010B50400064B074A15
:1048C0001B6812689B1ADB439B059B0DA34200DB10
:1048D00010BDFFF7D7FFF1E7881600208C160020E7
:1048E00070B50020FFF754F9FF260500002801D11C
:1048F000280070BD03681C143440FFF749F9DA2C16
:10490000F4D10500F2E7F7B5050056680191B00053
:10491000441C06301700FFF7CFFFFB20FFF768FFAE
:104920001C20FFF765FFE8B2FFF762FFE0B2241238
:10493000FFF75EFFE0B2FFF75BFF6B461879FFF70A
:1049400057FF0025AE4200DCF7BDAB00FB189C68AA
:104950000135E0B2FFF74CFF2012C0B2FFF748FF6D
:104960002014C0B2FFF744FF200EFFF741FFE9E734
:1049700070B5074E3368092B08DC0C255D43054CE8
:104980000133285164196160A260336070BDC04674
:1049900090160020242F0020F0B587B002900C0064
:1049A000012803DC1B20FCF7D1FA45E0244B086802
:1049B0000093C30709D4042807D90F2302681340C2
:1049C000042B02D1FEF790F900901D4B6068019313
:1049D000C30709D4042807D90F2302681340042B06
:1049E00002D1FEF781F901900027164B1B68049352
:1049F000049BBB42D6DD0C267E43134B0099F61870
:104A0000306806F08BF8051E05D17368B66805930B
:104A1000059B9D4201DB0137EAE730680199039667
:104A200006F07CF80836002808D121000298039B84
:104A3000083102385B68984707B0F0BD0135E7E7F9
:104A4000F6BD000090160020242F002010B5FCF7C2
:104A5000C9F9FFF701F8FEF76BF8FEF7B9FBFEF7AF
:104A6000EFFBFFF7B9FE00F063FE01F017F810BD91
:104A7000962210B512010021034805F0DDFC00224A
:104A8000024B1A6010BDC046F01B0020B405002088
:104A9000064B074A1B6812689B1ADB439B059B0D5C
:104AA0000122834200DC002210007047881600209B
:104AB0008C160020F8B505000C0016001F1E0ED144
:104AC0000320FFF7E5FF002808D0FA20FFF790FE4B
:104AD000E8B2FFF78DFEE0B2FFF78AFEF8BD501D89
:104AE000FFF7D6FF0028F9D0FB20FFF781FEE8B2E0
:104AF000FFF77EFEE0B2FFF77BFEF0B2FFF778FE35
:104B00003012C0B2FFF774FE3C00E31B9E42E5DDAD
:104B10002078FFF76DFE0134F7E7000070B5002440
:104B2000F0250B4B1B68A34202DCFFF7A1FF70BD11
:104B30002B006343074A9B181A78002A05D059783E
:104B4000002311201A00FFF7B5FF0134E9E7C04642
:104B5000B4050020F01B0020F8B507000024F02564
:104B60002B0063430C4A01349E18B74211D03178B0
:104B700000290BD00133D15C002311201A00FFF76C
:104B800099FF2A000021300005F056FC0A2CE7D1DD
:104B9000F8BD024B1C60F9E7F01B0020B4050020B3
:104BA000F0B5150001222F005E4C1740A54401907E
:104BB0000291002F11D005AB1A706A105A70120EB4
:104BC0001A710522691299706D140299DD70FFF750
:104BD00071FFCF239B009D44F0BD042D1ED90F23F0
:104BE0002A681340042B25D1023B04AA2800137124
:104BF000FEF77AF8040005F0A3FF4B4B984200D96A
:104C00001800B84204DC421C05AB02990198DEE7AB
:104C100001377B1EE35C05AAD355F2E7042D7CD156
:104C2000032304AA043D13716B425D4105AB55712A
:104C30000222EAE7092BCCD1042205AB1A706A687C
:104C4000511000916946521209789A70009A597071
:104C50001F2A01DD202200926A46127806ACDA7023
:104C6000009BBB4202DC05ABE21ACEE70126BB008B
:104C7000EB189868064006D1042837D90F2302683C
:104C80001340022B0CD10123237043106370421296
:104C90001B0E4014A270E070237105340137DFE76A
:104CA000042B21D1023B2370FEF71EF8039005F080
:104CB00047FFA31C0C2809D86070864201D19C19BB
:104CC000ECE7039A925D9A550136F6E70C22627082
:104CD000039A925D9A550136092EF9D12E23E3727B
:104CE000237363730E34D9E7012B07D103230438F0
:104CF00023704342584160700234CFE7092B09D139
:104D0000053B23704368E6705A105B126270A37013
:104D10000434C3E726700134C0E7002D00D058E703
:104D20007EE7C046C4FCFFFF2303000070B502000D
:104D30000024F0210D4E080060438019457895420B
:104D400003D001340A2CF6D170BDF022002105F009
:104D500073FB074A1368013BA34200D11460002390
:104D600029001A001120FFF7A5FEEDE7F01B002037
:104D7000B405002010B5B2B002236A4604001370D7
:104D800005F0DEFEC72800D9C7200023984207DCC3
:104D9000421C6B46FE211420FFF78CFE32B010BD82
:104DA000694601335A1EA25CCA54EFE730B5B3B06E
:104DB00002236A460500137005F0C2FE0400C728EE
:104DC00000D9C72400239C420BDC20003230FFF7BF
:104DD00073FD621C6B46FF211420FFF76BFE33B09E
:104DE00030BD694601335A1EAA5CCA54EBE7000085
:104DF000F7B5234B06001B68F02100930023009AAF
:104E00009A4211DC0024F0231A00624301920199B6
:104E10001C4A55182F78002F12D001340A2CF3D1D8
:104E20001948FFF7C3FF29E00A005A4315488218C2
:104E30005078B04202D11278002A1FD10133DEE748
:104E4000F0223900280005F0F7FA02230D4A0199F3
:104E5000EB6053540D4AF1008A58009B6E70AE709F
:104E6000AA602F616F61A34202DC054B01341C6014
:104E7000002331001A001020FFF71CFEF7BDC046CA
:104E8000B4050020F01B0020F5C8000050250020CC
:104E900010B5FFF743FEFF24084AE3005B429B186E
:104EA000074AD35C043B012B03D8E043C0B2FFF7B1
:104EB0009FFF013C002CEFD110BDC046FC07000055
:104EC00050250020F7B50F00FF247F2501901E4AD2
:104ED000E300D31A1D4A9A181278062A01D0032A31
:104EE00020D1FF22D2009B18186883682B401C2B0E
:104EF00018D1C3681A002A40042A13D102692A4033
:104F0000192A0FD11B0A01339B000C30C018FDF782
:104F1000EBFE03780600002B10D005F011FE0023F5
:104F2000B84209D0013C002CD1D1F7BD019AF15C07
:104F3000D25C9142F6D101339F42F7DCE043C0B22C
:104F4000FFF756FFEEE7C04650250020FC070000A3
:104F500070B50500FF24084AE3005B429B18074A2E
:104F6000D35CAB4203D1E043C0B2FFF741FF013C49
:104F7000002CF0D170BDC046FC0700005025002079
:104F8000F7B5FDF7AFFC514B1A68824201D90022F8
:104F90001A601A684E49821A8A4200D883E0186063
:104FA000FDF7AAFC071E00D101370020FDF796FD92
:104FB00001900020FDF7A6FD019B0090454C464D59
:104FC000002B14D02368002B00D07AE02B682760D8
:104FD000002B00D171E0414B01261B78002B63D1DF
:104FE0000920FFF7B5FF3E4B1E703C4B1E70009B27
:104FF000002B12D02B68002B0FD123682F60002BC1
:105000001ED0374B01261B78002B52D10920FFF709
:105010009FFF334B1E70314B1E702368002B0FD047
:105020002F4E3278002A0BD19F4200D2276023688E
:10503000FB1A312B04D90720FFF78AFF01233370B5
:105040002B68002B0FD0254E3278002A0BD1BB42A3
:1050500000D92F602B68FF1A312F04D90820FFF7E1
:1050600077FF012333702368002B0CD0019B002BAA
:1050700009D11B4E3378002B02D10720FFF768FFC0
:105080000023236033702B68002B0CD0009B002B77
:1050900009D1124C2378002B02D10820FFF758FFCA
:1050A00000232B602370F7BD0720FFF751FF0C4B47
:1050B0009CE70820FFF74CFFADE7009B002B9CD13D
:1050C000ABE7009A002A95D1AAE7C04680120020DB
:1050D0000F27000070120020781200207C120020A0
:1050E0007412002037B500240500FFF717FD01A852
:1050F0000194FDF7E1FC21002000FEF7C9F9FEF75D
:1051000055FBFDF713FDFDF712FDFEF79BFCFDF7C8
:105110000FFCA54204D0FDF793FD0248FFF746FEC1
:1051200037BDC046E6C80000002310B501001A00D4
:105130001120FFF7BFFC10BD07B56B46197069461B
:105140005A7013128B701314120ECB700A716B46C7
:10515000010005221320FFF7ADFC07BD10B50A00C2
:1051600001001220FFF71CFD10BD70B505000800FE
:105170000C003230FFF7A0FB2B00220000211B2087
:10518000FFF798FC70BD10B50C000300110014204F
:105190002200FFF78FFC10BD012370B5FF24084AE1
:1051A00041185B42884201D3D84370BD06781D0A7E
:1051B000234073409B009B5801306B40F2E7C04690
:1051C000C8C40000002313B501930B4BC2000400B8
:1051D000D058002805D0436808309900FFF7DCFF5D
:1051E00001900920FFF768FB01AB04222100172082
:1051F000FFF760FC13BDC04650250020F7B50190B5
:10520000FFF76EFB01250400FF276D42002C01D142
:105210002800FEBD266833143B40152B0DD121001C
:105220000198083105F07AFC002801D135123D4083
:105230002000FEF7ADFC0400E8E71D2BF8D10125A6
:105240006D42F5E7F0B580279DB0FFF71BFBA54C3D
:10525000A54D2068FF00391A4019FDF7ADFC236801
:105260000600C3182360002B0ED11DB0F0BD2068CE
:10527000391A2818FDF7A0FC236806001B182360C4
:10528000FDF730FB994B1860002EF0DC2B78FA2BE1
:1052900000D037E12368022B07DCFFF7DFFA002894
:1052A000E3D00120FFF7B2FADFE76878AC78023884
:1052B00018282BD802F0E8FE19002C00300034002A
:1052C000370040002A004A007C0086008A00A000C7
:1052D000F10002012A002A002A002A002A002A00DE
:1052E0002A002A002A002A001001FF2C0ED02000DC
:1052F000FFF71CFD00227E4BE100CA505B181A71BB
:105300002100009213001320FEF746FE0320C9E798
:105310002000FFF76DFDF9E72000FFF707FDF5E737
:10532000FFF7B6FDF2E7FFF7F9FB0020FFF7DAFE23
:105330007048FFF73BFDE9E7632CE7D86E4BA2000E
:10534000D25821001520FFF72BFCDFE7FFF7C8FA42
:10535000FF270400002CD9D025682B143B40152BC7
:1053600004D02000FEF714FC0400F3E7200008300E
:1053700005F0E6FB06000530FFF79EFAFB20FFF77D
:1053800037FA2D121D20FFF733FAE8B2FFF730FA93
:10539000F0B2FFF72DFA3012C0B2FFF729FA25005C
:1053A0002B1B9E42DDDD287AFFF722FA0135F7E755
:1053B00000211D2000910B000A00FEF7EDFDFDF716
:1053C0003FFCA3E72000FFF7FDFE9FE7FDF79CFAF7
:1053D00003AC4A4A64210090494B200005F03EFB93
:1053E00002232000237005F0ABFB23000200002104
:1053F0001620FFF75FFB89E700243D4AE300D558FC
:10540000002D27D06B689E00701DFFF755FA2B000A
:1054100000253200083321000120FFF74BFB2F004D
:10542000FFF75EFA2E00002818D1002F04D03A00B2
:1054300001212000FFF767FA002D04D02A00022185
:105440002000FFF760FA002E04D032000021200077
:10545000FFF759FA0134FF2CCFD157E7FF2103683A
:105460001A120A40A24209D11A140A400B2A08D182
:105470000B400CD0012B0CD0022B0CD0FEF788FB7C
:10548000D1E7132AFAD100252F002E00F6E70600F7
:10549000F4E70700F2E70500F0E70024FFF73EFB22
:1054A0002200210000942300DA20FEF775FDFF2280
:1054B0002100D2000E4804F0BFFF80E7012C02D18A
:1054C000FEF788FC22E7022C02D1FEF7C7FD1DE79C
:1054D0000120FFF707FE19E7002321001A001A2018
:1054E00087E7C046941A00209416002084120020FA
:1054F00050250020C8C80000482D0020DFC800004B
:10550000DAC80000FB2B00D0CBE62268042A00DCBE
:10551000C3E62E79E878574B360206439E4200DDFB
:10552000BFE6331D9A4200DCB7E6EB5CFE2B00D0F1
:10553000B7E66B78AC78771E1B2B61D019D8072B98
:1055400047D0082B1CD0012B18D1FF2C16D02000DF
:10555000FFF7ECFB6D79484AB31E009221002A0048
:105560000A20FEF719FD454BE400E0501B191D71A0
:1055700004E01D2B56D048D31E2B6AD0701D91E637
:10558000632CFBD86A79022A13D0032A1BD0012A84
:10559000F4D1E979AB79090219432B7AA4001B04F1
:1055A00019436B7A1B060B435B001343344AA35029
:1055B000E4E7002FE2DDB11E2F48FDF7A3FD304BDD
:1055C000A400E050DAE7AB79A4005A1E93419B0097
:1055D000ECE7632FD2DC03AD3A002A49280004F03F
:1055E0000FFF00232800EB55FFF708FE0028C5DB5E
:1055F000234B8000C25821001520FFF7D1FABDE7E8
:1056000039002048FFF75EFCB8E7FF2CB6D06A7976
:10561000022AB3D818490B2000912100B31EFEF7CF
:10562000BBFCABE7632F00DD6327002303A99F4288
:105630000ADCFB430022DB173B40CB181A70152015
:1056400000917B1C2100EAE7EA185279CA54013321
:10565000EDE7012C92D1002F90DD6B79002B03D068
:105660001C00322B00DD322464235C43064B1C609B
:1056700084E7C046F60300009A160020502500205B
:10568000482D0020991600200400002001207047BA
:1056900010B5064C200000F037FB0549200000F053
:1056A0005BFB0122034B1A6010BDC046C01A0020EC
:1056B000801A0600981A002010B501210D20FDF770
:1056C00029F901210E20FDF725F900210F20FDF712
:1056D00021F9044C200000F053FA1021200000F0C2
:1056E0006BFA10BDA01A002010B504680D20E30766
:1056F00003D56410FF2C03D91720FBF727FC10BD3E
:10570000FFF7DAFFE1B2024800F078FA0020F6E78E
:10571000A01A002010B5FFF7CFFF0021034800F0CA
:105720006DFA43000120184310BDC046A01A0020A6
:1057300010B5034A08210348FFF71AF910BDC04607
:105740000CC900004CC90000F8B5012306681E42D0
:1057500005D045681D4202D084681C4203D10D204B
:10576000FBF7F4FBF8BD76101520802EF8D86D10ED
:105770001620FF2DF4D86410FF2C01D91720EFE775
:105780000B4B1B68002B01D1FFF782FF094FF1B2D1
:10579000380000F078FBE9B2380000F07BFAE1B2A3
:1057A000380000F077FA380000F0D8FB0020D9E785
:1057B000981A0020C01A0020F7B501242300A04247
:1057C0001DDD0D682C421AD01A4B25411B684C6810
:1057D000002B01D1FFF75CFFE9B201272500164E2F
:1057E0003D40300000F04FFB002D0AD03C4130001E
:1057F000E1B200F04FFA300000F0B0FB00231800D7
:10580000FEBD042CF7D90F2322681340092BF2D1D7
:1058100063685B100193019BAB42ECDDAB00E318C6
:105820009968394204D04910C9B2300000F032FA08
:105830000135F0E7981A0020C01A0020144B70B50B
:105840001B6805000E00002B01D1FFF721FF114C52
:10585000EDB22900200000F016FBF1B2200000F0AC
:1058600019FA0021200000F019FB002801D0404265
:1058700070BD01222900200000F000FB200000F094
:10588000FAF90028FAD0200000F0FAF9F0E7C04653
:10589000981A0020C01A002010B501240368234282
:1058A00002D04168214203D10D20FBF74FFB10BD10
:1058B0005810802801D91520F7E74910FF2901D990
:1058C0001620F2E7FFF7BAFF40002043EFE710B5DC
:1058D0000400012814D105211820FFF7AFFF7F280D
:1058E0002BDC03007F3301DA7F20404264235B42DC
:1058F00058437F2102F05CFC052C00D1404210BDD2
:10590000032811D101001820FFF798FF7F2814DC2D
:1059100003007F3301DA7F20404264235B42584317
:105920007F2102F045FCEAE70020052CF5D1072194
:105930001830FFF783FF7F2802DD0138FF38D0E7FA
:1059400003007F3301DA7F20404264235B425843E7
:105950007F2102F02DFCD1E770B50120FFF7B7FFE2
:1059600004000320FFF7B3FF05000520FFF7AFFF9A
:105970006D43644340436419201804F029FC01F08E
:10598000F3F804F0EFFB43000120184370BD10B59D
:105990000120FFF79CFF43000120184310BD10B504
:1059A0000320FFF794FF43000120184310BD10B5FA
:1059B0000520FFF78CFF43000120184310BD10B5F0
:1059C00008211820FFF73AFF0300C00FC018012379
:1059D000401015304000184310BD0000F8B50123F9
:1059E0001C00984234DD0F683B4231D04E683500D0
:1059F0001D402DD1042E2BD90F2231680A40092ACF
:105A000026D173685C10202C00DD2024114B1B680C
:105A1000002B01D1FFF73CFE7F10F9B20E4F2200A0
:105A2000380000F02BFAA5420FDA380000F023F915
:105A30000028FAD0380000F023F90122AB00400022
:105A4000F31810439860AD18EDE70120640004439B
:105A50002000F8BD981A0020C01A002000207047CE
:105A600001207047002070470020704701207047D8
:105A700000207047002070470020704700207047CA
:105A800000207047002070470020704700207047BA
:105A900000207047704770477047000010B5034AF8
:105AA0000E210348FEF764FF10BDC0469CC90000EC
:105AB0000CCA000010B5FDF747F8FDF7E7F8FEF750
:105AC000C5FF0448FFF772F9FEF7CCFAFFF7E0F9DB
:105AD00010BDC04695CA000010B5FCF79DFE10BD74
:105AE00070B5002504AC24780573A94205D10A4B92
:105AF0000A4A23210A4804F015FC01600949920072
:105B000052589B0002715B58A400837163588560F2
:105B100043710223C37170BDADCA000012CB0000F7
:105B2000BBCA000070CB0000037B002B04D1437381
:105B30008373036101330373704700001FB5019144
:105B4000A02100240068C900D2B24450012A10D01C
:105B5000A24209D0032A0AD0074A8350074B019A70
:105B6000C250012343501FBD02221343F4E7042215
:105B7000FBE70622F9E7C0465405000024050000B3
:105B800010B50400FFF7D0FFA1222368A179D2004D
:105B900099506179064A2000995021790432995030
:105BA000044B19685A689B68FFF7C8FF10BDC046D0
:105BB0000C050000B41A00204BB2002B0FDB802331
:105BC0003F290FD81F290FD80F290FD807290FD821
:105BD00003290FD81B060168074A8B5070478023A2
:105BE0009B04F8E7DB04F6E71B05F4E75B05F2E747
:105BF0009B05F0E7DB05EEE7240500000368074A94
:105C000099501A00FC32D1680029FCD0A321C900A8
:105C100058580023C0B2D3607047C0461C0500002E
:105C200007B58022074BD2051A6000229A60023223
:105C30001A7111230E320093034905330348FFF70D
:105C40004FFF07BDB41A002000300040A01A00200A
:105C5000F8B505000E0017000024BC4208D02B68E0
:105C6000315D1B6828009847002801D00134F4E713
:105C70002000F8BD704710B51C3000F0A9F910BD28
:105C800010B51C3000F096F910BD10B51C3000F0B6
:105C9000A5F910BD70B5437E0D00002B01D1002089
:105CA00070BD6430040000F0A2F90028F7D1200094
:105CB000290000F070F90120F2E70000F7B5019328
:105CC000FA23002504009B0083600D4B45600833D8
:105CD00003601C300F00160000F052F92000643001
:105CE00000F04EF9074A2761B600B35820006375EB
:105CF000019B9B009B586576A576A375FEBDC046AB
:105D000050CB000070CB00000123A022C375837D1F
:105D10000E49C133FF33D2059B009950437DC133F7
:105D2000FF339B009950CC220169094B5204CA50A1
:105D300005220169243BCA50827D01690833CA509B
:105D40000269417D034BD1507047C0460C060000EC
:105D5000240500000C050000A022002310B50469F2
:105D6000D200A3500A4CA1420FD90A4C8C425B418D
:105D700009495B420B40CD21C9045B1804690749FE
:105D8000635005210369995010BDCC235B04F5E7EE
:105D9000A086010090D00300000098FD24050000BB
:105DA000F7B5040000200D000193824265D0160073
:105DB000402A00D9402627001C37380000F0F6F8AA
:105DC000B1232269DB00D550802201232169920092
:105DD0008B50A27E002A03D12269136222691360CC
:105DE0000025731EAB4207D1019B002B04D08022FB
:105DF0000221236992009950012223691A622369C2
:105E0000FC33DA68002A02D19A6A002AF9D09A6A29
:105E1000002A0BD1DA60A3232269DB00D1583800B5
:105E2000C9B2013500F0B7F8B542DAD3019B226957
:105E3000002B0FD11300FC339B6A002B0AD10133D6
:105E4000A376D3612369FC33DA6C002AFCD00022EC
:105E5000DA640AE000230121A37651611A00236964
:105E6000FC3399680029FCD09A602369FC339A6A54
:105E7000002A01D000229A62E8B2FEBD10B50123CB
:105E8000FFF78EFF10BD0300AC3310B5040019708E
:105E9000643000F08BF80123637610BD002302000C
:105EA00070B5AC3243760D001178B1220400006960
:105EB000D20081508022216992008B5022690133E7
:105EC00013622269936026006436300000F080F887
:105ED000002812D0300000F06DF81E4B2269D0501F
:105EE0002369FC331A6A002A02D19A6A002AF9D07F
:105EF0009A6A002A01D11A62E5E723690122002D7E
:105F00000DD11900FC31896A002908D1DA612369B1
:105F1000FC33DA6C002AFCD00022DA6407E05A6114
:105F20002369FC339A68002AFCD000229A60002082
:105F30002369FC339A6A82420BD098622169064A2F
:105F40008B588B501800022B03D0181F431E98410A
:105F5000033070BD1C050000C404000010B5012111
:105F6000FFF79CFF10BD000010B513231222024959
:105F70000248FFF7A3FE10BD00400040C01A0020F9
:105F800010B540220021040004F056FA002320003E
:105F90002364636410BD10B53F24026C531C23407E
:105FA000446C9C4201D08154036410BD00230364FF
:105FB00043647047436C026C934206D03F21C25C3D
:105FC00001330B4043641000704701204042FBE75F
:105FD000036C406C181A00D540307047436C026C5B
:105FE000934201D0C05C704701204042FBE73F2252
:105FF000036C406C01331340181A43425841C0B23D
:106000007047000003210A4802680A4302600948F9
:1060100002680A4302600849084A094B9B1A03DDDB
:10602000043BC858D050FBDC00F012F8FAF76CF8CB
:106030002405004054050040BCD0000000000020B2
:106040004C020020FEE7FEE7FEE7FEE7FEE7FEE784
:106050002D4B10B51A68D2B2012A0FD12B4A126803
:1060600012070BD12A4AE0241168F02208001040E0
:1060700021422DD12749096811422CD01A68D2B289
:10608000012A12D12149096809070ED1F0202049BF
:1060900009680140402908D11E490968014204D11C
:1060A0008020C121C005C90042501B68DBB2012B12
:1060B0000DD1164B1B681B0709D1154B1A68F0232D
:1060C0001A40A02A0FD1134A12681A420ED010BDEE
:1060D0003028CFD0D2E7104A104911608021104AF1
:1060E00009021160CAE7D02AF1D1ECE70D4B1A681A
:1060F000012A04D00C4A1A601A68012AFCD1C02275
:106100000A4B1A60E3E7C046E00F00F0E40F00F02E
:10611000E80F00F0EC0F00F004050040DFFF07C0BF
:10612000186C004000EC06407593000014EC06402B
:106130000120704710B503681322DB69984710BD32
:1061400070470000054B0269D1500369FC331A6A9D
:10615000002AFCD0002201201A6270471C050000B2
:10616000030010B55C331A781F231A401E3B190038
:106170009140114AD167C222042104699200A150C2
:10618000026953600269D360A02300220169DB0029
:10619000CA5001230169094A5B428B500169084AD0
:1061A0008B5001690C3A8B50016908328B501430C6
:1061B000FFF7FCFE10BDC04604E100E00C05000046
:1061C0001405000010B51430FFF702FF10BD10B524
:1061D0001430FFF703FF10BD10B51430FFF7EAFECF
:1061E00010BD0000030070B55E331A780469724B6D
:1061F000E25003005D331A780469704BE2500300EB
:1062000061331C7802696E4B012C00D09EE00500C2
:106210005F352E78A225ED005651020060321578C8
:10622000A1220669D200B5500269D4509623DB0042
:10623000994200D88CE096231B01994200D88AE04D
:1062400096235B01994200D888E096239B019942EE
:1062500000D885E0E1239B01994200D882E0962393
:10626000DB01994200D880E0E123DB01994200D8AC
:106270007DE096231B02994200D87AE0E1231B02BD
:10628000994200D877E096235B02994200D874E0E7
:10629000E1235B02994200D871E0E1239B0299421D
:1062A00000D86EE0474B994200D86CE0E123DB0256
:1062B000994200D86AE0E122002312038A425B413E
:1062C000414A5B421340802252059B1801693F4AB4
:1062D0008B50A02304220169DB00CA50002103690E
:1062E000FC33D9600369FC331962012301690B6037
:1062F00001698B60C1210469890062501F215C30F3
:1063000002780A4093406231314AFF3153500021F4
:10631000415600293CDA0F230B40083B2D4C9B08CB
:106320009B001B1903242140A140FC348C40DD69F3
:10633000A5432C00C0258D4029002143D9611F238E
:10634000017819401E3B8B40136070BD00246CE740
:106350009E23DB02BAE79D231B03B7E71E4BB5E77D
:106360001E4BB3E7EC239B03B0E71D4BAEE71D4B81
:10637000ACE71D4BAAE71D4BA8E71D4BA6E71D4B3D
:10638000A4E71D4BA2E78023DB049FE71B4B9DE79F
:106390008C080F4BA400E41803230B40FF21C025F9
:1063A000DB009940AD0066598E433100C0269E4007
:1063B00033000B436351C2E70C05000014050000D5
:1063C0006C05000090D0030000D0BEFE2405000044
:1063D00000E100E000ED00E000B0130000502700F5
:1063E00000A04E0000F0750000509D0000F0EB0092
:1063F00000903A0100E0D70100B0AF0300705F07E2
:10640000F7B5009308AB1B7800250193FA2304002D
:106410009B0083600E4B45600833036014300F000F
:106420001600FFF7ADFD23005C3327611E70009B53
:10643000084A9B00995823005D331970019B200086
:106440009B009A5823005E33DD701A70FEBDC04673
:10645000ECCB000070CB0000036910B51A00FC32D1
:10646000D2680400002A0AD0A322D200995814301E
:10647000C9B2FFF790FD00222369FC33DA6010BD3A
:1064800010B50248FFF7E8FF10BDC046781B00209A
:106490001D2307B502220093024901330248FFF78A
:1064A000AFFF07BD00200040781B002010B500287A
:1064B00001D004F07DFA10BD7047000010B500F067
:1064C00011F8FFF7F9FF012000F000FAFFF7F2FAE8
:1064D000FFF702FB024B002BFAD000E000BFF7E70A
:1064E00000000000C420114B80001A5810491140D0
:1064F000C02212020A431A50C0218022490092028F
:106500005A501A608023A3220021DB05D200995043
:106510000122F9309A60074BFF301950C120023137
:1065200080001950403019501A60704700E100E0B7
:10653000FF00FFFF00100140014B18607047C0468C
:1065400060000020F7B500231E285AD8384B800081
:10655000C258042A5BD007D8022A54D055D8042345
:10656000012A09D000234CE0062A54D051D31A2A1C
:1065700053D002231B2AF5D12E4A116808294ED97F
:1065800009294FD00A240226A02001252A4AC0004A
:1065900015502A482A4D07681C20BF00074029488B
:1065A000019700685759009027481B0207401F4376
:1065B000C02300989B020340FF2057515759000207
:1065C00007401F43019B1F43009B58016023184055
:1065D00007433E43565101251C4B1560586800285F
:1065E000FCD000205860A1230125DB00D358556062
:1065F000A025ED0050511BB2A14202D015D2611A64
:10660000CB401800FEBD0823B6E71023B4E72023D3
:10661000B2E74023B0E78023AEE70123ACE70824CC
:106620000026B1E70C000126AEE7091B8B40E8E726
:1066300070CB00005C0000200070004018000020BB
:10664000040500001C000020FF00FFFFFC7000405C
:10665000F0B51E285BD8364B8000C258354B1E68FB
:10666000002E30D1C227344BBF00D859334C0325FC
:106670000440C02000022043D851C0248020640080
:10668000800018512E4F18602E4B803CD859FF3C8B
:10669000A043D8510437D859A8432043D8510837CC
:1066A000D8590C35A8438446072065462843D8515D
:1066B000A820C0001E50C1208026800076021E50F7
:1066C0001C601C4B1C60142500202B001E4C2E004F
:1066D00046433659771C1BD14343E250A023032580
:1066E000C132FF329200DB05D550184B1A68082AD8
:1066F00014D114234343E3189A6812485132FF32ED
:10670000920059601150DA68C1239B00C250F0BD5D
:106710009642E1D001300328D9D1F8E7082A02D9FE
:10672000083AD140E5E708239A1A9140E1E7C046CC
:1067300070CB0000DC1B002000E100E0FF00FFFF49
:1067400004050000009000402000002060000020B0
:106750002149F0B54A6C2148002A14D0A025A12671
:1067600000230124ED05F600C258571C06D0C718B7
:106770007F68002F02D027009740AF5114333C2B85
:10678000F2D100234B64A0230121DB0500260F007A
:106790009C4614234B43C3181A1F1268104C0E4D0D
:1067A000920014195219526C002A10D01A00143A8F
:1067B0001268551C09D0103B1B68FF2B05D03B000D
:1067C000934065461A00074BEA50FC346664013179
:1067D0000429DED1F0BDC046FC900040200000201E
:1067E000009000400C05000000B51E2810D80C4A8F
:1067F0008000835803290BD8A0220800C133FF333F
:10680000D2059B0001F036FC020905070021D1509A
:1068100000BD0C21FBE70421F9E70321F7E7C0469F
:1068200070CB00001E280AD8074B8000C2580123F5
:106830009340A022D205002902D104495350704749
:10684000A121C900FAE7C04670CB00000C0500008A
:10685000030000201E2B0AD8A021A222C905D200C5
:106860008858034A9B009B58D84001231840704722
:1068700070CB0000F7B506000D000C008B180193DB
:10688000019B671B9C4207D0336821781B6830004E
:10689000984701340028F3D13800FEBD0849094A61
:1068A000094B10B51B688858FA22190A1B061843B1
:1068B0009200002301F0B4FD4904C00B084310BD51
:1068C0000010014004050000E01B002070B5041E0C
:1068D00009D0FFF7E3FF050000F014F8FFF7DEFF33
:1068E000401BA042F8D370BD0022044B9A60044ABA
:1068F00013680133DBB213607047C046FC100140DF
:10690000E01B002070470000F0B5C64600B5CB0F75
:106910009846404A4B005B0D9A1882B00D00040067
:10692000132A2FDC002A49DB3B4F17413E000E4063
:10693000064323D07F08390029400C430AD0374949
:10694000BD438C4663445C425C418023DB021341BF
:10695000E4071D434146CE0031492B008E19220029
:10696000346875682000290001F000FF0090019153
:106970000098019922002B0003F090F802B004BCAB
:106980009046F0BD332A08DD8023DB009A42F5D122
:1069900002000B0001F0EAFEF0E7224A94460122D1
:1069A00063445242DA400242E8D052080242D1D057
:1069B00094438022D2051A411443CBE74B005B0875
:1069C0000343DBD00B031B0B1C4363422343802494
:1069D0004D0C24031B0B23406D042B43190043462D
:1069E000DA000F4B9B181C685D6802000B0020004A
:1069F000290001F0BBFE009001910098019922004E
:106A00002B0003F04BF842464B005B08D60733439C
:106A10001900B3E701FCFFFFFFFF0F00EEFBFFFFD4
:106A200020CC0000EDFBFFFFF8B5274A4B005B0DC3
:106A30009A180C000700132A10DC002A36DB234BBF
:106A400013410B423AD080242403144100206418DF
:106A50009C430600250030002900F8BD332A0EDDD6
:106A600080230600DB000D009A42F4D102000B00E7
:106A70003800210001F07AFE06000D00EBE7144D0E
:106A80000600AC46012563446D42DD40AC466346DA
:106A90000D000342DFD033239A1A323B934018187B
:106AA000874200D94C1C63469843D2E7C90FCC07F4
:106AB0000020531CCDD1074B1C43CAE706000D0034
:106AC0000028C0D1C7E7C04601FCFFFFFFFF0F0051
:106AD000EDFBFFFF0000F03F30B5214A4B0087B0CF
:106AE0005B0893421EDD1F4A934205DD02000B0046
:106AF00002F0D4FF07B030BD02AA00F095F80323DE
:106B00001840049A059B012813D002281DD00028A4
:106B100014D00298039900F06FFB80231B069C465B
:106B20006144E7E7002300220093002301F0DEF830
:106B3000E0E70298039900F05FFBDBE7012402988D
:106B40000399009401F0D2F8D4E701240298039944
:106B5000009401F0CBF880231B069C466144C9E7F2
:106B6000FB21E93FFFFFEF7FF0B54746CE4680B5FA
:106B70008DB004000D0000F067FA294B06001B7869
:106B80000F005BB29846013310D022002B0020008A
:106B9000290003F0CBFA8146002807D10022002308
:106BA0002000290001F014FC002806D13000390033
:106BB0000DB00CBC90469946F0BD01230293194BD1
:106BC0000694079503934B460A9343460494059510
:106BD000002B15D0002300221900100002F0E2F86B
:106BE000434608900991022B0ED103F0B9FB2123F3
:106BF00003600A9B0193002B0CD1089E099FD5E7E7
:106C0000002300240893099402A801F0C1F9002888
:106C1000EFD1EAE703F0A4FB0A9B01930360ECE7E2
:106C20006400002030CC0000F0B54E464546DE46FC
:106C30005746E0B5E14B4C008FB09046894664085A
:106C40009C4200DC87E0DE4B9C4222DCDD4A0029CE
:106C500000DC92E0DC4B02F021FFDB4B06000F0072
:106C60009C4200D17EE1D94AD94B02F017FF0200C5
:106C70000B00414630000A604B60390002F00EFF05
:106C8000D34BD24A02F00AFF434601259860D960EF
:106C90006BE0D04B9C4200DC8FE0CF4B9C4200DD90
:106CA00055E1CE4A231592469A4451460905631A86
:106CB00019001D00040003F055FA03F089FA0200E0
:106CC0000B00200029000892099302F0E7FE002241
:106CD000C34B02F071FC0F00060003F043FA03F00F
:106CE00077FA04000D0002000B00300039000A940E
:106CF0000B9502F0D3FE0022B94B02F05DFC00229E
:106D000000230C900D9101F05DFB002800D192E171
:106D1000002300222000290001F054FB434243419C
:106D20000133B04A41460192022208A8009252461D
:106D300000F07CFB4B460500002B16DA8022434610
:106D40001206944642465B68454263445360D368EA
:106D50006344D36009E00B00020041460A604B60C7
:106D60000022002300258A60CB6028000FB03CBCC5
:106D700090469946A246AB46F0BD934B01F0F6FC17
:106D8000914B06000F009C4200D13DE18F4A904B91
:106D900001F0ECFC02000B00414630000A604B6041
:106DA000390002F07BFE894A894B01F0DFFC0125A6
:106DB00043466D429860D960D7E701F049F88A4AA6
:106DC0008A4B06000F0002F0F7FB0022884B01F00F
:106DD000CDFC03F0C7F9050003F0FAF9794A7A4BC4
:106DE0000490059102F0E8FB02000B00300039002E
:106DF00002F054FE754A06000F0004980599744B82
:106E000002F0DAFB029003911F2D00DCC7E0029A2A
:106E1000039B3000390002F041FE83468A46534608
:106E20005B0024155B0DE31A102B6CDD04980599AB
:106E3000D322674B520502F0BFFB02000B0030006B
:106E400039000292039302F029FE0A0001001300A8
:106E50000691079202003900300002F01FFE029AEC
:106E6000039B02F01BFE06000F0004980599614A7F
:106E7000614B02F0A1FB32003B0002F00FFE069EC8
:106E8000079F0B000200390030000292039302F0CA
:106E900005FE4B005B0D83468A46E41A312C32DD39
:106EA00004980599B822544B920502F085FB030023
:106EB0000C000200029303940B000698079902F05D
:106EC000EDFD02000B0006000F000698079902F086
:106ED000E5FD029A039B02F0E1FD484A029003910E
:106EE00004980599464B02F067FB029A039B02F057
:106EF000D5FD02000B00300039000292039302F02E
:106F0000CDFD83468A465A465346414630000A60C4
:106F10004B60390002F0C2FD029A039B02F0BEFDF5
:106F200044460B000200A260E3604B46002B00DBEE
:106F30001BE75B46236080231B065344636080236A
:106F40001B069C466144A060E1606D420DE70B00AA
:106F5000020002F0A3FD434600259860D960186046
:106F6000596002E7D3221A4B520502F097FD214ADD
:106F7000214B0D00040002F091FD02000B00414680
:106F800020000A604B60290002F088FD1A4B194A64
:106F900002F084FD434601259860D960E5E60200D1
:106FA0000B003000390002F079FD6B1E154A9B0082
:106FB0009B5883468A46A342A5D130E7FB21E93F8F
:106FC0007BD9024000004054FB21F93F3163621A33
:106FD00061B4D03DFB213941FFFFEF7FEAFBFFFFAA
:106FE00000007041B8CC000083C8C96D305FE43F39
:106FF0000000E03F7370032E8A19A33BC14920258E
:107000009A837B3938CC0000D3220C4B520501F017
:10701000ADFB0B4A0B4B04000D0001F0A7FB020077
:107020000B00414620000A604B60290002F036FD4B
:10703000034A044BB9E6032373E6C04661B4D03D6E
:107040007370032E8A19A33BF8B54746CE46674BAB
:1070500080B50A000F00190005003940994200D19F
:107060009BE004000100002F69DD3F1500D1B4E072
:107070005F4B12039C468023120B5B0313435B00A0
:10708000CA0F67449B184A00F80703D5D20F5B006C
:107090009B188A0079108C4600218020162489468E
:1070A00080030D189D4202DC29185B1B8144D50F1B
:1070B0005B00013C5B1952004008002CF1D100201C
:1070C0008046802020250027000609E08B425CD006
:1070D000D40F5B00013DE31852004008002D16D08C
:1070E000C4198B42F2DD27180E00002C49DB5B1A15
:1070F000A242894149425B1A121BD40F5B00013D39
:1071000080443100E31852004008002DE8D11343B9
:107110004ED143465B0837494A4688464946521095
:107120004244C90702D5802109060B4361460F0579
:10713000BD18180029000CBC90469946F8BD7B008C
:107140005B0803433900002BF5D0002F3CD1E30A44
:10715000153A6405002BFAD08020400303423FD14A
:10716000002700E00F005B00791C0342FAD02500E5
:1071700020208D40401A2900D71B2200C2401A430C
:1071800076E7FE43F60F8E19B1E79442A0D8271890
:10719000002CF6DB1E000023AEE702003B002800B7
:1071A000390002F009FA2A003B0001F0DFFAC2E7D9
:1071B0004346013303D0434601335B08ABE7012369
:1071C00098460023C144A6E73B00020002F066FC9B
:1071D00002000B0001F0E6FDADE713000022BBE763
:1071E0000127210020207F42C6E7C0460000F07F33
:1071F00001FCFFFF0000E03FF0B54746CE4680B5FA
:1072000087B000920193754B4F00814688467F08F6
:107210009F4263DC02F0A6FF002800D1D4E04A467A
:1072200043464846414602F0C7F904000D006C4A47
:107230006C4B02F0C1F96C4A6C4B01F097FA2200DA
:107240002B0002F0B9F96A4A6A4B02F027FC2200CF
:107250002B0002F0B1F9684A684B01F087FA22006E
:107260002B0002F0A9F9664A664B02F017FC2200D7
:107270002B0002F0A1F9644A644B01F077FA220076
:107280002B0002F099F9029003910022604B20003C
:10729000290002F091F9029A039B06000F002000DA
:1072A000290002F089F9009A019B04000D0048466C
:1072B000414602F081F902000B002000290002F093
:1072C000EDFB02000B003000390002F0E7FB02008A
:1072D0000B0000204F4902F0E1FB70E002000B00C0
:1072E00002F06AF904000D003D4A3E4B02F064F9D9
:1072F0003D4A3E4B01F03AFA22002B0002F05CF9C5
:107300003B4A3C4B02F0CAFB22002B0002F054F92E
:10731000394A3A4B01F02AFA22002B0002F04CF9CC
:10732000374A384B02F0BAFB22002B0002F044F936
:10733000354A364B01F01AFA2B00220002F03CF9D4
:10734000354B029003919F429FDD344B00229F42B8
:107350003DDC334900207B182E4916001F0002F047
:107360009DFB049005910022294B2000290002F08A
:1073700023F932003B0002F091FB029A039B0600C6
:107380000F002000290002F017F9009A019B040069
:107390000D004846414602F00FF902000B002000A4
:1073A000290002F07BFB02000B003000390002F0E4
:1073B00075FB02000B000498059902F06FFB07B003
:1073C0000CBC90469946F0BD00201249F7E7154BDA
:1073D000002604920593144FC5E7C046FFFF3F3EC9
:1073E000D43888BEE9FAA8BDC4B1B4BD9EEE213E32
:1073F000AD529C804F7E923E9015CB19A001FA3E73
:107400007751C1166CC1563F4C5555555555A53F42
:107410000000E03F0000F03F3233D33F0000E93F7F
:107420000000E0FF0000E73F0000D23FF0B5DE467D
:107430004E4645465746E0B5DC4CA5440D91140038
:107440001900A49A0993DA4B9200D6584D1E039066
:107450001821E01E0696029500F0AAFEC343010023
:10746000DB1719404B1C9A009B1ADB001B190B9170
:1074700005934C1B771918D4A59BA5009C463F1972
:1074800022AE6544013707E0286802F0A1FE01340E
:1074900003C60435BC4208D0002CF5DA00200021D8
:1074A000013403C60435BC42F6D1069B002B01DA39
:1074B00000F0FDFB069B03990133DB009A46099B14
:1074C000DA00944600920022914672AA0492B94AC8
:1074D0006144934688469AAB63449B44029B002BCD
:1074E00000DABCE15D4600260027039C4D442A6873
:1074F0006B6803CC02F060F802000B00300039002A
:1075000001F034F9083D06000F004445EFD1049B1B
:107510004B441E605F6008239C46E144D145DDD1A9
:107520000EA804218446494261448C46069A930081
:107530009C44614684460A910399083B63448C4607
:107540000C93009B009263449B46009A0498D100E0
:1075500003008C46634408911E685F68002A33DD8F
:10756000954980468C466244D300984470AB9A4655
:107570000EAB99460022914B3000390002F01CF806
:1075800002F0F0FD02F024FE00228D4B04000D00FD
:1075900002F012F802000B003000390002F07EFA0F
:1075A00002F0E0FD4B4601C39946434620001A68AD
:1075B0005B68290001F0DAF808235B429C46E0444E
:1075C00006000F00D045D5D1059B30001A003900C8
:1075D000984600F0DFFCFF2300229B0504000D000D
:1075E00001F0EAFF00F038FC0022764B01F0E4FFE6
:1075F00002000B002000290002F050FA0D000400E8
:1076000002F0B0FD814602F0E3FD02000B00200015
:10761000290002F043FA060040460F00002800DC73
:10762000EEE0009B18215A1E92000EAB9B58091ADF
:107630001D000D41A9448D405D1B0EAB9D501723CD
:107640001B1A1D41002D2DDD01239C46009BE144AA
:10765000002B00DC1CE20E9C0123002C00D0B5E0C6
:10766000009A012A09D099000EAA54580133002C1F
:1076700000D0ACE0009A9A42F5D1059B002B0EDDBC
:10768000012B00D1A8E1022B09D1009B0EA95A1EA3
:1076900092000EAB9B5807939B029B0A8B50022DC6
:1076A00000D1C1E0002300223000390000F08AFE42
:1076B000009B002800D194E2069A591E8A4210DCF1
:1076C000414A0A9894460EAA6344944600229B00BD
:1076D00063441C68043B22438342FAD1002A00D051
:1076E000C0E0069B0EAA013B9B00D358002B00D0A4
:1076F000B3E001220C9B043B596801320029FAD007
:10770000009B9C466244110007921A0001338B4291
:1077100046DC0B9863468046A59C4344A046099CE2
:107720009B00A1464A449844D30022AA9146049A59
:1077300099449446089BA59A6344844661449446C0
:107740009A468B00634400934346586802F040FD1C
:107750004B4618605960029B002B24DB4D46039C6E
:107760000026002701E0286869680CCC01F024FF9E
:1077700002000B003000390000F0F8FF083D060061
:107780000F005C45EFD153469E60DF6004239C46AA
:107790000433E0449C46009BE144E2449845D3D145
:1077A000079B0093D1E600260027ECE794FDFFFF3E
:1077B00000CE000018FEFFFFFFFFFF1F0000703E1D
:1077C0000000704100002040FFFFFF3F00218022A9
:1077D0005204141B0EAA5450009999420EDD0EA8B3
:1077E00084469B000EAA8900D25861446344CF4866
:1077F00000E01A68821A04C38B42FAD101243CE7E4
:10780000059B002B06D1009B0EAA013B9B00D5587F
:10781000ED1517E70022C64B300000F0F7FD0028F9
:1078200000D024E100253DE732003B000020C149A3
:1078300002F034F906000F00002C00D132E7059A5F
:107840000020BC4900F0A6FB02000B00300039000C
:1078500002F024F906000F0024E7012250E7002679
:10786000002754E64B46059A079388468B000EA9DD
:10787000CB58183A08950592002B0DD18C464146FD
:10788000AD4B43449B006344043B58680139183AAC
:107890000028F9D088460592059A0020A54900F0F5
:1078A00079FB434604000D00002B00DA05E29E0040
:1078B0000EAB9C464346DB0066449C46059370AB8A
:1078C0009946049F67440097306802F081FC2200CB
:1078D0002B0001F071FE002238607960974B200088
:1078E000290001F069FE083F04000D00043EB9457F
:1078F000EAD14AAB03939B4600239A46069B424635
:10790000994643460132029204934B46002B00DA1B
:10791000AAE080208A4B009D9846C0058949002630
:107920000027002408E008239C460835E04454451D
:1079300011DC4346186859682A686B6801F03CFE00
:1079400002000B003000390000F010FF0134060087
:107950000F00A145E7DA5B46C0C39B4601239C4666
:10796000009BE244083B0093029B9A45CDD1049BC7
:107970009846A49B022B00DD8EE0002B37DC1FD144
:10798000059B00271D00039B00249C461E006544A8
:10799000083E2A686B683800210000F0E7FE083DC9
:1079A00007000C00AE42F4D1089B002B03D08023CB
:1079B0001B069C4664443A0023000D990A604B6004
:1079C0000720079B18409B239B009D443CBC90468E
:1079D0009946A246AB46F0BD009B0EA95A1E9200E6
:1079E0000EAB9B5807935B025B0A8B5057E64346EE
:1079F000002B00DA70E100200021DB004AAAD61833
:107A000048AF32687368083E00F0B0FEB742F8D164
:107A1000089B002B00D025E10B0002004A984B99EF
:107A20000D9C2260636002F039F8434607000C00A9
:107A3000002B13DD01254CAEB14638002E0021008D
:107A40004C4601360CCC00F091FEA146B045F7DA69
:107A5000089B07000C00002B00D015E13A00230022
:107A60000D998A60CB60ABE70026002773E70123FE
:107A70009C46009BE1440225002B00DDEBE5320033
:107A80003B0000202B4902F009F806000F0009E630
:107A90000024F2E54AAB0393A49B032B00D08FE7AD
:107AA0004346002B00DC14E1039ADB009B461300E5
:107AB00091465B441E685F68234B43440293DB009E
:107AC000994448AB9A464B465C681B6818002100F5
:107AD00032003B000090019100F048FE04000D00D0
:107AE00002000B000098019901F0D8FF3B00320022
:107AF00000F03CFE4B469860D9601C605D60082336
:107B00005B429C46E14426002F00CA45DBD1434638
:107B1000012B00DCE3E0039A13005B441E685F68FE
:107B2000029BDB0099464A44904610E0FFFFFF00AD
:107B30000000E03F0000F03FFFFFFF3F0000703E0D
:107B4000C0CD0000FB21F93FFFFFFF1F98464346D1
:107B50005C681B681800210032003B000090019116
:107B600000F004FE04000D0002000B0000980199D3
:107B700001F094FF32003B0000F0F8FD4346039A09
:107B80009860D9601C605D60083B26002F009A4217
:107B9000DCD14D469446002600244746083565440E
:107BA0002A686B683000210000F0E0FD083D060007
:107BB0000C00AF42F4D1039B4A9F5D689968D86876
:107BC000089B002B65D08022120694460D9B6544CD
:107BD000604464441F605D609960D8601E615C61B0
:107BE000EEE69A464B460793059B30005A42390011
:107BF000089500F0CFF900223A4B06000F0000F084
:107C000005FC002824D0384B00223000390001F058
:107C1000D3FC02F0A7FA52460400950002F0D8FA0D
:107C20000022304B01F0C8FC02000B00300039008C
:107C300001F034FF02F096FA0EAA50510122059B82
:107C4000524418339046059393000EAAD45023E66D
:107C50005346300039009C0002F084FA0EAB1851F4
:107C6000D04619E680230D9A1B06CB18106053608E
:107C70000B0002004A984B9901F010FF43460700A1
:107C80000C00002B00DDD5E680231B069C466444D7
:107C9000E4E62B003A000D9D2A606B600A000300A9
:107CA000AA60EB60320023002A616B6188E6099BC1
:107CB000DB00009372AB049332E4A49B022B00DD43
:107CC000E8E6002B00DD92E600D079E600270024EC
:107CD0006AE6002600246EE70020002198E60026D0
:107CE000340068E7000070410000703EF0B5CE46F9
:107CF000474680B587B000920193474A4B008146C2
:107D000088465B08934207DC4146484602F02AFA5F
:107D10004146031E484666D04A46434648464146C9
:107D200001F04AFC04000D0002000B0048464146E9
:107D300001F042FC394A3A4B06000F0020002900AE
:107D400001F03AFC374A384B01F0A8FE22002B0024
:107D500001F032FC354A364B00F008FD22002B00C2
:107D600001F02AFC334A344B01F098FE22002B002C
:107D700001F022FC314B324A00F0F8FC0E9B0290DD
:107D80000391002B34D00098019900222D4B01F073
:107D900013FC029A039B049005913000390001F016
:107DA0000BFC02000B000498059901F077FE2200FD
:107DB0002B0001F001FC009A019B01F06FFE224AAA
:107DC00004000D00214B3000390001F0F5FB0200EA
:107DD0000B002000290000F0C9FC02000B004846FF
:107DE000414601F05BFE07B00CBC90469946F0BDE1
:107DF00002000B002000290001F0DEFB124A134BA9
:107E000001F04CFE32003B0001F0D6FB4A464346EF
:107E100000F0ACFCE7E7C046FFFF3F3E7CD5CF5A01
:107E20003AD9E53DEB9C2B8AE6E55A3E7DFEB157FB
:107E3000E31DC73ED561C119A0012A3F1111813F41
:107E4000A6F810110000E03F495555555555C53F5E
:107E500049004B0819007047474AF0B54F46914614
:107E60004B005B0D99444646D6464A46C0B50500D0
:107E70000C000E0088460700132A27DC002A4BDB83
:107E80003E4B13419A460B0052461340034318D011
:107E90003B4A3C4B2800210000F068FC00220023F4
:107EA00000F0AAFA002847D0002C04DA80234A46C2
:107EB0005B03134198444646534600279E433800CF
:107EC00031001CBC90469946A246F0BD332A08DD1D
:107ED0008023DB009945F4D102000B0000F046FC42
:107EE000EFE7294A9446012263445242DA4092461F
:107EF0000242E6D0224A234B2800210000F036FC43
:107F00000022002300F078FA002815D0002C1EDB98
:107F1000534646469F430FE0194A1A4B280021005A
:107F200000F024FC0022002300F066FA002803D0B1
:107F3000002C04DB0027002638003100C1E7640074
:107F4000640825430027002DF6D0104EF4E74B4679
:107F5000142B0BD03422D21A012393405D19BD4259
:107F600008D201239C462F00E044D1E7133B9C46F6
:107F7000E044CDE72F00CBE701FCFFFFFFFF0F0040
:107F80009C7500883CE4377EEDFBFFFF0000F0BFEE
:107F9000002070474B0070B55B0D14000A00002BE9
:107FA0001AD14B005B08034315D0234B002201F08C
:107FB00003FB224B9C422DDB0A004B005B0D363B42
:107FC0001F4DE318AB422ADC002B0DDD1D4C1B05B9
:107FD00022401A43110070BD1B4DAB42F0D102008C
:107FE0000B0000F0C3FBF6E71D00353519DA174B1F
:107FF00002009C4209DD0B001548164900F032F8DA
:10800000134A144B01F0D8FAE5E70B001248134964
:1080100000F028F8104A114B01F0CEFADBE702001D
:10802000E9E7084C363322401B05134319000022B0
:108030000B4B01F0C1FACEE700005043B03CFFFF0C
:10804000FE070000FFFF0F80FF07000050C3000085
:108050009C7500883CE4377E59F3F8C21F6EA50179
:108060000000903C30B54A00DB0FDB0752081A4392
:10807000110030BD02B4714649084900095C49004D
:108080008E4402BC7047C04603B4714649084000A4
:108090004900095A49008E4403BC70470022430836
:1080A0008B4274D303098B425FD3030A8B4244D3C0
:1080B000030B8B4228D3030C8B420DD3FF22090202
:1080C00012BA030C8B4202D31212090265D0030BC1
:1080D0008B4219D300E0090AC30B8B4201D3CB03B7
:1080E000C01A5241830B8B4201D38B03C01A5241F9
:1080F000430B8B4201D34B03C01A5241030B8B42FB
:1081000001D30B03C01A5241C30A8B4201D3CB02E5
:10811000C01A5241830A8B4201D38B02C01A5241CA
:10812000430A8B4201D34B02C01A5241030A8B42CD
:1081300001D30B02C01A5241CDD2C3098B4201D3E5
:10814000CB01C01A524183098B4201D38B01C01A63
:10815000524143098B4201D34B01C01A52410309DA
:108160008B4201D30B01C01A5241C3088B4201D389
:10817000CB00C01A524183088B4201D38B00C01A36
:10818000524143088B4201D34B00C01A5241411A5D
:1081900000D20146524110467047FFE701B500206A
:1081A00000F0F0F802BDC0460029F7D076E770472E
:1081B00003460B437FD4002243088B4274D3030948
:1081C0008B425FD3030A8B4244D3030B8B4228D3E9
:1081D000030C8B420DD3FF22090212BA030C8B420F
:1081E00002D31212090265D0030B8B4219D300E0AF
:1081F000090AC30B8B4201D3CB03C01A5241830B34
:108200008B4201D38B03C01A5241430B8B4201D3E3
:108210004B03C01A5241030B8B4201D30B03C01A0C
:108220005241C30A8B4201D3CB02C01A5241830A86
:108230008B4201D38B02C01A5241430A8B4201D3B5
:108240004B02C01A5241030A8B4201D30B02C01ADF
:108250005241CDD2C3098B4201D3CB01C01A524146
:1082600083098B4201D38B01C01A524143098B42CF
:1082700001D34B01C01A524103098B4201D30B01B8
:10828000C01A5241C3088B4201D3CB00C01A5241DD
:1082900083088B4201D38B00C01A524143088B42A2
:1082A00001D34B00C01A5241411A00D2014652413B
:1082B000104670475DE0CA0F00D04942031000D35A
:1082C0004042534000229C4603098B422DD3030AAF
:1082D0008B4212D3FC22890112BA030A8B420CD3BF
:1082E000890192118B4208D3890192118B4204D3E8
:1082F00089013AD0921100E08909C3098B4201D368
:10830000CB01C01A524183098B4201D38B01C01AA1
:10831000524143098B4201D34B01C01A5241030918
:108320008B4201D30B01C01A5241C3088B4201D3C7
:10833000CB00C01A524183088B4201D38B00C01A74
:108340005241D9D243088B4201D34B00C01A52414B
:10835000411A00D20146634652415B10104601D3D8
:108360004042002B00D54942704763465B1000D362
:10837000404201B5002000F005F802BD0029F8D008
:1083800016E770477047C046D0400B1C1141203A99
:1083900003D49C461341184363465242934018430A
:1083A0007047C0468446101C62468C46191C6346C2
:1083B00000E0C0461FB501F097F8002801D4002165
:1083C000C8421FBD10B500F0EFFF4042013010BDA4
:1083D00010B501F089F8002801DB002010BD012054
:1083E00010BDC04610B501F07FF8002801DD002067
:1083F00010BD012010BDC04610B501F011F80028D5
:1084000001DC002010BD012010BDC04610B501F0F8
:1084100007F8002801DA002010BD012010BDC04679
:10842000F0B5CE46474615042D0C2E0080B5070446
:10843000140C3F0C9946030C7E435D436743634332
:108440007F19340CE4199C46A54203D980235B02B2
:108450009846C4444B4643435143250C3604654477
:10846000360C2404A4195B19591820000CBC904642
:108470009946F0BDF0B54E4657464546DE46E0B556
:1084800043025B0A450083B00F1C99462D0EC60FB0
:10849000002D57D0FF2D24D08020DB00C0041843CE
:1084A000002381469A469B467F3D7C027A00FB0F63
:1084B000640A120E984623D0FF2A4BD0E300802492
:1084C0000020E4047F3A1C43AD186B1C474601931F
:1084D000534677403A000F2B48D87D499B00CB5834
:1084E0009F46002B00D085E008339A46063B9B460A
:1084F0007C027A00FB0FFF25640A120E9846DBD13E
:10850000002C00D090E0524601231A4392460120ED
:10851000DBE74C4658461700022824D0032800D138
:10852000CFE00022002301284DD15802D205400A95
:10853000FF071043384303B03CBC90469946A2461F
:10854000AB46F0BD002B5BD104239A46033B0025CC
:108550009B46AAE7FF35002C60D1524602231A43FE
:1085600092460220B1E7FF220023DEE74B461B0CB8
:108570009C464B462604360C180461463300220CF8
:108580006446000C43434E435043544380191A0C35
:108590001218964203D9802149028C4664441B0478
:1085A0001B0C1004C01883015E1EB341800E1843DB
:1085B000130C1B199B0103431C00230179D50123D4
:1085C00062081C401443019A7F32002A4DDD630784
:1085D00004D00F232340042B00D00434230103D5FF
:1085E0003C4B019A1C408032FE2ABCDCA3015B0A92
:1085F000D2B29AE70C239A46093BFF259B4654E7E3
:10860000180001F071FE4A46431F76259A40002368
:108610006D4291462D1A9A469B4646E752460323E1
:108620001A439246032050E7200001F05DFE431FED
:108630002D1A9C40763D002047E780230027DB036E
:10864000FF2272E7424666E74C463200584662E730
:1086500080234A46DB031A4222D01C4220D1234306
:108660005B025B0A4746FF225FE701239A1A1B2A37
:1086700021DC23000199D3409E318C401A00230055
:108680005C1EA34113435A0704D00F221A40042A48
:1086900000D004335A0111D49B015B0A002244E745
:1086A00080234A46DB0313435B025B0A3700FF2249
:1086B0003BE7019587E70022002336E701220023EC
:1086C00033E78023DB0323435B025B0AFF222CE7B3
:1086D00010CE0000FFFFFFF770B500283DD0C31794
:1086E000C5185D40C40F280001F0FEFD9E22121A3D
:1086F000962A07DCD2B2082833DD083885406802A4
:10870000400A23E0992A0BDD052329001B1AD940D2
:1087100003001B339D402B005D1EAB4119430D0030
:10872000052801DD431F9D402B000F490B406E07BC
:1087300009D00F263540042D05D004335D0102D544
:108740009F220B40121A9B01580AD2B24002D20556
:10875000400AE4071043204370BD0024002200209B
:10876000F4E76802400AF1E7FFFFFFFBF0B54F4670
:108770004646D6460C000903C0B5490A470F5E00BD
:1087800039431F03DB0F9C4665007B0A570F1F43CD
:108790006D0DE40F760DA146C000B846D200AB1BAC
:1087A00064457BD0002B5FDD002E00D0A4E03E00AE
:1087B000164300D112E15E1E002E00D09EE1871A02
:1087C0004346B84280410125C91A4042091A0B02AA
:1087D00000D431E149024E0A002E00D16EE1300092
:1087E00001F082FD0300083B1F2B00DD61E1202228
:1087F0003900D21A9E40D1409F400E439D4200DD79
:1088000051E15D1B6B1C1F2B00DD7CE12021C91A8F
:108810003D0030008F408840DD40791E8F4131009F
:1088200007222843D940002507433A40002A09D0AF
:108830000F233B40042B05D03B1DBB42BF417F4271
:10884000C9191F000B0200D426E26A1CC64B55054D
:108850006D0D9A4200D106E1C44AFF080A40530751
:1088600052023B43120B8EE0002B00D0B8E06B1C91
:108870005B055B0D012B00DC30E1871A4346B842F3
:10888000B641CB1A76429E1B330200D54CE13B0029
:108890003343A1D100220024002570E0002B00DC2E
:1088A000E5E0002E00D183E0AF4EB54260D08026D7
:1088B00036043743B846382B00DC3EE143461343C9
:1088C0001F007A1E97413F18874280414042091895
:1088D0000B0200D4B0E0A44B01359D4200D1C3E0AF
:1088E000A24A7B080A4001210F401F435108D307C9
:1088F00007221F433A4099E79B4EB54238D0802665
:1089000036043743B846382B00DDDCE01F2B00DC93
:1089100030E11E004746203EF740BC46202B04D0E5
:108920004026F31A46469E403243170063467A1E9D
:1089300097411F43CCE0002B00D104E24346134390
:1089400000D159E14B07C00818438023C9081B0315
:10895000194208D04546ED081D4204D14346D008CF
:10896000590708432900420FC9007F4D1143C00039
:108970004B07CA087C49C00803438D4268D01203E4
:108980006D05120B6D0D002112031800130B0A0D5B
:1089900012051A43764B2D0513402B435B00E40769
:1089A0005B08234319001CBC90469946A246F0BDC3
:1089B0003E00164312D05E1E002E00D000E1871844
:1089C0008742804141444042091801250B0233D5BA
:1089D000022585E764463300414610001D00C7E7C5
:1089E000002D00D0DAE00C000443F3D05C1C00D171
:1089F0009FE15D4CA64200D12FE1DB43382B00DD27
:108A000066E11F2B00DD83E120240500E41A0F003E
:108A1000DD40D940A0404346A7405B1A441EA04118
:108A200098462F433843171ABA429241434652425E
:108A3000991A64463500CAE607223A40002A00D057
:108A4000F6E64B07CA084849FF083B438D4296D1DA
:108A50001900114300D19EE1802109030A4312034A
:108A6000120B414D8FE71500002200238BE7002BEE
:108A700000D0C7E06B1C5F057F0D012F00DCF1E02B
:108A8000394DAB4200D1B9E085180A0085428941D1
:108A90004244494251180722CF076D082F43490825
:108AA0003A401D00C2E607223049ED1A31403A40F3
:108AB000BCE63E002838864000279FE6380001F0DB
:108AC00013FC20308EE6434613431F007A1E974165
:108AD000C71BB84280414042091A78E60E003B00AD
:108AE00006431343002D61D1002E00D0F4E0002B8B
:108AF00000D11BE164463900100039E71A4FBB4230
:108B00007AD03300FFE630001F3DE840202B03D031
:108B10004021CB1A9E4037437B1E9F4107220743CB
:108B20003A400021002589E7171A4346BA42B64168
:108B3000591A76428E1B64464EE61F2B00DDADE0CF
:108B400020264746F61AB740B9461700B246DF401E
:108B50004E463E4337005646B240561EB24117437A
:108B60004246DA408918AEE6FF070000FFFF7FFFAC
:108B7000FFFF0F8020264746F61AB740B946170078
:108B8000B246DF404E463E4337005646B240561E80
:108B9000B24117434246DA40891A99E77F4CA64210
:108BA0005BD0802424045B42214327E7002E0CD1B4
:108BB000002B00D1CBE0644639001000774DD7E69A
:108BC000764FBB4218D0330075E6002B14D04B070C
:108BD000C00818438023C9081B03194207D0FC08AA
:108BE0001C4204D17907D0080843E14621004C46D5
:108BF000420FC9001143C000684DB9E61D000022B4
:108C00000023C0E6002D5BD10D00054300D1E2E654
:108C10005D1C00D1B0E0614DAE421FD0DB43382B6C
:108C200071DC1F2B00DD96E020250F00ED1AAF4010
:108C3000B9460700AA46DF404D463D432F00554642
:108C4000A840D940451EA84188440743BF18974211
:108C500092415142414435003AE66446350041466E
:108C6000100085E60B000343002D00D063E6002BC7
:108C7000F5D04346134300D17AE6871887428041F6
:108C800007224144404209183A400B0200D4D5E67D
:108C9000434B01351940C9E5380069E61E004746D7
:108CA000203EF740BC46202B04D04026F31A46460F
:108CB0009E403243170063467A1E97411F4302E6E7
:108CC000364DAE42CAD080252D045B422943A6E72B
:108CD0000843411E8841A6E6002B00D148E6871ACA
:108CE0004346B842B641CB1A76429E1B33024BD55F
:108CF000171A4346BA429241591A5242891A072218
:108D000064463A4092E501430F00791E8F419DE78A
:108D10001C000F00203CE740202B03D04024E31A26
:108D200099400843411E884138437CE600220024D4
:108D300025E6171A4346BA429241591A5242891AF5
:108D40006446350043E541461000144D10E680228C
:108D50000024120380E61D000F00203DEF40BC46BA
:108D6000202B03D04025EB1A9940084307006346A7
:108D7000781E87411F4369E7871897429B4141440A
:108D80005B42C9183500A3E53B003343CED0072230
:108D900031003A4052E600231A00F4E5FF070000D4
:108DA000FFFF7FFFF0B55746DE464E464546E0B52D
:108DB000834607000E03480085B092461C00360B20
:108DC000400DCD0F002800D19DE0954B984239D041
:108DD0008023F6001B041E43924A7B0F33439946BF
:108DE000944603006344009300230026FF0002938F
:108DF00023031B0B98466300E40F52465B0D01945E
:108E000000D1B3E086498B4200D19EE04246D100BA
:108E1000802212040A435146490F11438B4681496F
:108E200052468C4600996344CB1A0021D20000932D
:108E30002B0063409A460F2E00D905E17A4BB6000D
:108E40009B599F465B463343994600D0B8E00223C6
:108E50000826002700900293CAE7CB463A00029901
:108E60000195019B9A46022927D0032900D180E26F
:108E7000012944D06D49009B8C4663441C00002CA2
:108E800038DD530700D013E2D2085B46DB0109D579
:108E90005946674B19408B468021C9008C46009B80
:108EA00063441C00634B9C4207DC5B4664055F0720
:108EB0005B0217431B0B620D02E000230027584A98
:108EC00000211B031C0B0B0D1B05234314055A4AE1
:108ED000380013401C4353466400DB0764081C43FE
:108EE000210005B03CBC90469946A246AB46F0BD79
:108EF0000122524201231B1B382B00DCADE1002272
:108F000000230027DCE75B46334399465ED0002E02
:108F100000D18AE1300001F0E7F903000B3B1C2B84
:108F200000DD7BE11D22D31A5A460100DA400839E0
:108F30008E4013005F46334399468F403F4B0026D7
:108F40001B1A00930023029352E7414653460B43FA
:108F50003B499B468C46009B634400935B46002B39
:108F60003BD1022300221E43022161E74346134303
:108F70009B4637D04346002B00D162E1404601F0CA
:108F8000B3F903000B3B1C2B00DD53E1020041460B
:108F9000083A914088461D21CB1A5146D9400B0012
:108FA00041460B439B46534693401A00009B25497C
:108FB0009C46604403008C4663440093002137E7DD
:108FC0000323B14600900C26029311E7002300937F
:108FD00001330426002702930AE70323C3461E43F6
:108FE000032125E701331E430022012120E700234E
:108FF0009A46802300271B03094A61E780234946DC
:109000001B03194200D1E2E05946194200D0DEE0CC
:109010000B431B0317001B0BA246014A50E7C04637
:10902000FF07000001FCFFFF50CE0000FF0300001F
:10903000FFFFFFFEFE070000FFFF0F800DFCFFFF9C
:1090400001F8FFFFF3030000D94500D9CBE000D1C0
:10905000C6E03C0048460027009B013B00935B466E
:10906000160E1B021E431302984633041B0C99462E
:10907000310C0191FFF798F84A4642430B04210C4A
:10908000050019438A4207D98919013D8E4203D848
:109090008A4201D9851E8919881A0199FFF784F837
:1090A00009048C464A46210464464243090C0300E5
:1090B00021438A4204D98919013B8E4200D8F1E04C
:1090C0002D041D43AB464346891A4246280C120420
:1090D0001D0C5B46140C22001B041B0C5A4303940A
:1090E0006B434443029568431B19150CEB189C42D3
:1090F00003D980246402A44660441C0C15041B049C
:109100002D0C20185D19814277D373D00C1AA24A16
:109110007D1BAF42BF419446009B7F426344E01BEE
:109120001C00864200D1DBE00199FFF73DF84A467A
:1091300042430B04290C070019438A4207D98919B5
:10914000013F8E4203D88A4201D9871E8919881AA5
:109150000199FFF729F809044A46894629044D4632
:109160004243090C030029438A4207D98919013B6C
:109170008E4203D88A4201D9831E89193F04891A75
:109180003A00039F1A43380013041B0C58438146CE
:109190000298150C6F43434345434846000C8446F0
:1091A000DB1963449F4203D9802040028446654412
:1091B00048461F0C00041B04000C7D191818A94216
:1091C00000D284E000D17FE001231A4357E68023D8
:1091D0004A461B0313431B031B0BAA466F4A6FE649
:1091E000BA4200D935E74B46DC0758087B081C43D8
:1091F000FF0734E70024AF4289D247444745A441E2
:109200005B466442A4196418013BA6421ED2A042E8
:109210006DD800D1B6E0241A9B4678E703005A4681
:10922000283B9A400027914688E6584601F05CF8B2
:10923000203072E603005246283B9A4093460022B3
:10924000B4E6504601F050F820309AE6A642E2D14A
:10925000B845DCD9341A9B4659E71F2B65DC504CC6
:109260000099A4465C46614408008C40110082408D
:10927000D940501E82410C4314435A46DA40130031
:10928000620709D00F222240042A05D02200141DB3
:109290009442894149425B181A0262D50122002397
:1092A00000270DE68A4200D80AE7831E891907E7DE
:1092B0000F231340042B00D1E6E5171D974292417E
:1092C00053429B44FA08E0E5002800D1D7E5711825
:1092D000531EB14227D3A94215D358D01A0073E7C1
:1092E000002B00DC04E6012300229B44CDE5022391
:1092F0004744474589415B429C46494289190C19BC
:10930000E344241A03E743465F0047459B41B846C0
:109310005B429E19023A8919A94200D054E74045A0
:1093200000D051E7ABE51A00F6E71F215F4649423E
:109330000C1BE740202B07D01A49009B8C46634446
:1093400018005B4683401A43501E82413A43072768
:109350000023174009D00F210023114014000429D5
:1093600095D122005F075B021B0BD2081743002236
:10937000A6E5802359461B030B431B0317001B0B59
:10938000064A9DE5BD42B2D89B460024BFE6804513
:10939000B9D31A00C3E7C046FF030000FF0700006F
:1093A0001E0400003E040000F0B54F464646D64677
:1093B0008446C0B58046194E18030F034D00000BBC
:1093C0005C0082463F0B6D0DC90F9146640DDB0FAB
:1093D0000120B5420AD0B44203D0A54201D157457D
:1093E0000CD01CBC90469946A246F0BD66463E4352
:1093F000F7D1AC42F5D154461443F2D10120C8450F
:10940000EFD1994207D0002DEBD163461F433800BE
:10941000471EB841E5E70020E3E7C046FF0700002C
:10942000F0B54F464646D6464D00C0B50E03C90FAF
:109430008A462C491F035C008046360B6D0D914611
:109440003F0B640DDB0F8D421ED08C4216D0002DD9
:109450001ED130438446002C01D13A4323D06246CA
:10946000002A1AD09A4529D05146022001390840D5
:1094700001381CBC90469946A246F0BD3900114304
:10948000E5D002204042F4E73043FAD1AC420FD09D
:10949000002C0FD13A43E7D00CE00122013B93436B
:1094A00018000130E5E763460020002BE1D0DBE740
:1094B0003A43E6D19A45D7D1A542D5DCA54205DB92
:1094C000BE42D1D808D00020BE42D2D2504601239D
:1094D000013898430130CCE7C845C5D80020C845BD
:1094E000F4D3C6E7FF070000F0B54F464646D64620
:1094F0004D00C0B50E03C90F8A462E491F035C00FC
:109500008046360B6D0D91463F0B640DDB0F8D428F
:1095100018D08C4211D0002D18D130438446002C35
:109520001ED13A431CD163460020002B30D0514657
:1095300002200139084001382AE039001143EAD0FD
:10954000022025E03043FBD1AC4226D0002C26D1AE
:109550003A4324D15146022001390840013817E02E
:109560006246002A0FD09A45E1D1A54205DBBE42F2
:10957000DDD819D00020BE420AD25046012301385E
:109580009843013004E00122013B9343180001306D
:109590001CBC90469946A246F0BD3A43D0D19A45AC
:1095A000C5D1A542C3DCE0E7C845C0D80020C84506
:1095B000E3D3EDE7FF070000F0B55746DE464E4621
:1095C0004546E0B5834606000F03480087B0924643
:1095D0001D003F0B400DCC0F002800D16FE0DE4B8B
:1095E000984238D08023FF001B041F43730F3B4376
:1095F0000193DA4B0027994600239B46F6008144ED
:109600002B0369001B0B52469846490DED0F0029AC
:1096100000D185E0D04B994200D173E04346DA0097
:1096200080231B0413435246CC48520F84461343F5
:10963000524600206144D2008944210069400091D3
:109640008C46012149448A460F2F00D990E0C44935
:10965000BF00CF59BF465B463B43019300D06AE150
:1096600002230827002681469B46C9E73200584658
:10967000019B61460091022800D175E0032800D1CA
:10968000FEE1012800D02CE1002300270026002560
:109690003F032A0D3F0BB34812053A4302401B0516
:1096A0001343009A5B00D1075B080B43300019009D
:1096B00007B03CBC90469946A246AB46F0BD5B461F
:1096C0003B43019300D12FE1002F00D1A5E13800E9
:1096D00000F00AFE03000B3B1C2B00DD96E11D226F
:1096E000D31A5A460100DA405E4608398F4013000B
:1096F0008E403B4301939C4B00271B1A9946002345
:109700009B467DE7414653460B4393498C46E144D3
:10971000002B00D01AE102220220174300228CE71E
:10972000134300D10DE14346002B00D181E14046B7
:1097300000F0DAFD02000B3A1C2A00DD72E10100A4
:10974000434608398B4098461D239A1A5346D34006
:109750001A004346134352468A404946081A824932
:1097600089468144002068E77B4B002700268EE76E
:10977000140C1204120C1100370C3604350C79430A
:1097800028008C462E0060436044834656432100E7
:10979000300C80465846794340440291844506D9AE
:1097A0008846802149028C46E044414602913604B5
:1097B000010C360C00048B4681191E0C1B041B0C7B
:1097C0000391190079438C46280075436544A846E7
:1097D0005843050C45447743A94203D980214902E7
:1097E0008C466744290C8C4639000004000C2D047B
:1097F0002D186144AB4405915946049101990F0419
:109800003F0C080C390051434243904602008C46FD
:10981000090C8B4662437C4344445C44A04503D915
:109820008021490288464244210C88466146090449
:10983000090C8C4639005943434370437E430F0C57
:10984000F6182404BE19644442448C46B34203D93A
:1098500080235B0298464044029B61469846049BE5
:10986000370443449B46AB45AD416B420D0405991B
:109870002D0C8C467F196744FD18A8465D462D19AE
:10988000A542A44193466442A446C344DC448F42AB
:10989000BF4198459B4193459241A445A4415B42F9
:1098A0007F421F43360C52426442BF192243BF1805
:1098B000624638184302D20D039913436A020A43E1
:1098C000501E82416146ED0D2A434E023243D901BA
:1098D00000D4B3E00126500832400243DE07324391
:1098E0005B08224C5444002C62DD510709D00F2044
:1098F0001040042805D0101D9042924152429B18FE
:109900000200D90104D580241948E40003405444DE
:109910001848844200DD27E75E075B02D2081F0B70
:10992000630516435B0DB2E6002399460133042715
:1099300000269B4664E60323019781460C279B463D
:109940005EE6012201201743002276E6032303206E
:109950001F43434671E6C046FF07000001FCFFFFBE
:1099600090CE0000FFFF0F800DFCFFFFFF03000003
:10997000FFFFFFFEFE0700000023802700933F0348
:109980000026434B83E6019B3200A446584670E60E
:10999000AC466EE6802701993F0339422DD03B4209
:1099A0002BD11F433F033F0B00951600384B6EE64B
:1099B00001252D1B382D00DD66E61F2D40DC3548C6
:1099C0001C005044160082408440EE40501E8241EC
:1099D00034431443EB40620709D00F222240042A8B
:1099E00005D02200141D9442804140421B181A02E7
:1099F0003ED501230027002649E68027019B3F032F
:109A00001F433F033F0B0094214B40E603005A469F
:109A1000283B9A40002601926DE6584600F064FC0F
:109A2000203057E603005246283B9A40130000229C
:109A300093E6504600F058FC20307BE6CA4650E7DB
:109A40001F201E004042041BE640202D03D0124C74
:109A50005444A3401A43501E824132430726002734
:109A6000164009D00F200023104014000428B9D15B
:109A700022005E075B021F0BD2081643002306E696
:109A800080273F031F433F033F0B1600004BFEE5BB
:109A9000FF0700001E0400003E040000F8B5574612
:109AA0004E464546DE460C000903E0B5490A460F1E
:109AB0005F0031431E03DB0F760A9B46530F33438F
:109AC000C84E6500C000E40FD2006D0DA24681466D
:109AD0007F0D9C469046B74200D1B9E05B46012617
:109AE00073409B46EE1BA34500D183E0002E63DD4F
:109AF000002F00D0B1E06346134300D123E1731E71
:109B0000002B00D0BAE1861A6346B042804101259D
:109B1000C91A4042091A0B0200D447E149024B0A14
:109B200098464346002B00D189E1404600F0DCFB1B
:109B30000300083B1F2B00DD7CE120223000D21AFD
:109B40004146D040994002009E400A439D4200DDBC
:109B50006AE15D1B6B1C1F2B00DD94E120211000CE
:109B60003500C91A8E40DA408840DD40711E8E41B2
:109B7000110007222843002506433240002A09D05D
:109B80000F233340042B05D0331DB342B641764238
:109B900089191E000B0200D43DE26A1C914B550549
:109BA0006D0D9A4200D119E18F4AF6080A40570715
:109BB00052023743120B9BE0002E00D0C5E06E1C12
:109BC0007605760D012E00DC48E16746861ACB1B30
:109BD000B042BF417F42B8461F004346FF1A3B00D8
:109BE000B8461B0200D55FE137439AD1002200241A
:109BF000002579E0002E00DCFAE0002F00D18DE096
:109C0000784B9D4267D0802367461B041F43BC46A8
:109C1000382E00DC52E1634613435A1E93411E184E
:109C200086428041404209180B0200D4BEE06D4BD1
:109C300001359D4200D1D2E06B4A73080A400121F0
:109C40000E401E435108D30707221E43324095E7BA
:109C50001E00164300D045E740E7624B9D423AD0D4
:109C6000802367461B041F43BC46382E00DDEBE013
:109C70001F2E00DC3AE133006746203BDF403B000B
:109C8000202E05D04027BF1B6646BE40324390467B
:109C90004646721E96413343DAE0002B00D114E2AF
:109CA0006346134300D168E180234E07C008C9080A
:109CB0001B030643194208D06046C008184204D16D
:109CC00063460100D2085E071643F3009946C900B7
:109CD000720F444D11434B46DE08424B4F0737434A
:109CE000CA089D4200D16EE012036D05120B6D0D86
:109CF00000211203130B0A0D12051A433B4B2D05CD
:109D000013402B435B00E4075B0823433800190032
:109D10003CBC90469946A246AB46F8BD6346134309
:109D200011D0731E002B00D007E1861886428041B7
:109D300061444042091801250B0237D502257BE713
:109D40003E00614691463500C5E75C46002D00D0D7
:109D5000E1E00B000343F3D0731C00D1ACE1214BD5
:109D60009F4200D13AE1F343382B00DD6FE11F2B16
:109D700000DD8CE120250E00ED1AAE40B046060055
:109D8000AA46DE40454635432E005546D940A840F8
:109D90006346451EA8415B1A9C463043161AB242E0
:109DA000924163465242991A3D00B4E6072232407E
:109DB000002A00D0E4E60B4BF6084F073743CA08E9
:109DC0009D4200D090E73B00134300D1A6E18023E1
:109DD0001B031A431203120B024D89E715000022E0
:109DE000002785E7FF070000FFFF7FFFFFFF0F80D1
:109DF000002E00D0C7E06B1C5E05760D012E00DC46
:109E0000F0E0C84DAB4200D1B9E085180A008542A8
:109E100089416244494251180722CE076D082E43FA
:109E2000490832401D00A9E6BF49ED1A114007223A
:109E30003240A3E6320028388240002686E6300011
:109E400000F052FA203073E6634613435A1E9341E2
:109E5000C61AB04280414042091A5CE60E006746CD
:109E600006431743002D5ED1002E00D0F3E0002FF3
:109E700000D11EE15C46614691462CE7A94FBE42E7
:109E80007BD01E00F1E610001F3DE840202B03D0E0
:109E90004021CB1A9A401643731E9E410722064367
:109EA00032400021002583E7161A6346B242804102
:109EB000591A40420B1A98465C4632E61F2E00DDC6
:109EC000ABE02027BB1B9A4663465746BB409946EA
:109ED00013004F46F3401F433B005746BA40571EFE
:109EE000BA4113436246F240891898E62027BB1B0B
:109EF0009A4663465746BB40994613004F46F34087
:109F00001F433B005746BA40571EBA4113436246AF
:109F1000F240891A9CE7834B9F425FD080252D0435
:109F20007342294320E7002E0CD1002F00D1D0E04E
:109F30005C46614691467B4DCDE67A4FBE421CD0D1
:109F40001E0065E6002F18D0C0084E07064380208B
:109F5000C9080003014208D06346DC08044204D16A
:109F60002100DA46D2085E071643F3009946012421
:109F70005346C900720F11431C406A4DABE61D00E9
:109F800000220027B4E6002D59D10B00034300D175
:109F9000D6E6731C00D1B2E0624B9F421ED0F34361
:109FA000382B6FDC1F2B00DD97E020250E00ED1A0B
:109FB000AE40B0460600AA46DE40454635432E0078
:109FC0005546A840D940451EA8418C440643B618C2
:109FD00096429241514261443D0025E63D00614672
:109FE000914678E60B000343002D00D055E6002B88
:109FF000F5D06346134300D16DE686188642804152
:10A0000061444042091800220B0200D4D0E6464BBE
:10A0100001351940B2E5B1465DE633006746203BA5
:10A02000DF403B00202E05D04027BF1B6646BE40C8
:10A03000324390464646721E96413343EFE5394B14
:10A040009F42CBD080252D0473422943A8E70843C3
:10A05000411E8841A2E6002F00D13CE66346861AE5
:10A06000CF1AB0429B415B42FB1A98461B024ED569
:10A07000161A6346B2429241591A5242891A5C46F4
:10A0800000227BE501430E00711E8E419FE71D00FB
:10A090000E00203DEE40B046202B04D04025EB1AA8
:10A0A00099400843814648464346411E884118432B
:10A0B00074E60022002417E6161A6346B242924163
:10A0C000591A5242891A3D0025E561469146154DBF
:10A0D00001E680220024120379E61D000E00203DD7
:10A0E000EE40B046202B04D04025EB1A994008439F
:10A0F00081464E464346711E8E411E4367E78618D1
:10A1000096429B4161445B42C9183D008CE547463D
:10A110003743CED007224146324049E600273A0075
:10A12000E6E5C046FF070000FFFF7FFF70B50C4E5D
:10A130000D031C0349005B002D0B490D240B5B0D27
:10A14000B14208D0064900208B4203D114432000BD
:10A15000441EA04170BD05430120002DFAD1F1E756
:10A16000FF07000030B5144D0A034B00120B5B0DC6
:10A17000C90F0024AB4211DD104CA34210DC802437
:10A18000640322430E4CE41A1F2C0CDD0D48C31A45
:10A19000DA4013005C42002900D11C00200030BDD1
:10A1A000094BCC18FAE7094DE040AC4663449A40AD
:10A1B00013000343EEE7C046FE0300001D04000049
:10A1C0003304000013040000FFFFFF7FEDFBFFFFDF
:10A1D00070B500282DD0C317C5185D40C40F2800E6
:10A1E00000F082F8154B1B1A5B055B0D0A2815DD84
:10A1F0000B38854000222D032D0B002110002D036C
:10A200000A0D2D0B12052A430D4D1B052A40134341
:10A210005B00E4075B082343190070BD02002900BE
:10A22000153291400A000B21081AC5402D032D0B51
:10A23000E3E70024002300250022DEE71E040000DF
:10A24000FFFF0F804100090E4B1C70B5DBB24602C8
:10A25000750AC40F012B14DDE0239B006D07360B3C
:10A26000CB1800210A0D280012051C4D32435B0556
:10A270002A405B0813435B00E4075B082343190093
:10A2800070BD002914D1002D1ED0280000F02CF83C
:10A290000A281CDC0B232A001B1ADA4003001533A2
:10A2A0009D400F4B12031B1A5B05160B5B0DD8E785
:10A2B000002D06D0320B802636036D071643094B5E
:10A2C000CFE7084B0026CCE700230026C9E70300B0
:10A2D0002A000B3B9A400025E3E7C046FFFF0F80B2
:10A2E00089030000FF0700001C2101231B04984282
:10A2F00001D3000C10391B0A984201D3000A083917
:10A300001B09984201D30009043902A2105C4018CD
:10A310007047C04604030202010101010000000071
:10A320000000000030B51C00094B05001B6885B01B
:10A33000D868084B002A01D1074B1A0002920193FA
:10A3400000912B002200054900F026F800F08EFD58
:10A3500068000020D0CE0000F6BD0000DDCE000079
:10A36000014B18687047C04668000020084B10B5C4
:10A370000400002B02D0002100E000BF054B18684C
:10A38000836A002B00D09847200001F045FBC046AF
:10A39000000000000CCF00000EB403B5010003ABB9
:10A3A000044804CB0068019300F076F802B008BCC2
:10A3B00003B018476800002070B500260C4D0D4C06
:10A3C000641BA410A64209D1002601F027FB0A4D08
:10A3D0000A4C641BA410A64205D170BDB300EB5813
:10A3E00098470136EEE7B300EB5898470136F2E79D
:10A3F00038020020380200203802002048020020E5
:10A40000002310B59A4200D110BDCC5CC454013376
:10A41000F8E710B5884202D98B18984203D300237D
:10A4200007E08B5C8354013AFBD210BDCC5CC45472
:10A4300001339A42FAD1F8E703001218934200D18F
:10A44000704719700133F9E7936810B5013B9360C9
:10A45000002B04DA9469A34207DB0A2905D01368AC
:10A46000581C10601970080010BD00F033FC01008A
:10A47000F9E7F8B506000F001400D518AC4201D179
:10A48000002007E021783A003000FFF7DDFF0134BB
:10A49000431CF3D1F8BD0000F0B59FB002900F004F
:10A4A00016000593002805D083690493002B01D181
:10A4B00000F0DCFD7B4B9F425BD1029B5F68BB8958
:10A4C0001B0762D53B69002B5FD0002306AC63619C
:10A4D000203363761033A37635002B78002B01D020
:10A4E000252B5CD1AB1B04930CD0320039000298B1
:10A4F000FFF7BFFF431C00D1C4E06269049B944690
:10A50000634463612B78002B00D1BBE00122002360
:10A510005242626002A9543252186E1C2360E360FA
:10A52000A3601370A365317805225F4800F0BCFE7C
:10A53000751C002835D12268D30604D5532302A9FF
:10A540005B1820211970130704D5532302A95B1847
:10A550002B21197033782A2B2CD0350000210A20AA
:10A56000E3682A786E1C303A092A64D900292ED073
:10A5700026E04E4B9F4202D1029B9F689FE74C4BC7
:10A580009F429CD1029BDF6899E73900029800F056
:10A59000F7FB002899D0012040421FB0F0BD0135E3
:10A5A0009BE7414B2268C01A012383401343236079
:10A5B0002E00B8E7059B191D1B680591002B01DBD8
:10A5C000099304E05B42E3600223134323602B788A
:10A5D0002E2B0AD16B782A2B35D1059B02351A1DFB
:10A5E0001B680592002B2BDB0793324E2978032240
:10A5F000300000F059FE002806D04023801B834025
:10A600002268013513432360297806222A486E1CEC
:10A61000217600F049FE00283AD0284B002B25D1A6
:10A620000722059B07339343083305936369039A15
:10A630009B18636150E7434301219B18350090E765
:10A6400001235B42D0E700230A201A000135636032
:10A6500029786E1C3039092903D9002BC5D00792FF
:10A66000C3E74243012352183500F1E705AB0093DD
:10A670003A00134B2100029800E000BF0390039BB7
:10A680000133D3D1BB895B0600D584E70B9884E7FF
:10A6900005AB00933A000A4B2100029800F080F8C5
:10A6A000ECE7C04664CF000010CF000084CF00006C
:10A6B00044CF000016CF00001ACF000000000000B9
:10A6C00073A40000F7B5150001938A680B69009028
:10A6D0000C00934200DA130022002B604332127800
:10A6E000002A01D001332B6023689B0602D52B681A
:10A6F00002332B60062723681F4027D023004333F3
:10A700001B785A1E93412268920630D42200019988
:10A7100043320098089EB047431C25D0062320688A
:10A720002A68E16803400025042B03D18D1AEB430E
:10A73000DB171D40A3682269934201DD9B1AED18C7
:10A740000027BD4220D1002010E00137E3682A68CD
:10A750009B1ABB42D2DD22000123193201990098D5
:10A76000089EB047431CF0D101204042FEBD30207E
:10A77000E1184331087021005A1C45310978A218AC
:10A78000433202331170C1E7220001231A320199CA
:10A790000098089EB047431CE6D00137D1E700007F
:10A7A000F0B589B004920A004332059303900292F7
:10A7B0000A7E0C000E9B6E2A00D186E01FD8632A09
:10A7C00033D008D8002A00D18CE0582A4DD025007B
:10A7D00042352A7030E0642A01D0692AF7D119681D
:10A7E00025680A1D280629D508681A60002803DA9A
:10A7F0002D23029A404213706B4E0A274FE0732AB2
:10A8000074D008D86F2A1FD0702AE0D1202209689E
:10A810000A43226003E0752A16D0782AD7D1220095
:10A82000782145321170614E22E025001A684235C8
:10A83000111D196013682B70012365E008681A6008
:10A840006906D3D500B2D1E719682568081D1860DC
:10A8500008682E0605D5544E08276F2A1BD00A27F4
:10A8600019E06D06F7D580B2F5E745314E4E0A7016
:10A8700018682268011D00681960150621D5D307E4
:10A8800002D520231A4322601027002803D1202359
:10A8900022689A4322602300002243331A706368BF
:10A8A000A360002B58DB042221689143216000281B
:10A8B00054D1029D002B5AD02500337842352B709D
:10A8C00055E05506DBD580B2D9E71A680D68101D32
:10A8D0004969186013682E0601D5196002E06D06FB
:10A8E000FBD519800023029D23614FE01A68111DDA
:10A8F0001960156800216268280000F0D5FC002866
:10A9000001D0401B6060636823610023029A1370CA
:10A910003CE023692A0004990398059DA847431C3D
:10A920003ED023689B0715D4079BE068984239DA2C
:10A93000180037E022000123193204990398059E7C
:10A94000B047431C2CD00135E368079A9B1AAB42F1
:10A95000F0DCE9E70025F7E70028ADD0029D3900DB
:10A96000FDF722FC735C013D2B700028F7D1082F06
:10A9700009D12368DB0706D563682269934202DCAC
:10A980003023013D2B70029B5B1B2361059B07AAB3
:10A9900000932100049B0398FFF794FE431CB8D159
:10A9A0000120404209B0F0BD21CF000032CF0000AD
:10A9B0000D4B70B51C680500A36B002B0FD1182040
:10A9C00000F056FC094BA0630360094B0122436071
:10A9D000084B83600B2383810023026143610022C3
:10A9E000A36B1D615A6170BD680000200E33CDABB2
:10A9F00034126DE6ECDE0500124B10B51C68A36B3B
:10AA0000002B0FD1182000F033FC0F4BA063036024
:10AA10000E4B012243600E4B83600B238381002386
:10AA200002614361A46B0B4A206961690A4BFDF71F
:10AA3000F7FC012200238018594120616161480020
:10AA4000400810BD680000200E33CDAB34126DE617
:10AA5000ECDE05002D7F954C2DF451580CB430B52B
:10AA6000164B9DB00C1E1D6808DA8B2301202B604D
:10AA700040421DB030BC08BC02B01847822302A976
:10AA80009B008B810023029008619C4200D0631ED2
:10AA90008B604B6101235B42CB81209A21AB280064
:10AAA000019300F03DFD431C01DA8B232B60002C49
:10AAB000DFD00023029A1370DBE7C0466800002055
:10AAC0000EB400B50B499CB01DAB029006900791E7
:10AAD00004910948094904CB0591006802A9019332
:10AAE00000F01EFD0023029A13701CB008BC03B0D6
:10AAF0001847C046FFFFFF7F680000200802FFFFE5
:10AB0000020010B51378541C002B05D1CC5CD45432
:10AB10000133002CFAD110BD2200F3E702780B7844
:10AB2000002A03D0013001319A42F7D0D01A704781
:10AB300003000A7801311A700133002AF9D17047F5
:10AB40000023C25C0133002AFBD1581E704730B588
:10AB50000500002A00D130BD0C78013A6B1C2C7026
:10AB60000131002C05D19A189A42F4D01C7001339F
:10AB7000FAE71D00EDE710B50378002B0FD10B7835
:10AB80005A4253415B42184010BD0023CA5C002A60
:10AB9000FAD0C45C944201D10133F7E70130037865
:10ABA000002BF2D11800EFE7F0B51F000E0087B0C0
:10ABB0000590019102920C98347800F0EAFA08228C
:10ABC00000194378751C134036D12D2C36D1B51C95
:10ABD00074780126002F62D0102F09D1302C07D1B4
:10ABE00020222B789343582B54D110276C780235B0
:10ABF0002D4B3900F31818000393FDF7D5FA049193
:10AC000001210023494202008C46180021003039FE
:10AC100009291AD80C00A74223DD591C09D0634624
:10AC2000824206D302D10499A14202DB0123784378
:10AC300020182C780135E9E72E00BCE72B2C01D039
:10AC40001E00C7E7B51C7478FAE7210041391929BD
:10AC500001D8373CDFE721006139192901D8573C79
:10AC6000D9E75A1C08D1059A23331360029B039835
:10AC7000002B09D107B0F0BD002E00D04042029A4F
:10AC8000002AF7D0002B01D06B1E0193029B019A82
:10AC90001A60EFE73024002FAAD10827A8E7302C4C
:10ACA0009ED00A27A4E7C046FFFFFF7F37B51300F9
:10ACB000064A05001068046A002C00D1044C0A0002
:10ACC00000942900FFF770FF3EBDC04668000020D9
:10ACD000CC000020F8B505000E001400002804D0B8
:10ACE0008369002B01D100F0C1F9224B9C422DD188
:10ACF0006C68A369A360A3891B0731D52369002B66
:10AD00002ED023682269F7B2981A6369F6B283429B
:10AD100005DC2100280000F03BF9002826D1A368BB
:10AD20000130013BA36023685A1C22601F706369D5
:10AD3000834204D0A389DB071AD50A2E18D121003B
:10AD4000280000F025F9002812D00FE00A4B9C42A1
:10AD500001D1AC68CDE7094B9C42CAD1EC68C8E789
:10AD60002100280000F00CF80028CAD00126764205
:10AD70003000F8BD64CF000084CF000044CF000055
:10AD8000364B70B51D6806000C00002D05D0AB6970
:10AD9000002B02D1280000F069F9314B9C420FD101
:10ADA0006C680C23E25E93B219072DD4D90611D436
:10ADB00009230120336037331343A381404270BD20
:10ADC000284B9C4201D1AC68EBE7274B9C42E8D171
:10ADD000EC68E6E75B0713D5616B002908D0230018
:10ADE0004433994202D0300000F06AFA00236363D2
:10ADF0002422A3899343A3810023636023692360F2
:10AE00000823A2891343A3812369002B0BD1A0211E
:10AE10008022A389890092000B40934203D0210035
:10AE2000300000F0E1F90123A289134011D0002382
:10AE3000A36063695B42A361002023698342BED1A2
:10AE40000C23E25E1306BAD540231343A3810138D5
:10AE5000B5E7920700D46369A360EDE768000020BE
:10AE600064CF000084CF000044CF000010B506205E
:10AE700000F090FC012000F0CFFD0000F7B58A89BA
:10AE800005000C00130760D44B68002B04DC0B6C2E
:10AE9000002B01DC0020FEBDE76A002FFAD0002362
:10AEA0002E682B6080235B01216A1A4034D0606DCC
:10AEB000A3895B0706D56368C01A636B002B01D0BA
:10AEC000236CC01A0200216A00232800E76AB847F1
:10AED000A189431C06D12B681D2B30D82B4ADA40A0
:10AEE000D3072CD50023636023692360CB0405D5E9
:10AEF000431C02D12B68002B00D16065616B2E6072
:10AF00000029C7D023004433994202D0280000F022
:10AF1000D7F900206063BEE701232800B847431C2F
:10AF2000C6D12B68002BC3D01D2B01D0162B01D10D
:10AF30002E60AFE74023A2891343A381ABE74023F0
:10AF40000B430120A3814042A5E70F69002FA1D048
:10AF50000B680F60DB1B01930023920700D14B6944
:10AF6000A360019B002B00DC94E7019B3A00216A5F
:10AF70002800A66AB047002803DC4023A2891343B7
:10AF8000DFE7019B3F181B1A0193EAE7010040200D
:10AF90000B6970B505000C00002B01D1002070BDBD
:10AFA000002804D08369002B01D100F05FF80B4B1F
:10AFB0009C4209D16C680C22A35E002BEED02100CC
:10AFC0002800FFF75BFFEAE7054B9C4201D1AC6824
:10AFD000F1E7044B9C42EED1EC68ECE764CF000053
:10AFE00084CF000044CF0000002310B504000360AC
:10AFF0004360836081814366C281036143618361F1
:10B00000190008225C30FFF717FA054B24626362CF
:10B01000044BA362044BE362044B236310BDC046A0
:10B02000D5B70000FDB7000035B8000061B80000DA
:10B0300010B5024900F08CF810BDC04691AF000079
:10B0400070B568254A1E55430E002900743100F082
:10B0500081F9041E08D000212A00016046600C30EE
:10B06000A0606832FFF7E8F9200070BD836913B56E
:10B070000400002B28D18364C3640365134B144A76
:10B080001B6882620193984201D1012383612000F1
:10B0900000F020F86060200000F01CF8A0602000A4
:10B0A00000F018F80022E06004216068FFF79CFFC0
:10B0B00001220921A068FFF797FF02221221E06810
:10B0C000FFF792FF0123A36113BDC0460CCF000020
:10B0D00031B00000F8B51C4B07001E68B369002BA7
:10B0E00002D13000FFF7C2FF4836B4687368013BF5
:10B0F00004D53368002B07D03668F6E70C22A55E2E
:10B10000002D0DD06834F2E704213800FFF798FFD6
:10B1100030600028F0D10C2304003B602000F8BD13
:10B1200020000A4B656625606560A560E3602561C7
:10B130006561A561082229005C30FFF77DF9656330
:10B14000A563A564E564E9E70CCF00000100FFFFFB
:10B15000F7B504000700002601914834002C01D106
:10B160003000FEBD6368A5680093009B013B00931F
:10B1700001D52468F2E7AB89012B08D90E22AB5E1A
:10B18000013304D029003800019B984706436835F5
:10B19000EBE7EC300068704770B50E001D000E2321
:10B1A000C95E96B01400002907DA00232B60B3892A
:10B1B0001B0611D48023DB000FE06A4600F088FBF9
:10B1C0000028F2DBF022019B12021340054A9B1873
:10B1D0005A4253412B60EDE740230020236016B014
:10B1E00070BDC04600E0FFFFF7B502268B89050061
:10B1F0000C00334206D02300473323602361012330
:10B200006361F7BD01AB6A46FFF7C6FF009907000F
:10B21000280000F09FF8002808D10C22A35E9A05B0
:10B22000EFD4032293431E43A681E4E70F4BAB62A6
:10B230008023A28920601343A381009B2061636166
:10B24000019B002B0DD00E23E15E280000F052FB85
:10B25000002806D00322A38993431A000123134335
:10B26000A381A0893843A081CBE7C04631B000005C
:10B2700010B5034B0100186800F06CF810BDC04613
:10B280006800002082B0002900D101A9101E06D05C
:10B29000002B06D013780B601078431E984102B043
:10B2A000704702204042FAE7C9B28218904201D1A9
:10B2B0000020704703788B42FBD00130F6E7000096
:10B2C00070B50500002910D00C1F2368002B00DA90
:10B2D000E418280000F034FB1D4A1368002B05D148
:10B2E00063601460280000F02CFB70BDA34209D9F4
:10B2F000216860188342F3D118685B6841182160A7
:10B30000EEE713005A68002A01D0A242F9D9196861
:10B310005818A0420BD120680918581819608242A9
:10B32000E0D110685268411819605A60DAE7A0420B
:10B3300002D90C232B60D5E721686018824203D123
:10B34000106852684118216062605C60CAE7C046BC
:10B35000E41B0020032370B5CD1C9D430835060077
:10B360000C2D1ED20C25A9421DD8300000F0E8FAA1
:10B37000254A14682100002919D1244C2368002B88
:10B3800003D1300000F0CAF920602900300000F03D
:10B39000C5F9431C2BD10C233000336000F0D1FAE7
:10B3A00003E0002DDFDA0C233360002070BD0B6852
:10B3B0005B1B19D40B2B03D90B60CC18256003E061
:10B3C0004B688C420DD11360300000F0BAFA2000B7
:10B3D00007220B30231D9043C31AE7D05A42E25094
:10B3E000E4E763600C00EFE70C004968C3E7032360
:10B3F000C41C9C43A042E1D0211A300000F08EF919
:10B40000431CDBD1C7E7C046E41B0020E81B00203B
:10B41000F8B507000D001600002905D11100FFF74F
:10B4200099FF04002000F8BD002A03D1FFF748FF70
:10B430003400F7E700F086FA2C00B042F2D2310077
:10B440003800FFF787FF041EECD029003200FEF71A
:10B45000D7FF29003800FFF733FFE3E7F0B58E6828
:10B4600085B007000C00039201939E423CD89023C4
:10B470008A89DB001A4234D00325096923685B1AE4
:10B480000293636902985D43EB0F5D19019B6D1098
:10B4900001331B18AB4200D91D00530532D52900DA
:10B4A0003800FFF757FF061E09D10C233B604023ED
:10B4B0000120A28940421343A38105B0F0BD029A46
:10B4C0002169FEF79DFFA389144A1A408023134384
:10B4D000A381029B2661F61826606561019EED1A24
:10B4E000A560019B9E4200D9019E3200039920680D
:10B4F000FEF78FFFA36800209B1BA36023689E19A3
:10B500002660DAE72A003800FFF782FF061EE0D146
:10B5100021693800FFF7D4FEC7E7C0467FFBFFFF75
:10B52000F0B59FB0029005938B890F0016001B06A3
:10B5300011D50B69002B0ED14021FFF70BFF3860AE
:10B540003861002805D10C23029A013813601FB01E
:10B55000F0BD40237B61002306AC6361203363763A
:10B560001033A37635002B78002B01D0252B46D144
:10B57000AB1B04930CD0320039000298FFF76EFF2A
:10B58000431C00D1AEE06269049B9446634463614E
:10B590002B78002B00D1A5E00122002352426260EB
:10B5A00002A9543252186E1C2360E360A36013702A
:10B5B000A365317805225448FFF776FE751C0028F4
:10B5C0001FD12268D30604D5532302A95B1820217A
:10B5D0001970130704D5532302A95B182B21197086
:10B5E00033782A2B16D0350000210A20E3682A7808
:10B5F0006E1C303A092A4ED9002918D010E00135C6
:10B60000B1E7414B2268C01A0123834013432360F2
:10B610002E00CEE7059B191D1B680591002B01DB51
:10B62000099304E05B42E3600223134323602B7819
:10B630002E2B0AD16B782A2B35D1059B02351A1D8A
:10B640001B680592002B2BDB0793304E29780322D1
:10B650003000FFF729FE002806D04023801B8340DE
:10B6600022680135134323602978062228486E1C7E
:10B670002176FFF719FE00283CD0264B002B25D160
:10B680000722059B07339343083305936369039AA5
:10B690009B18636166E7434301219B183500A6E7C9
:10B6A00001235B42D0E700230A201A0001356360C2
:10B6B00029786E1C3039092903D9002BC5D007928F
:10B6C000C3E74243012352183500F1E705AB00936D
:10B6D0003A00114B2100029800E000BF0390039B49
:10B6E0000133D3D1BB890B985B0600D42FE701202F
:10B6F00040422CE705AB00933A00074B210002982B
:10B70000FFF74EF8EAE7C04610CF000016CF000062
:10B710001ACF0000000000005DB40000002370B5E7
:10B72000064C05000800236000F060F9431C03D1BB
:10B730002368002B00D02B6070BDC0469C2F0020DA
:10B7400070B504000D001F2904D9162303600120E1
:10B75000404270BD436C002B04D08A009B181A68CD
:10B76000002A08D1200000F031F82A000100200052
:10B7700000F01AF8EDE70020012AEAD0511C03D1AD
:10B78000162301302360E4E7002428001C60904762
:10B790002000DEE710B5034B01001868FFF7D0FF6B
:10B7A00010BDC04668000020002370B5064C05009F
:10B7B00008001100236000F001F9431C03D1236845
:10B7C000002B00D02B6070BD9C2F002010B500F026
:10B7D000E5F810BD70B50C000E25495F00F0BAF811
:10B7E000002803DB636D1B18636570BDA389024AE3
:10B7F0001340A381F9E7C046FFEFFFFFF8B51F0034
:10B800008B8905000C001600DB0505D50E23C95EEB
:10B810000022022300F080F8A389054A2800134083
:10B82000A38132000E23E15E3B0000F02BF8F8BD4F
:10B83000FFEFFFFF70B50C000E25495F00F06CF8BC
:10B84000A389421C03D1054A1340A38170BD802205
:10B8500052011343A3816065F8E7C046FFEFFFFF85
:10B8600010B50E23C95E00F021F810BD0B1E04D0E8
:10B87000FF2A04D98A2303608B3B180070470A70A3
:10B880000123FAE770B50500080011000022064CFC
:10B8900022601A0000F0B8F8431C03D12368002B83
:10B8A00000D02B6070BDC0469C2F0020002370B5D7
:10B8B000064C05000800236000F060F8431C03D12B
:10B8C0002368002B00D02B6070BDC0469C2F002049
:10B8D000002370B5064C050008001100236000F03D
:10B8E00055F8431C03D12368002B00D02B6070BD9A
:10B8F0009C2F0020002370B5064C05000800236033
:10B9000000F054F8431C03D12368002B00D02B60B7
:10B9100070BDC0469C2F002070B5050008001100C6
:10B920000022064C22601A0000F050F8431C03D19C
:10B930002368002B00D02B6070BDC0469C2F0020D8
:10B94000704770470B1F1B68181F002B01DA0B583C
:10B95000C018704770B50500080011000022064CA1
:10B9600022601A0000F03AF8431C03D12368002B30
:10B9700000D02B6070BDC0469C2F002058220120B3
:10B98000014B40421A6070479C2F00205822012032
:10B99000014B40421A6070479C2F00205822012022
:10B9A000014B40421A6070479C2F00205822024BE6
:10B9B00000201A607047C0469C2F002058220120AA
:10B9C000014B40421A6070479C2F002058220120F2
:10B9D000014B40421A6070479C2F002058220120E2
:10B9E000014B40421A6070479C2F0020044A1368A4
:10B9F000002B00D1034B1818106018007047C04688
:10BA0000EC1B0020A02F002058220120014B4042B7
:10BA10001A6070479C2F0020FEE7C046F8B5C0466C
:10BA2000F8BC08BC9E467047F8B5C046F8BC08BCD8
:10BA30009E4670476461746100000000B0BA000067
:10BA4000EB010000B9BA000017040000C1BA000001
:10BA50002D070000C8BA00003D080000CDBA000064
:10BA6000DF020000D8BA000083040000DDBA000045
:10BA7000B5090000E9BA00001B020000F3BA00009B
:10BA80003506000001BB0000A105000072616E6474
:10BA90006F6D00616C6C006C6173740066616C7337
:10BAA00065007472756500252E3135732E2E2E00BB
:10BAB0006D616B654C697374006164644C6173748F
:10BAC0000064656C657465006A6F696E00636F7011
:10BAD0007946726F6D546F0066696E64006A6F69B3
:10BAE0006E537472696E677300756E69636F646517
:10BAF000417400756E69636F6465537472696E6733
:10BB000000667265654D656D6F727900CC0F00003F
:10BB1000DC0F0000F60F000074100000AC100000F5
:10BB2000E21000001A110000401100007C1100001A
:10BB3000BE1100001412000058120000C4120000D0
:10BB40000C130000321300006A130000B013000051
:10BB5000D613000004140000361400006E14000018
:10BB6000F2140000BA150000301600009C16000008
:10BB7000F01600001017000032170000E417000054
:10BB80002A180000A2180000CC0F0000CC0F000003
:10BB9000D018000038190000BC190000021A00007B
:10BBA0004A1A0000BC1A00002E1B0000761B000081
:10BBB000BC1B0000F21B0000381C00007E1C0000B3
:10BBC000C61C00001A1D0000781D0000B61D0000F4
:10BBD000201E0000561E00009E1E0000E61E0000F3
:10BBE0002E1F0000681F0000B01F0000F81F00009B
:10BBF000CC0F0000CC0F0000CC0F00006020000034
:10BC0000CC0F000096200000C2200000F8200000A9
:10BC100024210000CC0F0000CC0F0000CC0F00004E
:10BC2000CC0F00005A210000A6210000CC0F00001C
:10BC3000CC0F0000EC2100003C220000622200003A
:10BC4000CC0F0000CC0F0000CC0F000090220000B1
:10BC5000C0220000F0220000262300005023000034
:10BC600086230000B0230000D82300000024000039
:10BC700030240000602400008A240000B424000066
:10BC8000E42400000E250000CC0F0000CC0F0000C3
:10BC9000CC0F0000CC0F0000CC0F00003E250000B0
:10BCA00084250000B0250000DC25000008260000E7
:10BCB0003E26000074260000AA260000E0260000B0
:10BCC0000C270000382700006E270000CC0F000072
:10BCD000CC0F0000CC0F0000CC0F0000CC0F0000F8
:10BCE000CC0F0000CC0F0000CC0F0000CC0F0000E8
:10BCF000CC0F0000CC0F0000CC0F0000CC0F0000D8
:10BD0000CC0F00009A270000D027000028256420CF
:10BD10006974656D206C6973742900286F626A65A7
:10BD2000637420747970653A202564290053746126
:10BD3000636B20756E646572666C6F77000000003F
:10BD4000070000000300000089BD0000B5280000C6
:10BD500091BD0000B92800009ABD0000B128000084
:10BD6000A3BD0000BD280000150000000100000078
:10BD700002000000040000000500000006000000B2
:10BD800043616C6C696F706500686173546F6E65B8
:10BD900000706C6179546F6E6500686173536572F1
:10BDA000766F00736574536572766F004743207435
:10BDB0006F6F6B2025642075736563733B2066721B
:10BDC000656520256420776F726473003C496E744A
:10BDD000656765723E003C4F626A6563743E003C75
:10BDE0004C6973743E000D0A564D2050616E6963B4
:10BDF0003A2025730D0A006D697363000CBE0000C4
:10BE00007D31000015BE00003531000068657854B2
:10BE10006F496E740073696E0000000068BE000018
:10BE2000E931000070BE0000ED3100007ABE000074
:10BE30000B32000083BE0000153200008EBE0000F1
:10BE40001F3200009ABE000029320000ABBE000085
:10BE500033320000C1BE0000F7310000DABE00003E
:10BE6000013200006E6574006861735769466900AD
:10BE70007374617274576946690073746F7057699F
:10BE800046690077696669537461747573006D79EA
:10BE9000495041646472657373007468696E6744E5
:10BEA00065736372697074696F6E00636C6561724B
:10BEB0005468696E674465736372697074696F6E04
:10BEC00000617070656E64546F5468696E67446594
:10BED000736372697074696F6E00617070656E640F
:10BEE000546F5468696E6750726F70657274790030
:10BEF0000D0E0F04050C0B0A0607080900000000D0
:10BF00000008080800080A4A4000000A5FEA5FEAE1
:10BF10000ED92ED36E19324489330C924C924D08AF
:10BF20000800000004880808040804848488000AC3
:10BF3000448A4000048EC480000000048800000E83
:10BF4000C000000000080001224488100C925252E8
:10BF50004C048C84848E1C824C901E1EC244924CD5
:10BF600006CA525FE21FF01EC13E02448ED12E1F50
:10BF7000E24488100ED12ED12E0ED12EC488000896
:10BF800000080000048004880244880482000EC077
:10BF90000EC008048244880ED126C0040ED135B3E9
:10BFA0006C0C925ED2521C925C925C0ED010100E01
:10BFB0001C9252525C1ED01C901E1ED01C90100E63
:10BFC000D013712E12525ED2521C8808081C1FE238
:10BFD00042524C1254981492101010101E113B75BE
:10BFE000B131113935B3710C9252524C1C925C90A4
:10BFF000100C92524C861C925C92510ED00C825CBA
:10C000001FE4848484125252524C1131312A44115B
:10C010003135BB7112524C9252112A4484841EC491
:10C0200088101E0EC808080E10080482410EC24275
:10C03000424E048A400000000000001F08048000F7
:10C0400000000ED2524F10101C925C000ED0100E49
:10C0500002424ED24E0C925C900E06C81C88080E0E
:10C06000D24EC24C10101C92520800080808024020
:10C0700002424C10149814920808080806001B7518
:10C08000B131001C925252000C92524C001C925C36
:10C0900090000ED24EC2000ED010100006C80498B8
:10C0A00008080EC807001252524F0011312A4400EE
:10C0B000113135BB00124C8C9200112A4498001E9D
:10C0C000C4881E06C48C8486080808080818080C52
:10C0D000881800000C8360000000000001000000D0
:10C0E0000200000003000000040000000500000042
:10C0F0000600000007000000080000000900000022
:10C100000A0000000B0000000C0000000D00000001
:10C110000E0000000F0000001000000012000000E0
:10C120001400000016000000180000001A000000B3
:10C130001C0000001E000000200000002300000082
:10C1400026000000290000002C0000002F00000045
:10C1500032000000360000003A0000003E000000FF
:10C1600042000000460000004B00000050000000AC
:10C17000550000005A000000610000006800000047
:10C180006F000000760000007D00000084000000C9
:10C190008B0000009200000099000000A000000049
:10C1A000A7000000AE000000B5000000BC000000C9
:10C1B000C3000000CA000000D1000000D800000049
:10C1C000DF000000E6000000ED000000F4000000C9
:10C1D000FB000000FF00000028C2000059320000F0
:10C1E00033C20000813700003DC2000091340000DE
:10C1F0004AC20000B134000051C200000135000005
:10C200005AC200005135000066C200002D34000003
:10C2100077C200009136000084C200004D37000054
:10C22000646973706C6179006C696768744C6576D9
:10C23000656C006D62446973706C6179006D624475
:10C240006973706C61794F6666006D62506C6F74D3
:10C25000006D62556E706C6F74006D624472617730
:10C260005368617065006D625368617065466F72F6
:10C270004C6574746572006E656F506978656C53B7
:10C28000656E64006E656F506978656C53657450B7
:10C29000696E004E6F7420656E6F75676820726FEF
:10C2A0006F6D206576656E20616674657220636FC0
:10C2B0006D70616374696F6E00436F6D706163745C
:10C2C000656420466C61736820636F6465207374D5
:10C2D0006F72650A256420627974657320757365D1
:10C2E0006420282564252529206F662025640042C6
:10C2F0006164207265636F726420666F756E64207E
:10C30000647572696E6720696E697469616C697AB7
:10C310006174696F6E0025642025642025642028DF
:10C32000256420776F726473290025642072656329
:10C330006F7264732C20256420776F7264732C20D5
:10C340006D617849442025642C20636F6D706163B2
:10C3500074696F6E206379636C6573202564005285
:10C360006573746F726564202564207363726970ED
:10C370007473005374617274656400726164696FF0
:10C380000000000012C40000514100001FC4000062
:10C39000C14300002FC40000614300003DC4000001
:10C3A0004145000048C400006941000058C4000035
:10C3B000DD4100006CC40000794100007BC4000036
:10C3C0002347000087C40000A146000090C400007D
:10C3D000454600009BC400008D450000A6C4000037
:10C3E000C9450000AFC40000FD450000B8C400000E
:10C3F0008D4100006E756D626572006E6F6E650036
:10C400006F74686572007061697200737472696E2E
:10C41000670064697361626C65526164696F006D85
:10C4200065737361676552656365697665640070FD
:10C4300061636B65745265636569766500706163FD
:10C440006B657453656E64007265636569766564D7
:10C45000496E7465676572007265636569766564C7
:10C460004D657373616765547970650072656365C6
:10C4700069766564537472696E670073656E6449AA
:10C480006E74656765720073656E645061697200F1
:10C4900073656E64537472696E6700736574436884
:10C4A000616E6E656C0073657447726F75700073B2
:10C4B0006574506F776572007369676E616C537451
:10C4C00072656E67746800000000000096300777A0
:10C4D0002C610EEEBA51099919C46D078FF46A7078
:10C4E00035A563E9A395649E3288DB0EA4B8DC7998
:10C4F0001EE9D5E088D9D2972B4CB609BD7CB17E18
:10C50000072DB8E7911DBF906410B71DF220B06AE7
:10C510004871B9F3DE41BE847DD4DA1AEBE4DD6DF7
:10C5200051B5D4F4C785D38356986C13C0A86B64F7
:10C530007AF962FDECC9658A4F5C0114D96C066317
:10C54000633D0FFAF50D088DC8206E3B5E10694CF7
:10C55000E44160D5727167A2D1E4033C47D4044B37
:10C56000FD850DD26BB50AA5FAA8B5356C98B24217
:10C57000D6C9BBDB40F9BCACE36CD832755CDF4597
:10C58000CF0DD6DC593DD1ABAC30D9263A00DE51C7
:10C590008051D7C81661D0BFB5F4B42123C4B356B7
:10C5A0009995BACF0FA5BDB89EB802280888055F37
:10C5B000B2D90CC624E90BB1877C6F2F114C685897
:10C5C000AB1D61C13D2D66B69041DC760671DB0185
:10C5D000BC20D2982A10D5EF8985B1711FB5B60657
:10C5E000A5E4BF9F33D4B8E8A2C9077834F9000F97
:10C5F0008EA8099618980EE1BB0D6A7F2D3D6D0837
:10C60000976C6491015C63E6F4516B6B62616C1C26
:10C61000D83065854E0062F2ED95066C7BA5011B56
:10C62000C1F4088257C40FF5C6D9B06550E9B712F6
:10C63000EAB8BE8B7C88B9FCDF1DDD62492DDA15B6
:10C64000F37CD38C654CD4FB5861B24DCE51B53AD6
:10C650007400BCA3E230BBD441A5DF4AD795D83DD6
:10C660006DC4D1A4FBF4D6D36AE96943FCD96E3416
:10C67000468867ADD0B860DA732D0444E51D0333F6
:10C680005F4C0AAAC97C0DDD3C710550AA41022706
:10C6900010100BBE86200CC925B56857B3856F20D6
:10C6A00009D466B99FE461CE0EF9DE5E98C9D92936
:10C6B0002298D0B0B4A8D7C7173DB359810DB42E76
:10C6C0003B5CBDB7AD6CBAC02083B8EDB6B3BF9AC2
:10C6D0000CE2B6039AD2B1743947D5EAAF77D29D4E
:10C6E0001526DB048316DC73120B63E3843B64942E
:10C6F0003E6A6D0DA85A6A7A0BCF0EE49DFF09932E
:10C7000027AE000AB19E077D44930FF0D2A308879D
:10C7100068F2011EFEC206695D5762F7CB6765804D
:10C7200071366C19E7066B6E761BD4FEE02BD3894D
:10C730005A7ADA10CC4ADD676FDFB9F9F9EFBE8EAD
:10C7400043BEB717D58EB060E8A3D6D67E93D1A1ED
:10C75000C4C2D83852F2DF4FF167BBD16757BCA6CD
:10C76000DD06B53F4B36B248DA2B0DD84C1B0AAF6D
:10C77000F64A0336607A0441C3EF60DF55DF67A8ED
:10C78000EF8E6E3179BE69468CB361CB1A8366BC7D
:10C79000A0D26F2536E2685295770CCC03470BBBCD
:10C7A000B91602222F260555BE3BBAC5280BBDB2CD
:10C7B000925AB42B046AB35CA7FFD7C231CFD0B56D
:10C7C0008B9ED92C1DAEDE5BB0C2649B26F263EC5F
:10C7D0009CA36A750A936D02A906099C3F360EEB6D
:10C7E0008567077213570005824ABF95147AB8E22D
:10C7F000AE2BB17B381BB60C9B8ED2920DBED5E50D
:10C80000B7EFDC7C21DFDB0BD4D2D38642E2D4F15C
:10C81000F8B3DD686E83DA1FCD16BE815B26B9F6EC
:10C82000E177B06F7747B718E65A0888706A0FFF4C
:10C83000CA3B06665C0B0111FF9E658F69AE62F80C
:10C84000D3FF6B6145CF6C1678E20AA0EED20DD70C
:10C850005483044EC2B30339612667A7F71660D02C
:10C860004D476949DB776E3E4A6AD1AEDC5AD6D96C
:10C87000660BDF40F03BD83753AEBCA9C59EBBDE8C
:10C880007FCFB247E9FFB5301CF2BDBD8AC2BACA3C
:10C890003093B353A6A3B4240536D0BA9306D7CDAC
:10C8A0002957DE54BF67D9232E7A66B3B84A61C4CC
:10C8B000021B685D942B6F2A37BE0BB4A18E0CC38C
:10C8C0001BDF055A8DEF022D416C6C207461736B78
:10C8D000732073746F707065640076303732002097
:10C8E0002573202573004D656D6F727920636C652B
:10C8F00061726564004E6F206672656520746173B5
:10C900006B20656E747269657300000054C9000085
:10C910005959000061C90000BF5900006DC90000ED
:10C920008F59000073C900009F59000079C90000A9
:10C93000AF5900007FC900008D56000089C9000072
:10C94000DD59000091C90000B957000073656E738E
:10C950006F727300616363656C65726174696F6E99
:10C960000074656D70657261747572650074696CD0
:10C9700074580074696C74590074696C745A00744A
:10C980006F75636852656164006932635265616402
:10C9900000693263577269746500000010CA0000B4
:10C9A0005D5A00001ECA0000615A000027CA00003C
:10C9B0006D5A000031CA0000715A00003ACA0000E6
:10C9C000755A00003FCA0000795A000044CA0000AE
:10C9D0007D5A000050CA0000815A000057CA00006A
:10C9E000855A000060CA0000895A000065CA00002C
:10C9F0008D5A000070CA0000915A00007ACA0000E7
:10CA0000655A000084CA0000695A00007466740008
:10CA1000656E61626C65446973706C61790067650D
:10CA200074576964746800676574486569676874F9
:10CA300000736574506978656C006C696E6500728E
:10CA400065637400726F756E64656452656374002B
:10CA5000636972636C6500747269616E676C65000E
:10CA60007465787400746674546F756368656400E7
:10CA7000746674546F7563685800746674546F7587
:10CA800063685900746674546F7563685072657397
:10CA9000737572650057656C636F6D6520746F20E8
:10CAA0004D6963726F426C6F636B732100705F73CB
:10CAB000706920213D204E554C4C002F686F6D65EC
:10CAC0002F62726F6D61676F73612F2E706C61746E
:10CAD000666F726D696F2F7061636B616765732F2D
:10CAE0006672616D65776F726B2D61726475696EC8
:10CAF0006F6E6F726469636E7266352F6C696272F5
:10CB000061726965732F5350492F5350492E6370DA
:10CB10007000535049436C6173733A3A5350494320
:10CB20006C617373284E52465F5350495F5479705D
:10CB3000652A2C2075696E74385F742C2075696EB7
:10CB400074385F742C2075696E74385F7429000026
:10CB50000000000000000000955C0000515C000037
:10CB6000775C0000815C00008B5C0000755C00005D
:10CB7000000000000100000002000000160000009C
:10CB8000040000000500000006000000070000008F
:10CB900008000000090000000A0000000B0000006F
:10CBA0000C0000000D0000000E0000000F0000004F
:10CBB0001A0000001B000000140000001300000019
:10CBC0001100000003000000100000001C00000025
:10CBD0001D0000001E0000001200000015000000F3
:10CBE00017000000180000001900000000000000FD
:10CBF000000000004561000075680000C56100008C
:10CC0000D9610000CF610000416100003561000082
:10CC1000E56100006161000031610000000000007A
:10CC2000000000000000304300000000000030C39E
:10CC30007371727400000000FB21F93FFB21094071
:10CC40007CD91240FB2119407A6A1F407CD92240CE
:10CC5000BBFD2540FB2129403A462C407A6A2F40F3
:10CC60005C4731407CD932409C6B3440BBFD354041
:10CC7000DB8F3740FB2139401BB43A403A463C40F9
:10CC80005AD83D407A6A3F404C7E40405C47414024
:10CC90006C1042407CD942408CA243409C6B444083
:10CCA000AC344540BBFD4540CBC64640DB8F4740DA
:10CCB000EB584840FB21494083F9A200444E6E00E6
:10CCC000FC291500D1572700DD34F50062DBC000D8
:10CCD0003C999500419043006351FE00BBDEAB00E0
:10CCE000B761C5003A6E2400D24D42004906E0000B
:10CCF00009EA2E001C92D100EB1DFE0029B11C0098
:10CD0000E83EA700F535820044BB2E009CE9840074
:10CD1000B4267000417E5F00D691390053833900FC
:10CD20009CF439008B5F840028F9BD00F81F3B009C
:10CD3000DEFF97000F980500112FEF000A5A8B00B5
:10CD40006D1F6D00CF7E360009CB2700464FB70020
:10CD50009E663F002DEA5F00BA277500E5EBC7002D
:10CD60003D7BF100F739070092528A00FB6BEA0025
:10CD70001FB15F00085D8D00300356007BFC46004C
:10CD8000F0AB6B0020BCCF0036F49A00E3A91D0085
:10CD90005E619100081BE60085996500A0145F00A4
:10CDA0008D40680080D8FF0027734D0006063100D3
:10CDB000CA561500C9A873007BE260006B8CC000E6
:10CDC00000000040FB21F93F000000002D44743EAC
:10CDD000000000809846F83C0000006051CC783B91
:10CDE00000000080831BF0390000004020257A38C5
:10CDF000000000802282E336000000001DF3693548
:10CE00000200000003000000040000000600000013
:10CE10006C85000016850000168500004486000021
:10CE200012850000128500003A860000448600004A
:10CE3000128500003A86000012850000448600003A
:10CE400048860000488600004886000050860000A2
:10CE500048900000BA8E0000FE8E0000628E000036
:10CE6000FE8E0000EE8F0000FE8E0000628E00003D
:10CE7000BA8E0000BA8E0000EE8F0000628E0000B5
:10CE80005A8E00005A8E00005A8E0000FC8F00005F
:10CE90007097000072960000729600009099000052
:10CEA0006C9600006C960000789900009099000044
:10CEB0006C960000789900006C9600009099000034
:10CEC00086990000869900008699000094990000D8
:10CED0002C2066756E6374696F6E3A2000617373FF
:10CEE000657274696F6E2022257322206661696CF9
:10CEF00065643A2066696C6520222573222C206CBB
:10CF0000696E65202564257325730A006C00002076
:10CF1000232D302B2000686C4C0065666745464722
:10CF200000303132333435363738394142434445A5
:10CF30004600303132333435363738396162636414
:10CF40006566000000000000000000000000000016
:10CF500000000000000000000000000000000000D1
:10CF600000000000000000000000000000000000C1
:10CF700000000000000000000000000000000000B1
:10CF800000000000000000000000000000000000A1
:10CF90000000000000000000000000000000000091
:10CFA000000000004300504F53495800002020204B
:10CFB0002020202020202828282828202020202049
:10CFC0002020202020202020202020202088101019
:10CFD0001010101010101010101010101004040475
:10CFE0000404040404040410101010101010414133
:10CFF0004141414101010101010101010101010121
:10D000000101010101010101101010101010424234
:10D0100042424242020202020202020202020202F0
:10D020000202020202020202101010102000000090
:10D0300000000000000000000000000000000000F0
:10D0400000000000000000000000000000000000E0
:10D0500000000000000000000000000000000000D0
:10D0600000000000000000000000000000000000C0
:10D0700000000000000000000000000000000000B0
:10D0800000000000000000000000000000000000A0
:10D090000000000000000000000000000000000090
:10D0A0000000000000000000000000000000000080
:04D0B000000000007C
:08D0B4005430FF7F0100000071
:10D0BC00FFFFFFFF40060000010000001800000009
:10D0CC0019FCFFFFFFFFFFFF020000000300000040
:10D0DC00FFFFFFFF00000000010000000000020045
:10D0EC0001000000FFFFFFFF000000000200000035
:10D0FC000000040002000000FFFFFFFF0000000022
:10D10C000300000000000800030000000A000000FB
:10D11C0008000000010000006C000020000000006E
:10D12C0064CF000084CF000044CF0000000000005A
:10D13C0000000000000000000000000000000000E3
:10D14C0000000000000000000000000000000000D3
:10D15C0000000000000000000000000000000000C3
:10D16C0000000000000000000000000000000000B3
:10D17C000000000000000000000000004300000060
:10D18C000000000000000000000000000000000093
:10D19C000000000000000000000000004300000040
:10D1AC000000000000000000000000000000000073
:10D1BC000000000000000000000000004300000020
:10D1CC000000000000000000000000000000000053
:10D1DC000000000000000000000000004300000000
:10D1EC000000000000000000000000000000000033
:10D1FC0000000000000000000000000043000000E0
:10D20C000000000000000000000000000000000012
:10D21C0000000000000000000000000043000000BF
:10D22C0000000000000000000000000000000000F2
:10D23C00000000000000000000000000430000009F
:10D24C0000000000000000000000000000000000D2
:10D25C000000000000000000000000006DB800009D
:10D26C0085B2000000000000ACCF0000AEBA000098
:10D27C00F6BD0000F6BD0000F6BD0000F6BD0000D6
:10D28C00F6BD0000F6BD0000F6BD0000F6BD0000C6
:10D29C00F6BD0000FFFFFFFFFFFFFFFFFFFFFFFFDB
:10D2AC00FFFF00000100415343494900000000000A
:10D2BC000000000000000000000000000000000062
:10D2CC0000000000000041534349490000000000E9
:10D2DC000000000000000000000000000000000042
:10D2EC000000000000000000E9000000215C0000CC
:0CD2FC00695F000091640000C1000000A8
:040000030000600594
:00000001FF
